:020000040800F2
:1000000000A0002059D6000831A300089DC70008B1
:100010002FA300082DA300082BA300080000000058
:1000200000000000000000000000000029A30008FC
:1000300027A300080000000025A30008157C000885
:10004000C1D60008C1D60008C1D60008C1D6000834
:10005000C1D60008C1D60008C1D60008C1D6000824
:10006000C1D60008C1D60008C1D60008C1D6000814
:10007000C1D600081DA00008D7970008C1D6000807
:10008000C1D60008C1D60008C1D60008C1D60008F4
:1000900091A30008C1D60008C1D60008C1D6000847
:1000A00095940008C194000885940008D194000834
:1000B000B5940008A5940008C1D60008C1D6000870
:1000C000C1D60008C1D60008C1D60008C1D60008B4
:1000D000C1D600088D960008819600087596000824
:1000E000257C0008C1D6000805C70008C1D6000855
:1000F000C1D60008C1D60008C1D60008C1D6000884
:10010000000000000000000000000000C1D6000850
:10011000C1D60008C1D60008C1D60008C1D6000863
:10012000C1D60008C1D60008C1D60008C1D6000853
:10013000C1D60008C1D60008000000000000000081
:10014000C1D60008C1D60008C1D6000800000000D2
:10015000000000000000000000000000000000009F
:100160000000000000000000C1D60008C1D6000851
:10017000C1D60008000000000000000000000000E0
:0801800000000000C1D60008D8
:100188002DE9F04F2DED028B924D934B2B60A9B0CA
:1001980000236B6008F047FE18B908F067FE05F009
:1001A80019FE05F0D9FE8D4B8D4C1A7842F00102EC
:1001B8001A708C4A4FF47001C2F888100022099214
:1001C8000A92226842F4803222600493236803F47E
:1001D80000330A93099B013309930A9B1BB9099BB6
:1001E800B3F5A04FF2D1236813F4003318BF0123ED
:1001F8000A930A9B012B6FD07A4F7B4BFB60636A93
:10020800AB60636ADFF814A2DFF81482DFF8149297
:1002180043F080736362636943F4FC0328AE63614F
:1002280003238DF8523041F6FF7326F8503D4FF006
:100238009040314609F006FF4FF6FF7350463146AD
:10024800ADF8503009F0FEFE6848314609F0FAFE74
:100258006748314609F0F6FE6648314609F0F2FE75
:100268003146654809F0EEFE304604F021FF149B44
:10027800624AB3FBF2F3624A62491360624B00229E
:100288001A60624B5960F02187F823109A60604F1A
:1002980007221A60BB68C8F8003099E80F0086E8A2
:1002A8000F006369149843F480236361636943F41E
:1002B800802363611023CAF818302023CAF8183045
:1002C80015A909F0BFFE169817A909F0BBFED8F8C2
:1002D8000030180729D4A7E04E4B12221A60636831
:1002E800636063686360636843F480636360636842
:1002F80023F47C136360636843F4E8136360236842
:1003080043F0807323602268354B9101FBD55A680E
:1003180022F003025A605A6842F002025A60636887
:1003280003F00C03082BFAD166E797F89231012BFA
:100338007AD8D9F8100030603146504697F893B112
:1003480009F080FE0A2007F005FBBAF8103003F424
:1003580080539BB2002B67D11E4A9268D20040F1AD
:100368008784DB0760D52C4BDFF8B0A018684FF006
:10037800200BAAF828B0314614904FF0904009F0AD
:1003880061FE4FF0904308229A613C2007F0EDFA95
:10039800CAF818B04FF0000A97F893319A4543DA33
:1003A8001E4A4FF0904B1021082391617820069146
:1003B8000592ABF82830039307F0CCFA059A069912
:1003C800039B11857820CBF8183007F0C3FA0AF19F
:1003D800010AE1E77001002091560008BA220020C6
:1003E8000010024000ED00E00005FA050008004892
:1003F800000C0048001000480014004840420F005C
:10040800781100203F190100B411002010E000E02D
:10041800541A0020002002409006010800040048F9
:10042800242200207C060108642007F09EFAC822D6
:10043800CB4800210EF0C5FCE369CA4A43F0030328
:10044800E361A36943F4A123A361636943F4C0236F
:10045800636102F1B00C937B506892F80FE003F0EF
:100468000701DB0800EB83038900186A4FF00F0AC5
:100478000EFA01FE0AFA01F120EA01011962196A6D
:1004880010324EEA010162451962E4D10023DFF817
:100498000CA30AF10C020021995401330B2BF6D15D
:1004A800FF23B14A8AF817308AF818308AF81930C9
:1004B8008AF81A308AF81B30AC4BDFF8E4B21360C4
:1004C800AB4A039304201070584630220EF079FC92
:1004D800142202218BF800208BF824100122A54950
:1004E800039B8BF8182097F805B081F800B0A3F5A6
:1004F800EE71CAF81C10A049D8F80080A3F58E73D5
:100508000B609E4B03EBCB0318F0200F5B78CAF807
:10051800203018BFCAF820200023994A40F2DC5145
:1005280022F813100133082BF7D10DA800211C2243
:100538000EF047FCBBF10E0F03D00BF0EF03082BB6
:1005480002D101238DF84430022007F067F818B172
:100558004088003018BF0120C8F340038DF83A30B6
:10056800C8F380138DF83C30C8F340338DF834302D
:10057800C8F3C03300F001008DF8373018F4006379
:100588008DF8390007D097F8863103F1FF3EDEF188
:10059800000343EB0E038DF83830C8F300438DF8A1
:1005A8003D302B6AB7F84801ADF84800003318BF52
:1005B80001238DF83E30C8F300538DF83F30B7F86B
:1005C8004A31ADF8423018F4805FB7F8563118BF99
:1005D8006C48ADF84030C8F380438DF83B30B7F82D
:1005E80054311CBFB0F85001ADF84800B3F5FA7F9C
:1005F800ADF8463084BF0023ADF84830624897F81C
:10060800D63185F82430002385F8253043709DF8CD
:10061800443008F00101002BC8F3C0028DF83510F2
:100628008DF836200CBF0023022301B902B1013333
:1006380009EB83094FF0000AD9F818309A1E1433D1
:1006480003920593039A32F8023F03924FF6FF7222
:10065800934200F04581DAB2190A9DF839307BB12E
:10066800404B4A4F03EB02135868B84208D11B8924
:10067800B3F5806F00F02F81B3F5006F00F02B8188
:100688009DF83A3053B1374B03EB02135868B0F179
:10069800904F03D11B89102B00F01D81022902D134
:1006A8009DF8343003E0012904D19DF83530002B42
:1006B80000F011812B4F9DF83F304FEA02194F444B
:1006C80033B19DF844301BB9043A032A40F2EC8058
:1006D8000129CBB266D1FF2385F86C3085F86D30DF
:1006E800204BEF6703EB09024FF00008517B50687D
:1006F8008DF8521002F1080B1289ADF8502014A998
:10070800022285F8708006938DF8532085F828809A
:10071800C5F82C80C5F83080C5F83480C5F86880E5
:1007280085F86E8085F86F8009F08CFC069B9BF835
:10073800021053F80900424609F0B6FB38460AF0A1
:10074800A7FA134B1349C5F88030134BC5F884300A
:10075800C5F8888038460A1D08F02EFFBBE000BFA8
:10076800C80F0020881F01081C110020441C00200D
:1007780006040020680600200C11002078220108D9
:10078800F6030020541A00209501002000040048B8
:10079800699C0008F0010020499D000870010020B4
:1007A80020110020022B46D15FFA8AF21C2101FB9E
:1007B80002FC05EB0C089B4A88F871A0012188F817
:1007C800701002EB09014FF0000B91F80DE048683A
:1007D80088F872B001F108020989ADF8501088F85C
:1007E8007AB014A9C8F87C70CDF81CC08DF852E016
:1007F80006928DF8533009F025FC8A4B069A53F877
:10080800090091785A4609F04FFB38460AF040FA39
:10081800DDF81CC08449854AC8F880206144844AB0
:10082800C8F88420C8F888B038460A1D08F0C4FE05
:100838000AF1010A4FE0032B34D19DF83B30DFF871
:100848002C823BB195F82690384608214FF6FF7266
:1008580000231BE0BDF846207649BDF8483091F8E2
:100868002690B2F5FA7F0BD97349B1FBF2F23846FC
:10087800082192B209F00FFC704B48F829000AE0F1
:100888006F49B1FBF2F23846012192B209F003FC3C
:100898006C4B48F82900C36095F82630013385F879
:1008A800263018E0042B16D195F82580BDF8402095
:1008B800634B93FBF2F23846BDF84230012192B205
:1008C80009F0E9FB95F8253005EB88080133C8F8ED
:1008D800500185F82530039B059A93427FF4B2AE08
:1008E80095F8252085F87021574A584B92F800E072
:1008F800AEF117020027022A1F709C461AD8EB692E
:100908003B44D3ED007AF5EE407AF1EE10FA02D1CD
:100918002B6A73BB26E04E4A07EB02080FCB88E828
:100928000F009CF8003010370133C02F8CF80030CE
:10093800E5D1EDE7474B13F83E908CF8009003EBB8
:10094800CE03D3F804A0BAF1000FE1D04F45DFDAA7
:100958003F4A3B0103EB020853440FCB013788E8B9
:100968000F00F3E73C4B03931A6812F4805F24D11D
:100978001DE03A4B3A4A13F83E00107003EBCE03E1
:100988005D68002DEED000238342EBDAC3EBC30190
:100998006A18DFF8DC80D2F8009041F8089001EB83
:1009A80008079188B9809279BA710133ECE70EF0A3
:1009B800EF03082B2B4B20D122E09CF80020012AC2
:1009C800F5D9294B03EB0212103210339342EED0C3
:1009D80053ED047AB6EE007A67EE877A43ED047A2F
:1009E80053ED057A67EE877A43ED057A53ED037A7E
:1009F80067EE877A43ED037AE7E7BEF10E0F09D178
:100A08001A7842F010021A70BEF1180F32D106F0AF
:100A18003BFB2FE01A7822F010021A70BEF1190F72
:100A2800F4E700BF881F0108F0010020AD9F00080F
:100A3800419C00087001002000127A00699D00089E
:100A480040420F00599D0008680600205B0F0020F7
:100A5800A405002078220108242200201C0B01088C
:100A680098100020920B0020AC050020980F002061
:100A78009910002006F0ECFA039B1B685D0358BF31
:100A8800AE4BAF4D5CBF01221A70049B049A1B78D1
:100A980043F0040313702023ADF8503011238DF870
:100AA800523063694FF0020843F4003331468DF841
:100AB80053804FF09040636109F0C4FAA14BA24AF9
:100AC8001A60002007F0B2F8A04B1D60636943F478
:100AD80000336361E36943F48003E361236B23F02C
:100AE80020032363236B43F080534FF0904743F078
:100AF800200323637B6A23F0F0037B627B6A43F065
:100B080040037B627B6A23F470637B627B6A43F4F5
:100B180080634FF000097B6231464FF400734FF059
:100B2800030A384614938DF856908DF857908DF82F
:100B380054808DF855A004F029FC4FF480633146A9
:100B48003846149304F022FC2B68814E23F00103ED
:100B58002B602A687F4B13402B607F4B2B612B68DF
:100B680043F001032B60C5F80890C5F80C90C5F850
:100B78000890AB6843F40043AB602B682B606B684C
:100B880023F0784323F400436B602B6843F00103A0
:100B98002B60039B4FF0100B1D68304649465A46A0
:100BA8000EF00FF905EA08054FF6FF730B938DF861
:100BB80031808DF832908DF833908DF830A065B182
:100BC80028A9384641F874BD04F0E0FB0125072345
:100BD800357086F80190F370B570E36A23F4F87302
:100BE800E362E36A43F4D873E362636943F08053D2
:100BF80043F002036361594C204604F0CDF9002309
:100C0800169318931E9319934FF480731A934FF405
:100C18008063534A1B932023204614921C93514A05
:100C280015924FF4005314A91D93ADF85C5004F0CD
:100C380095F9236843F0010323604B4CA36823F024
:100C48004053A360A36843F08053A3600A2006F0D2
:100C58008CFEA36823F08043A360A368A360A36805
:100C680043F00043A360A3683F4A002B08DAFAE781
:100C78000BF1FF33092B8CBF00230123FFF771BB56
:100C880093683A4923F040539360936843F00053C4
:100C980093608868364B034043F468338B60D168AF
:100CA800344B0B4043F40053D360136B013D23F0E6
:100CB8000F031D431563002401233219917800297D
:100CC80000F08B805D1C042B375DD078DFF898E04E
:100CD800EDB20ED803EB43035A00DEF830101F23A1
:100CE800934021EA030107FA02F30B43CEF83030B0
:100CF80050E0092B0ED8053B06225A43DEF8341083
:100D08001F23934021EA030107FA02F30B43CEF8AD
:100D180034303FE00E2B4FF006012DD8A3F10A0224
:100D28004A43DEF838C01F2393402CEA030107FA30
:100D380002F30B43CEF838302CE000BFD00A002075
:100D480000580040C422002029720008181A002008
:100D5800E40D0020FFE0CF007A25E00008040240FF
:100D680040010050F40D0020000100500003005025
:100D7800E010FCFF07C0FFFD0F3B01FB03F2DEF8AC
:100D88003CC01F2393402CEA030107FA02F30B43EC
:100D9800CEF83C30092FA34A0FD99369A7F10A036B
:100DA80003EB430397690721994027EA0101916101
:100DB80091699840084390610EE053697B1E03EBEC
:100DC800430357693821994027EA01015161516964
:100DD80003339840084350612B460434102C7FF4A9
:100DE8006CAF904B9A6842F001029A601A461168FB
:100DF8008C4BC807FBD5DA688B4C22F00202DA600C
:100E0800DA6842F00202DA60DA6842F00102DA6077
:100E18009A6842F004029A60B4F85C31002B40F002
:100E28007384B4F95E21002A40F06E84B4F960211D
:100E3800002A40F069847D4B7D4E1B687D48B3F8DD
:100E48005630049300210C22B4F8647194F863B10D
:100E5800B4F80C9094F80FA0DFF80C82764D0DF0E2
:100E6800B0FF3046002114220DF0ABFF002388F8B4
:100E78000030C5F8743108F0EDFA002833D06F4B14
:100E880033606F4B73606F4BF360B7F5807F6E4BC9
:100E980033616E4B01D1002216E0BB2F01D901222C
:100EA80012E0612F01D902220EE0292F01D9032275
:100EB8000AE0132F01D9042206E0092F01D90522DF
:100EC80002E0002FE7D006221A706149614A0591B5
:100ED800042388F8003002230B70136843F00103E1
:100EE80013605A460EE0032006F0FCFEF8E04FF0CF
:100EF800010B0BFA02F140F2B2330B4043B1012A65
:100F08005BD9002254490023092A0B70F9D8EEE76F
:100F180011F04D0FF3D00692C5F8743108F09AFA23
:100F2800069A0028EBD00620014614AA09F02CFEE8
:100F38009DF8551001EA0B029DF8531001EA0B01C8
:100F480001FA0BF343EA82019DF8512002EA0B03F0
:100F58000B430AD05BB25B4501D1002302E0022BB0
:100F68000DD1012385F8783110E00C2059460BAAE1
:100F780009F00AFE9DF82C3013F00F0303D1052069
:100F880006F0B0FE02E0042BEBD1E6E7294B334A2A
:100F98001A60334A5A6095F87821002A0CBF6F22EC
:100FA8006E221A722C4B04221A70059A032353706E
:100FB800284A136843F002031360264B1A6812F09C
:100FC800020F9B4602D01B4B1B689847254ABAF173
:100FD800000F4BD017F0FF0F0BD1DBF8003013F0E8
:100FE800020F4FF07D0140F2712308BF4FF4FA73EE
:100FF80002E04FF47A731946994505DBB9F57A6F23
:10100800A8BF4FF47A6900E099464B1E4B44B3FBE6
:10101800F1F3013BDBB203FB011185F87931116073
:1010280028E000BF00010050541A0020FC110020E5
:10103800A02100204422002070010020218D0008FA
:10104800598C0008358C000890C1793D00000020BB
:10105800FC00002040220020DB220020818D0008B7
:10106800978C000804050020D10A002085F879A192
:10107800C2F8009033689847BF4B00221A7094F862
:1010880058210AB188F8002094F859210AB1BB49BF
:101098000A7094F85A2102B11A70DBF80030B84986
:1010A80013F0080F1AD0BDF91000DFEDB66A6422FC
:1010B80090FBF2F302FB130212B207EE902AB8EE8D
:1010C800E77A07EE903AF8EEE77AE7EE267AB2EE9C
:1010D800047A67EE877AC1ED007A01E000230B609D
:1010E800A94B1A7842F002021A70A84A20211185E9
:1010F800102191610A279946DFF89082B8F81430D8
:101108009BB283F02003A8F81430B8F814309BB2CF
:1011180083F01003A8F81430192006F026FC0120EB
:1011280006F084FD192006F020FC013F002006F09F
:101138007DFD17F0FF07DFD11023C8F818302023F2
:10114800C8F81830924B9FED938A1B689FED920A5E
:101158001B7BDFF8708207EE903AF8EEE77AA7EE8D
:10116800880A04F0DAFCB8F8003007EE903AF8EE96
:10117800E77A27EE800A0EF033F8884B9FED887ADD
:101188001880B8F8003007EE903AF8EEE77A854B09
:10119800C7EE277AFF211B229FED837AC7EE877A55
:1011A8009FED827AC5ED5F7AD6ED047A804E67EEC0
:1011B800887A304667EE877AC3ED007A0DF001FE33
:1011C8007C4A7D4B12683770012112F0020F18BF5C
:1011D800717019701FBF032119700221B170510776
:1011E80048BF1978304641BF4E1C1E70032646542E
:1011F80012F00A0F0CD01A7804218154511CC9B27C
:1012080005264654D11C0232D2B2197006218154E7
:10121800039A11688A0641BF1A78561C1E70072661
:1012280048BF86546679082E01D00E2E04D11A784C
:10123800571C1F700B2787541A7811F0040F4FF0B2
:101248000C0E00F802E002F101071CBFDFF868E1AC
:101258000232FFB21F701FBF8EF80020544A4FF0B1
:10126800100E02F807E01A78571CFFB24FF0120E62
:1012780011F4806F1F7000F802E00ED094F814E2A9
:10128800BEF1000F09D0DFF830E102328EF80020FD
:10129800474A4FF0130E02F807E01A7811F4007F5E
:1012A8004FF0140E00F802E002F101071CBFDFF84E
:1012B80008E10232FFB21F701FBF8EF800203C4ABF
:1012C8004FF0150E02F807E0182E0DD11A781627E0
:1012D8008754571CFFB24FF0170E00F807E0D71CD1
:1012E8000232D2B21F708654CE0541BF1A78511C03
:1012F80019701A2348BF8354002198222F480DF0F3
:1013080060FD012006F05EFA002600285CD0012E60
:101318005AD82A4B4FF04C0A0AFB06F803EB080B85
:101328000BF148039F78049317B10136F6B2ECE746
:1013380090F9003090F804E01846214B03228DE81C
:10134800840001213A4653F82E3006F018FB059028
:1013580068B15246584639460DF033FD174A059B89
:1013680042F808300123049A1E449370F6B2012013
:1013780006F00EFAC9E700BFDA220020DB220020BF
:10138800181100208988883CBA22002000040048EF
:10139800B004002035FA8E3CDB0FC93FCC04002096
:1013A8000AE81C41AC04002000401C46BD378635C5
:1013B800D503002040220020D40300203803002059
:1013C800A408010802000020A14BA24A1A60A24BFF
:1013D800B4F852111980A14900230B808B70A049E1
:1013E8000A60B4F8982190B29E4921F8130001339D
:1013F800122BF9D1039B1B68D8045CBFB4F89E017B
:1014080008801F0740F1C18094F89231062B00F242
:10141800B680DFE803F004070E3C5674740045F20A
:10142800F05201E042F6F8228F4B1A8009F0F7FDDE
:10143800A4E007EE902ADFED8D6A8B4BB8EEE77AD1
:10144800DFED8B7AE7EE267A42F6F8211980002341
:10145800FCEEE77A874A17EE901A42F82310013318
:10146800122BF7D1844A85491160854A40201370B0
:1014780006F0A8F9002800F082800123072690F9D9
:101488000000804A8DE8480040217F4B71E0764B90
:1014980042F6F8221A80784B7C4A1A60784B102260
:1014A80040201A7006F08EF9002868D00123002524
:1014B80090F90000764A8DE8280040214FF4E13386
:1014C80057E0694B42F6F8221A806B4B714A1A6052
:1014D8006B4B082240201A7006F074F900284ED091
:1014E8000121002390F900006B4A8DE80A00402191
:1014F8004FF4E13306F043FAC5F880013BE05A4A5D
:10150800DFF8F8C1DFF8F8E1644F654E654D6648CD
:1015180042F6F82111805A490C22062B0A700DD088
:1015280000238CF800308EF800303B701B2333709A
:1015380005232A7003704FF4E1350AE000218CF886
:1015480000108EF8001039702A702121574D317023
:101558000370494B564A1A60402006F033F970B1BF
:101568000122002390F900008DE80C00514A402127
:101578002B4606F004FA003018BF012028B90820CD
:1015880004F0EEFB3C4B4C4A1A604C4D3C4A2B682D
:1015980013F4804F1FBF082111703749484818BFFE
:1015A800086042F20101194003F0010003F40056FB
:1015B80079B12D4B44F62061198026B108231370A8
:1015C8002D4B4049196020B10C2313702A4B3E491A
:1015D80019601378043B537006F0A0F93B4B186070
:1015E8006379052B02BF3A4B4FF4C8721A80394B06
:1015F8004FF47A721A80384A137843F0080313704C
:10160800364A137823F0020313702A6840F602035F
:1016180013406BB1324B334A1A60334B03221A70B2
:10162800324B01221A70324A00231380314A138048
:10163800A3682B60304B01221A7099F8003063F0D0
:101648007F0389F8003029B0BDEC028BBDE8F08F2C
:101658008C0B0020DE1B0020900B0020D8210020DE
:1016680020220020E00C002020050020CDCCCC3F1B
:101678000000B0C4980C002074000020594A0008EB
:1016880048210020C54C0008A0860100454A0008F2
:10169800194C00082D4A0008CD4B0008240D0020E5
:1016A800260D0020230C0020270D002090D00300D9
:1016B80049490008AD4A00083DBB00082422002023
:1016C8008D4A000831BB00089D4A0008FC04002030
:1016D800A20B0020D8220020920B0020E02200203C
:1016E800E00D0020D01B00203C220020000100203B
:1016F8001003002012030020D00A0020240C002030
:10170800250D002035FA8E3C1BB207EE903A5FEDAE
:10171800036AB4F95E31104AF8EEE77A07EE103A38
:1017280067EEA67AB4F96031CDED147A07EE903AF7
:10173800B8EEC77AF8EEE77A002127EE267A67EE48
:10174800A67A117014A805498DED157ACDED167A93
:1017580004F046FAFFF76FBB46000020BC0D0020DE
:101768002DE9F04FC14BB3F90610C14B2DED028B9B
:101778001E68728989B09142039311DBB1F5FA6F43
:1017880096F807B0BDBF8B1A03FB0BF3A2F5FA6BF3
:10179800CBF1640BBCBF93FBFBFB0BF1640B01E0CB
:1017A8004FF0640BB34DB44B2A68059293F962214C
:1017B800B3F898A1059C029392B2079200225300B5
:1017C8000693AA4B33F912300493CAEB030303F2CE
:1017D800F31740F2E630874203D8002BB8BF5B42CC
:1017E80001E04FF4FA73022A01934FF06400059B5D
:1017F800A24F34D093F811E1BEF1000F06D0019B3F
:101808007345CCBFCEEB030300230193019BDFF8A4
:10181800B8E293FBF0FC6FF063093EF81C8009FB0B
:101828000C390CF1010C069B3EF91CE00FFA88FC00
:10183800CCEB0E0E0EFB09FE9EFBF0FEC64427F80D
:1018480003E0B718019B3F797B438D4F93FBF7F378
:1018580064339BB20BFB03F393FBF0F031E093F896
:1018680012E1BEF1000F06D0019B7345CCBFCEEB51
:10187800030300230193019BDFF8388293FBF0F008
:101888006FF0630C38F910E00CFB00390130BDF83B
:101898001C3038F91000CEEB000000FB09F999FB69
:1018A800FCF9CEEB090919FB03F9019BA7F8049091
:1018B800B079002BB8BF5B424343714893FBF0F00B
:1018C800643063786F4F4FF0640E434393FBFEF32D
:1018D800BB546D4FE37A434393FBFEF3BB54637DE4
:1018E800664F5843694B90FBFEF0022A9854684BA8
:1018F8000FD183F802E0049B53450FDB5E4CB4F82C
:101908009A21914216DBB1F5FA6FA8BF4FF4FA613C
:1019180011E003F802B0049B534504DA069B0698CD
:10192800FB5A5B423B520132032A04F101047FF463
:1019380046AFE3E71146891A4FF47A735943554B7A
:101948004E4E6FF0630CC2F5FA624FF0640EB1FBB5
:10195800F2F191FBFEF233F812000CFB0211013296
:1019680033F9122003B2D21A514391FBFEF3034418
:10197800FB80494B1B88580637D5484B484A1B887B
:101988001288DFED487A9FED480A9B1A1BB208EED1
:10199800103AB8EEC88A28EE278A38EE000A04F012
:1019A800BCF8F0EE408AB0EE480A04F0B6F8B6F992
:1019B800023006EE903AB6F90030F8EEE66A07EE25
:1019C800903A20EE667AF8EEE77AA7EEA87A67EE04
:1019D800807ABDEEC77AE6EEA87A17EE103AFDEEE9
:1019E800E77A338017EE903A7380304E3368990760
:1019F80040F1AA802E4B2F491A684B6945F20720FF
:101A0800D31A8342884640F39F804A6103F0ACFDB5
:101A1800294BDFF8B8A01A78032A9946BAF800309B
:101A280056D10A2B60D90023282089F8003005F008
:101A38009CFF03F099FD214B188803F07FFD204B94
:101A48001A68D37890FBF3F0013008281D4BA8BF23
:101A580008201870537980B213FB00F3A8F81830E7
:101A6800137913FB00F0A8F81A003DE0E00C002001
:101A780004220020FC110020541A0020BA0E002075
:101A88000CFEFFFF400F002006030020580F002027
:101A9800C80E002052110020B80E00209C0B002018
:101AA800B822002035FA8E3CDB0FC93F24220020E3
:101AB800C0220020F80200203C220020FC0D00205B
:101AC800E00D0020000100206A110020880E00208F
:101AD8000A2B09D80323A64A89F80030002313707B
:101AE800A8F81830A8F81A3099F80030A14A012B44
:101AF8000DD002D3022B1DD026E0B8F81820BAF872
:101B080000309A4220DD012389F8003010E0BAF84D
:101B18000010B8F81A308B4202DD0223137010E06F
:101B2800954B1B8B0133994202DD002313700BE0A8
:101B3800082007E0B8F81A30BAF8002001339A42B2
:101B4800E1DC072006F090F8D6F800B08B4E1BF4C5
:101B5800006F7ED08A4B88491A68CB69C3EB0209AB
:101B680045F207239945884673DD864BB7F9067019
:101B7800D3F800A0CA619AF80A30B4F85211012BC0
:101B88004FF47A72A7F57A7799FBF2F903D045D327
:101B9800022B23D045E07C4BD8F82000597B7B4BA7
:101BA80033F81110082789B290FBF7F3C01A4318CD
:101BB800A8F82410C8F8203040F6E44193FBF7F366
:101BC8009BB24B43BAF80810C1EB13335A43BAF926
:101BD800063092FBF3F2C8F8282022E03278BAF8EF
:101BE8000830C8F8283052071BD56948019305F01A
:101BF8007BFE019B18B91BF0100F18BF002707FBCD
:101C080007F2322192FBF1F21744BAF90620574342
:101C18004FF47A7297FBF2F73B4400E00023C8F8D0
:101C28002830D8E90C01D8F828305A4A03FB09F3C0
:101C38004FF47A7993FBF9F310EB030A41EBE37B5A
:101C4800C8E90CAB5046594600230AF0BDFDC8F858
:101C58003800514B1A6812F4805F984602D00A2067
:101C680006F002F84D4F3B68002B52D0DFF854E1E4
:101C78004B4ADEF8000011688142F246914648D886
:101C8800484ADFF828B110785968D8B90123137089
:101C9800BBF800208A5C22B31846019305F0C6FF02
:101CA800414A019B13700AF07BF8BBF80030C3B9B6
:101CB8003B681B78053B012B13D805F02FFE2E4BF4
:101CC800D8630EE000231370BBF800208A5C42B191
:101CD8001846019305F0AAFF334A019B13700AF0D6
:101CE8005FF83A68BBF8003052683048D25CFE2A88
:101CF80001D100230CE0FF2A02D105F09DFF08E086
:101D0800DAF800700A2111FB0272C9F800200133C9
:101D1800038033785F0703D5254B10221A8561E0CD
:101D2800D8F80020D0075EBF144943F001030B70B8
:101D3800204B1B7819075EBF337823F001033370FB
:101D4800D30242BF337823F0010333701A4B1A8849
:101D5800154B1AB1194A1268970702D4184A128803
:101D680092B302221A70337823F00103337030E003
:101D7800000100203C220020F8020020E022002080
:101D8800C0220020E00D0020E40D0020F40D00200A
:101D9800DE1B0020407E05006C0B0020C4110020D3
:101DA800BC110020B811002028220020C0110020FA
:101DB80000040048920B0020A20B002040220020C3
:101DC800D82200204C1A00203178C80758BF0222B8
:101DD8001A7005F0A3FDB44B1B68C01A002801DB7C
:101DE80009F0DEFFB14F3E78002E00F0D080B04BF6
:101DF8001A689846002A01F01C80D8F80000036889
:101E08005B689847002801F01480A94BA94C186812
:101E180003689B689847092801D03F2852D14FF0A2
:101E2800000A2668DFF8CC92554636B1A248D9F8A0
:101E3800001032460DF012F810B9CA4605B94D46E1
:101E48009E4B09F110099945EFD3EDB1D5F800C0C3
:101E5800DAF8009023681CF803E019F803007045CD
:101E680012D15A1C944958B92D2B09D8DFF844E2ED
:101E7800CEF800204FF0200E01F803E0885403E06C
:101E880001F803E02260E5E723680BB1554510D05F
:101E98008B480AF07BF8554507D855F8100B0AF01F
:101EA80075F809200AF06AF8F5E786480AF06EF82E
:101EB800002623689E42A0D27F4B985D0AF05EF808
:101EC8000136F6E72368002B40F09487042841F098
:101ED8006C84794806F088F800F0ABBFD8F80000A9
:101EE800DFF8F0B103685B689847002845D0DBF855
:101EF800000003689B689847D9F8003093F8482099
:101F08008246002A51D1242840F08880012283F893
:101F18004820D9F8002092F848000628DED192F827
:101F280049304B2B00F0DB8600F28781322B00F022
:101F3800088700F22181222B00F06C8500F2DC80FA
:101F4800032B00F01D8200F2A480012B40F090804A
:101F5800032009F093FF002009F063FF012009F036
:101F680060FF0D2009F05DFF574F3B68987909F035
:101F780058FF3B68002283F84820544B93F81331EC
:101F8800002B40F025874C36982E00F05287504A97
:101F9800931993F84A100129F5D14B4FB2583B6079
:101FA8004C4BB9461A60984698E7012A04D14D2847
:101FB80014BF00220222AAE7022A04D13C2814BF37
:101FC80000220322A3E7032A0AD140284FF0000287
:101FD8009FBF1A71DA715871987198BF042296E7F9
:101FE800042A08D19A7983F8490080EA020A83F81A
:101FF80006A005228BE7052A8BD159791A799142D7
:10200800997906D941409971511C19711344187274
:102018007FE781420CBF0622002278E72E4B1A7810
:1020280052073FF576AF2328DBF8002013D11F496C
:102038000193012008701E4928480A602349C1F805
:10204800D82009F0A3FF1F4809F0A0FF019B1A78C8
:1020580042F002021A70224B1B681B78534501BFDD
:10206800204B214A1A60214B04BF214ADA6050E70D
:10207800022B40F00187042009F000FF432009F0FB
:10208800D0FE4C2009F0CDFE462009F0CAFE4C20B7
:1020980068E7042B00F07F81052B40F0ED861A20BD
:1020A80009F0ECFE002787E12C220020DC2200202A
:1020B80038220020F8110020C81100205C0A01080D
:1020C800382001083D20010830220020F8020020B5
:1020D8003803002034220020E02200206D2001086F
:1020E8001C110020FC9F0020EFBEADDE00ED00E0DB
:1020F8000400FA05DC080108282B00F0D68515D85D
:10210800242B00F0B885262B40F0B686B64F062063
:1021180009F0B4FEB7F85C0109F0B3FEB7F85E0148
:1021280009F0AFFEB7F8600100F022BE2A2B00F0DC
:10213800CF852C2B40F0A086AB4F0C2009F09EFEDB
:1021480097F8920109F06DFEB7F89C0109F099FE25
:10215800B7F8980109F095FEB7F89A0109F091FED1
:1021680097F8930109F05DFEB7F89E0109F089FE22
:10217800B7F8A00100F0FCBD3D2B00F01D8323D86B
:10218800382B00F07E8512D8342B00F06684362B6D
:1021980040F07286954B944F93F80E01C0EBC00047
:1021A800C0B209F06BFE07F1200800F0F0BD3A2B31
:1021B80000F0A8823B2B40F05F86012009F05EFE0C
:1021C8008B4B1B681878CDE6452B00F0EE8527D899
:1021D800402B00F0BE85422B40F04E86824F1020E7
:1021E80009F04CFE787909F01CFEB86809F052FE37
:1021F80097F8920109F015FEB7F85C0109F041FE65
:10220800B7F85E0109F03DFEB7F8600109F039FE44
:10221800B7F8820109F035FEB7F8840100F0A8BDCF
:10222800462B00F0B885492B40F02686022009F09D
:1022380025FE6D4B988900F09BBD702B00F0E8825D
:1022480056D8682B00F0368224D8652B00F0E4803D
:1022580015D84D2B00F05285642B40F00D860720D1
:1022680009F00CFEE72009F0DCFD5F4B587909F016
:10227800D8FD002009F0D5FD042000F0A5BD662B8F
:1022880000F08B81672B40F0F785102009F0F6FDF0
:102298000027A3E16D2B00F02F8213D8692B00F0E3
:1022A80015826C2B40F0E885524F062009F0E6FDB8
:1022B800388809F0E6FD788809F0E3FD4E4B188868
:1022C80000F056BD6E2B00F021826F2B40F0D485B4
:1022D8004A4F0B2009F0D2FD3B68187809F0A1FDA0
:1022E8003B68587809F09DFD4FF00009B8466FE249
:1022F800782B00F07B811ED8742B00F0D7830BD885
:10230800722B00F04984732B40F0B685082009F041
:10231800B5FD012700F090BC752B00F06F83772B7B
:1023280040F0AA85DFF8C48098F8DC0009F0A6FD23
:10233800002700F027BCF02B00F0908414D87B2BEA
:1023480000F0F882A02B40F097850C2009F096FD4C
:102358002B4B186809F09EFD2A4B186809F09AFD66
:10236800294B186800F030BDF12B00F07D81FE2B61
:1023780040F08285082009F081FD002000F064BC4F
:10238800184609F07BFD012009F04BFD0A2009F0F1
:1023980048FD0020E6E5062009F070FD412009F01F
:1023A80040FD572009F03DFD462009F03AFD332055
:1023B80009F037FD00F050BC144BD85D013709F027
:1023C80030FD0B2FF8D10027114BD85D013709F0EC
:1023D80028FD082FF8D100270E4BD85D013709F0EA
:1023E80020FD072FF8D1BFE5541A0020F80200207D
:1023F800FC110020221A00209C0B0020042200203F
:10240800ACF7FF1FB0F7FF1FB4F7FF1FA5200108A7
:10241800B1200108BA2001080B2009F02FFDCF4B8D
:10242800188809F02EFDCE4B1A68CE4B9A420CBF85
:10243800CD4BCE4B188880B209F023FDCC4B1B68DE
:10244800C3F3C000C3F38002800040EA4200C3F334
:1024580040021043C3F3401240EAC20003F01003E5
:10246800184309F00EFDC34B1A88C34B12F0010F35
:1024780014BF4FF002084FF0000812F0020F14BF0B
:102488004FF0040C4FF0000C12F0040F14BF4FF083
:10249800100E4FF0000E12F0400F14BF2027002737
:1024A80012F0100F14BF4FF40070002012F0200F2C
:1024B8001B6814BF4FF4806B4FF0000B12F4807F41
:1024C80014BF4FF400610021019102F0080903F4E0
:1024D800475141EA090903F4804149EA010903F433
:1024E800004149EA010903F4803149EA010903F48A
:1024F800003149EA010903F4802A49EA0A0903F488
:10250800002149EA010103F4801941EA090903F0AD
:10251800007349EA0303DFF8909299F80090C9F331
:10252800800943EA090343EA080343EA0C0C4CEA2E
:102538000E0E4EEA07073843019B12F4007F40EA6B
:102548000B0B4BEA030B14BF4FF4001100218B4B0C
:1025580012F4806F4BEA01014FF0000014BF4FF0F6
:10256800806B4FF0000B93F8DC7041EA0B010346D7
:10257800BB420CD2824A13F802E0012202FA0EFE94
:102588001EEA010F1CBF9A4010430133F0E709F01F
:1025980081FC7C4B93F8C806E4E4122009F06EFC39
:1025A800794B1B88B3F5806F8CBF4FF008084FF04C
:1025B80001080027754B33F9170090FBF8F0013735
:1025C80080B209F05EFC032FF4D1714F388809F00E
:1025D80058FC788809F055FCB88835E36D4BD85D10
:1025E800013709F01EFC102FF8D1BDE4702009F066
:1025F80045FC4FF000082B680E2707FB08F73B4403
:1026080008F10108B3F8190109F03BFC2B683B44B9
:10261800B3F81B0109F035FC2B683B44B3F81D01E6
:1026280009F02FFC2B683B4493F81F0109F0F9FBD4
:102638002B683B4493F8200109F0F3FB2B683B44DB
:1026480093F8210109F0EDFB2B683B4493F8220134
:1026580009F0E7FB2B681F44D7F8230109F01AFC9F
:10266800B8F1080FC7D17FE47020464F09F006FC87
:1026780007F1700897F8D40009F0D3FB97F8D50054
:1026880009F0CFFB97F8D60009F0CBFB97F8D700F5
:1026980009F0C7FB97F8D80009F0C3FB97F8D900F1
:1026A80009F0BFFB073797F8D30009F0BAFB474595
:1026B800E0D159E4102009F0E1FB0027364BD85D42
:1026C800013709F0AEFB102FF8D14DE4DFF8DC80BC
:1026D80098F80000400000F0FE0009F0CFFB00274A
:1026E80098F800309F42BFF43FAC2C4B33F81700EA
:1026F80009F0C7FB0137F3E709F0C0FB002009F038
:10270800C9FBA9E2042009F0B9FB5CE3072009F042
:10271800B5FB234B194F1888FF28A8BFFF20C0B26C
:1027280009F07FFBB86B4FF6FF784045A8BF4046DD
:1027380020EAE07080B209F0A4FB1A4B188809F06F
:10274800A0FB104BB86A93F887318BB30A23584320
:102758004045A8BF404620EAE0702BE05422002004
:10276800181A002000540040502200205222002055
:1027780040220020B80E00206C0B0020F802002038
:10278800D5030020541A002002000020F003002086
:10279800C20E0020F6030020800F0020E00C00206D
:1027A800880E0020700B0020E02200204821002025
:1027B80000F30F0080B2DBE2D24F022009F05EFB8B
:1027C80097F8E20109F02DFB97F8E101FFF7CABB82
:1027D800D8F80030CC4F4B4409F10109187909F0B9
:1027E80020FBB9F1030FF3D13B68D87909F019FB45
:1027F8003B68987809F015FB3B68D87809F011FB1D
:102808003B68588909F03DFB3B68187AFFF7AABB7B
:10281800BE4F1E2009F032FB3B681B78022B4FF09D
:10282800000871D13B6803EB880393ED080AB2EE08
:10283800048A20EE080A0CF0D3FC80F30800C0B22A
:1028480009F0EFFA3B68DFEDB27A03EB880393ED0A
:102858000B0A20EE270A0CF0C3FC80F30800C0B274
:1028680009F0DFFA3B68DFEDAB7A03EB880393ED01
:102878000E0A20EE270A0CF0B3FC80F30800C0B261
:1028880008F1010809F0CDFAB8F1030FCAD1B8F17F
:10289800070F3B6823D193ED110A20EE080A0CF0CC
:1028A8009FFC80F30800C0B209F0BBFA3B6893EDC7
:1028B800120A20EE080A0CF093FC80F30800C0B25C
:1028C80009F0AFFA3B6893F84C3000EE103AB8EED6
:1028D800400A0CF085FC80F30800C0B20BE04344CA
:1028E800587809F09EFA3B684344D87A09F099FA77
:1028F8003B684344587D08F1010809F092FAB8F1A1
:102908000A0FC4D1FFF730BB3B684344587809F03D
:1029180088FA3B684344D87A09F083FA3B68434411
:1029280008F10108587D09F07CFAB8F10A0FEBD1DB
:10293800FFF71ABB3C2009F0A1FA0027DFF8CC8189
:102948009FED748AD8F8003003EB870393ED080AEB
:1029580020EE080A0CF044FC80B209F092FAD8F88C
:10296800003003EB870393ED0B0A20EE080A0CF006
:1029780037FC80B209F085FAD8F8003003EB8703FA
:1029880093ED0E0A20EE080A0CF02AFC013780B2FB
:1029980009F077FA032FD1D1072FD8F8003018D1D2
:1029A80093ED110A20EE080A0CF01AFC80B209F027
:1029B80068FAD8F8003093ED120A20EE080A0CF0F5
:1029C8000FFC80B209F05DFAD8F8003093F84C009B
:1029D8000DE03B44587809F054FAD8F800303B44ED
:1029E800D87A09F04EFAD8F800303B44587D0137C0
:1029F80009F047FA0A2FCFD1FFF7B6BA2F2009F00E
:102A08003DFA454F17F8010F00283FF4ADAA09F029
:102A180008FAF7E7502009F031FA00273B4B1B680A
:102A280003EB87083D4B98F879200C2101FB023312
:102A3800013793F8380009F0F4F998F87A0009F0AA
:102A4800F0F998F87B0009F0ECF998F87C0009F0A7
:102A5800E8F9142FE2D1FFF787BA482009F00EFAF7
:102A68004FF00008294B1F68062303FB087708F17D
:102A7800010897F8CE0009F0D4F997F8C90009F0D1
:102A8800D0F997F8CA0009F0CCF997F8CB0009F00B
:102A9800C8F997F8CC0009F0C4F997F8CD0009F007
:102AA800C0F9B8F10C0FDDD1FFF75EBA4FF000089E
:102AB8004FF001094FF0000A194B93F8DC209245BA
:102AC80042DADD334FF0000B1AF80320134F0C23C2
:102AD80007F1300103FB0BF3595C914209D13B44E8
:102AE800586B0CF0B2F90246B9F1000F07D14B460A
:102AF80018E00BF1010BBBF11C0FE7D121E080447A
:102B08001FE000BF541A002004220020FC110020FE
:102B18000000C84200007A44D7060108D806010818
:102B2800F802002093420CDA0C2101FB0B7104928D
:102B3800496B0193C85C09F074F9019B049A01334D
:102B4800F0E70AF1010AB7E7B9F1000F3FF40CAA60
:102B58005FFA88F009F092F94FF00009AAE701310D
:102B68001C290ED0CC480C2200F1300C02FB01F3DA
:102B780013F80C207245F2D1034493F8380009F099
:102B880050F9013798F8DC309F42BFF4EDA9C34BE8
:102B9800002117F803E0E5E7162009F06FF9029B1A
:102BA800B3F8980109F06DF9029BB3F8440109F0F4
:102BB80068F9029BB3F8460109F063F9029BB3F880
:102BC800480109F05EF9029BB3F8DA0109F059F9F6
:102BD800002009F026F9002009F023F9002009F067
:102BE80020F9029B93F8870109F01BF9029B93F8DF
:102BF800940109F016F9002009F013F9A84B1B6895
:102C08000A20B3F9563093FBF0F080B209F039F995
:102C1800029B93F87C0109F004F9029B93F8800168
:102C280009F0FFF8029B93F87F0109F0FAF8029B7C
:102C380093F88101FFF796B9F8B2013709F0F1F876
:102C4800092FF9D1FFF790B909F01BF9002009F015
:102C580018F9002009F015F9002089E0904F0420A8
:102C680009F00CF93B68B3F85A0009F00AF93B6817
:102C7800B3F858007CE0042009F000F9894B986803
:102C8800A2E0884F042009F0F9F897F87C0109F0D0
:102C9800C8F897F8800109F0C4F897F87F0109F09F
:102CA800C0F897F88101FFF75DB97E4F072009F05A
:102CB800E5F8B7F8820109F0E4F8B7F8840109F0FB
:102CC800E0F897F8860109F0ACF8B7F888014FE00A
:102CD800012009F0D3F8734B5879FFF743B9714FC6
:102CE800042009F0CBF897F8D80109F09AF897F87A
:102CF800D90109F096F8B7F8DA0139E06A4FDFF838
:102D0800D081387800EB4000C0B209F0B7F84FF036
:102D180000093B78994508F10208BFF425A918F87D
:102D2800020C09F07EF818F8010C00EB800000EBAB
:102D3800800000F2EE2080B209F0A3F809F1010941
:102D4800E7E7012009F09AF8564B93F89401FFF74A
:102D580009B9082009F092F80027524B3B44013783
:102D680093F88A0109F05DF8082FF6D1FFF7FCB84F
:102D780009F087F8FFF7F8B84C4AD25C904264D063
:102D88000C33302BF8D1083747453FF4EDA897F8B6
:102D9800F2010023F0E70D2009F070F8002009F097
:102DA80040F8002009F076F80AE0132009F066F8E8
:102DB80000273F4BD85D013709F033F80B2FF8D1C6
:102DC800002009F067F8002009F064F8FFF7CCB894
:102DD800384BF05804F0BEFF18B9322004F0C5FD96
:102DE800F6E704F011F902F0CBFF334B334ADA600F
:102DF800FFF7C9B80C2800F0DA840A2840F0DB8411
:102E08002F4D304809F0C2F8284623210CF00FF85E
:102E180008B1401B20602368002B40F0D08428486C
:102E28002360002130220BF0CCFF3B78002B40F0D0
:102E3800FB84254B9B68002B00F01D85234809B0B7
:102E4800BDEC028BBDE8F04F184708F0EAFFB7F871
:102E5800F40109F016F897F8F60108F0E2FF97F880
:102E6800F70108F0DEFF97F8F90108F0DAFF97F8A4
:102E7800F80108F0D6FF86E74C2B3BD108F0B4FFE9
:102E8800084F87F8D80108F0AFFF87F8D90108F094
:102E9800B5FFA7F8DA0128E0D8060108D503002015
:102EA800FC110020541A0020482100202011002085
:102EB800A52001083803002000ED00E00400FA0511
:102EC800C8110020112C0108A02100200C040020AA
:102ED800F61B0020D42B00F05183D22B40F06184E4
:102EE800CA4B1B785B0740F19083002008F0C6FFAF
:102EF800FFF73AB800F27B81352B27D108F074FF31
:102F08000B28804602D908F0CBF8EEE7C04B1F68C3
:102F180008F06AFF0328F6D8062303FB087787F82A
:102F2800CE0008F061FF87F8C90008F05DFF87F858
:102F3800CA0008F059FF87F8CB0008F055FF87F85A
:102F4800CC0008F051FF87F8CD00CEE700F2A5804D
:102F5800292B11D108F052FFAE4FA7F8820108F0D3
:102F68004DFFA7F8840108F03FFF87F8860108F0B5
:102F780045FFA7F88801B8E759D8252B07D1A54BF5
:102F880000229A6008F044FF02F0F2FEADE7272B1A
:102F98000DD108F033FF9F4FA7F85C0108F02EFF12
:102FA800A7F85E0108F02AFFA7F860019DE7232B28
:102FB80040F0F78308F018FF13288146A3D8DFF8FC
:102FC8005082D8F8007008F00FFF002292490C23B5
:102FD800534301EB030E9EF838E0864523D10B449A
:102FE8000FFA89F907EB890793F8303087F87930B9
:102FF80008F0FAFE87F87A0008F0F6FE87F87B00FA
:1030080008F0F2FE854B864A1A6087F87C00854BEB
:10301800D8F800001860793007F0B2FF824B80F0D2
:103028000100187061E701321C2ACFD16BE72D2B04
:1030380023D108F0D9FEDFF8DC8188F8920108F086
:10304800DDFEA8F89C0108F0D9FEA8F8980108F060
:10305800D5FEA8F89A0108F0C7FE3B6888F89301E6
:103068005B79082B7FF641AF08F0C8FEA8F89E01EF
:1030780008F0C4FEA8F8A00137E7332B05D108F003
:10308800B3FE644B83F894012FE72B2B40F0898320
:1030980008F0AAFE5F4B587127E73E2B09D108F0CC
:1030A800A3FE5C4F87F8E20108F09EFE87F8E10175
:1030B8001BE759D8392B11D108F096FE554F87F8E0
:1030C8007C0108F091FE87F8800108F08DFE87F8F2
:1030D8007F0108F089FE87F8810106E73C2B0BD1B8
:1030E8004B4FD7F8008008F07FFE88F800003B6857
:1030F800187804F069F8F8E6372B40F052835379D2
:103108000727B3FBF7F2C2EBC2029A1A12F0FF0FBD
:103118007FF4F9AEB3FBF7F7013FFFB2FF2F3FF49F
:10312800E4AE08F061FE5FFA80F94FFA89F004F026
:1031380075FA804600283FF4E6AE80F8009008F063
:103148005DFEA8F8020008F04FFE88F8040008F0B9
:103158004BFE88F8050008F047FE88F8070008F0DD
:1031680043FE88F80600D7E7432B22D108F03CFE3F
:10317800284F0023BB60787108F04AFE02F0F8FD82
:1031880008F032FE87F8920108F038FEA7F85C01D3
:1031980008F034FEA7F85E0108F030FEA7F86001D9
:1031A80008F02CFEA7F8820108F028FEA7F8840191
:1031B8009BE60DD8412B40F0F482002708F014FE5E
:1031C800144B3B440137082F83F88A01F6D18CE66B
:1031D800442B04D1154B012283F8132185E64A2B91
:1031E80040F0DF8208F00AFE0A4B98817DE6D02B7A
:1031F8001ED1064B1B7858073FF577AE05F036FE13
:1032080002F0E8FD02F0A8FE6FE600BFE022002011
:10321800FC110020541A0020D8060108DC0B0020FD
:10322800981B0020E00B002014000020F80200206A
:1032380000F28E81CC2B50D15379092B7FF663AEE7
:10324800039BD3F8008008F0CFFD039B88F80000AB
:10325800D3F8008008F0C8FD88F8010008F0C4FD24
:10326800039B64281B68A8BF6420187108F0BCFD84
:10327800039B64281B68A8BF6420587108F0B4FD3C
:10328800039BFF281B68A8BFFF20987108F0ACFDBE
:10329800039B6428D3F8008028BF642088F80700BF
:1032A80008F0A2FD039B88F80200D3F8008008F01C
:1032B8009BFD039B88F80300D3F8008008F09EFD6F
:1032C8003B68A8F80A005B790A2B7FF60EAEDC4B48
:1032D8001F6808F089FD387207E600F2DC80C82B09
:1032E80015D157797F08122F3FF60DAE4FF0000821
:1032F800B84507D208F082FDD24B23F8180008F130
:103308000108F5E7D04B012283F81221EDE5CA2B1D
:1033180040F09280CD4F3B681B78022B4FF000089D
:103328006FD1D7F8009008F05FFD07EE900AF8EE2D
:10333800677AB2EE048AC7EE887A09EB8809C9ED84
:10334800087AD7F8009008F04FFD07EE900A9FED35
:10335800C07AF8EE677A09EB8809C7EE877AC9ED73
:103368000B7AD7F8009008F03FFD07EE900A9FED22
:10337800B97AF8EE677A09EB8809C7EE877A08F117
:103388000108B8F1030FC9ED0E7ACAD1B8F1070FD9
:10339800D7F800901CD108F027FD07EE900AF8EE48
:1033A800677AC7EE887AC9ED117AD7F8009008F0E5
:1033B8001BFD07EE900AF8EE677AC7EE887AC9ED2A
:1033C800127AD7F8009008F00FFD89F84C0012E047
:1033D80008F00AFDC14489F80100D7F8009008F008
:1033E80003FDC14489F80B00D7F8009008F0FCFCF5
:1033F800C14489F8150008F10108B8F10A0FC5D1D0
:1034080073E5D7F8009008F0EFFCC14489F8010093
:10341800D7F8009008F0E8FCC14489F80B00D7F809
:10342800009008F0E1FCC14408F10108B8F10A0F66
:1034380089F81500E5D158E54E2B40F0B28157794F
:103448000323B7FBF3F7122F3FF65DADDFF81082C9
:103458004FF00009B945BFF448AD08F0C5FC88F83D
:10346800A20108F0CBFC40F2ED23984205DD40F6BE
:10347800CA039842A8BF184601E040F2EE20A0F225
:10348800EE20192309F1010990FBF3F008F1020875
:1034980088F8A101DEE7CE2B0AD16F4B1B785A07BB
:1034A8003FF523AD6D4A137843F0040313701CE510
:1034B80044D908F0A3FC6FF4AF67C3199BB2C62BBD
:1034C8009CBF674BA3F8980108F098FCA4F8440146
:1034D80008F094FCA4F8460108F090FCA4F8480110
:1034E80008F08CFCA4F8DA0108F07EFC08F07CFCFB
:1034F80008F07AFC08F078FC84F8870108F074FC7E
:1035080084F8940108F070FC504B1F6808F076FCB2
:1035180000EB80004000A7F8560008F065FC84F82E
:103528007C0108F061FC84F8800108F05DFC84F8F7
:103538007F0108F059FC84F88101D6E4464B1B78DA
:1035480059073FF5D2AC474B4FF4C8721A80CCE408
:10355800D62B09D1002708F051FC434B23F817005C
:103568000137082FF7D1C0E45BD8D32B7FF4B2AC76
:1035780008F044FC344BA3F81001B6E453790F2B40
:103588007FF4C1AC08F030FC072807463FF6BBAC17
:10359800DFF8B880D8F8009008F030FC0E235F43BD
:1035A800B944A9F81901D8F8009008F027FCB944E3
:1035B800A9F81B01D8F8009008F020FCB944A9F834
:1035C8001D01D8F8009008F00FFCB94489F81F01D4
:1035D800D8F8009008F008FCB94489F82001D8F818
:1035E800009008F001FCB94489F82101D8F800904E
:1035F80008F0FAFBB944D8F8008089F8220108F0ED
:1036080007FC4744C7F823016FE408F0EDFB144BAF
:10361800022883F8C8067FF6F3AD002283F8C8268F
:10362800EEE5EF2B22D1094FD7F8008008F0E6FB32
:10363800A8F85A003F6808F0E1FBA7F8580054E4DE
:1036480004220020E00C0020F8020020FC110020D9
:103658000000C84200007A44E0220020920B0020BB
:10366800541A0020A20B0020082200206DD8D82B65
:1036780040F097800027DFF834829FED818AD8F8E0
:10368800009008F0BBFB07EE900AF8EE677A09EBAA
:103698008709C7EE887AC9ED087AD8F8009008F04B
:1036A800ADFB07EE900AF8EE677A09EB8709C7EEDB
:1036B800887AC9ED0B7AD8F8009008F09FFB07EEDE
:1036C800900AF8EE677A09EB8709C7EE887A01371E
:1036D800032FC9ED0E7ACED1072FD8F800901CD150
:1036E80008F08CFB07EE900AF8EE677AC7EE887A46
:1036F800C9ED117AD8F8009008F080FB07EE900A1F
:10370800F8EE677AC7EE887AC9ED127AD8F8009091
:1037180008F074FB89F84C0012E008F06FFBB9441C
:1037280089F80100D8F8009008F068FBB94489F8D6
:103738000B00D8F8009008F061FBB94489F815002F
:1037480001370A2FC8D1FFF7D0BBF22B22D108F0DE
:103758004BFB0F2807463FF6D6AB08F045FB494B15
:10376800C7EBC7071F44387108F03EFB787108F0B3
:103778003BFBB87108F038FBF87108F035FB38727C
:1037880008F032FB787208F02FFBB87203F07CFC6B
:10379800FFF7ABBBFA2B04D13B4B1B785B077FF5DC
:1037A8002FAD07F07DFCFEF7DFBB0C284AD1374868
:1037B80008F0ECFB38E00D2838D1FFF721BB5A1E82
:1037C800A95C202902D11346FFF726BB304A2360A3
:1037D8000021D1542F4B304DD3F800A0D5F800B0BC
:1037E800DFF8AC9058460BF030FB064632464846A8
:1037F80059460BF033FB294A28B919F806305344C7
:103808005B78590703D010359542E7D306E0954217
:1038180004D2701CEB684844984702E0204808F03E
:10382800B5FB0023FFF7FBBA1E4807E07F280DD140
:10383800013B174A1C4823600021D15408F0A6FB1D
:10384800FEF7DBBA7F2804D1FEF7D7BA2F2B3EF656
:10385800D4AAA0F12002D2B25E2A3EF6CEAA13B9AB
:1038680020283EF4CAAA5A1C2260094AD05408F0FB
:1038780085FBFEF7C2BA09B0BDEC028BBDE8F08F3C
:1038880000007A44241B0020E02200204220010886
:10389800C811002004010020DC0801085C0A0108A6
:1038A8004D2001083D20010869200108FC11002075
:1038B800984A13682DE9F04F03F59C43964C203342
:1038C8002360964B196889B011F4804F05929B4686
:1038D80005D108F059FA10B92379013323716779B2
:1038E800A7B18D4B013F5F71DCE0D8F800308C4800
:1038F800072D98BF595D8B4B88BF29461B68984791
:10390800032D0BD904EB45050137E880844BDFF81C
:103918002C821E78FDB2AE42E7D820E0D8F800200D
:1039280005F10E0302EB83039988DA880028E9D0B1
:103938004FF47A73401A5843531A90FBF3F040F649
:10394800C90300F57A70984205DC40F2EE239842EC
:10395800B8BF184601E040F6CA0080B2D2E70F238C
:10396800277984F82A3094F82B300193032594F8AA
:103978002C30B7FBF5F505EB45057D1B0393D8F80F
:1039880000300293DFF8C091EBB204930025B542F2
:1039980054DA6549019B31F815A04FEA450853B937
:1039A80008F0F2F928B1039B002B08BF4FF0000A7A
:1039B80001E0DDF804A0029B988A504502D8D88A15
:1039C80050450ED2E8B208F0B9F9032D8246DFBFA0
:1039D80094F82AE00120A8402EEA0000D8BF84F815
:1039E8002A0008F0D1F918B1504828F800A021E0C1
:1039F800049B94F8760029F813A028B9022F15D94A
:103A08004549012081F87600B9F80210B9F800009C
:103A18000844B9F804100844454980B228F8010060
:103A280000B2032190FBF1F080B200E050463F491C
:103A380028F80100013509F10609A8E794F82A20B9
:103A48003C483D4BA2F10F014A424A4184F890207C
:103A580072B1314AD2F89420520109D40268D96867
:103A68009A60521AC82A1DD9012283F8212019E028
:103A780002689868DA605B68121A9A4288BF2E4B0F
:103A88004FF0000184F82B1088BF83F8211000251F
:103A9800B54207DAE8B208F051F9244B23F81500CB
:103AA8000135F5E7DBF80030DF0405D5D4F89430AC
:103AB800DE0701D408F060FE059B19681F4B1F68DC
:103AC800BB7A002B42D0013B18483A7B30F81330C0
:103AD8001AB1C3F53B6308339BB21BB2A3F57A73E3
:103AE800B3F57A7FA8BF4FF47A7323EAE37307EE3E
:103AF800903A9FED137AF8EEE77AC7EE877A9FED52
:103B0800117A67EE877AFCEEE77A17EE903AA4F816
:103B1800983062E0C0220020D80A00202422002029
:103B28004821002074000020DE0A0020E00C00205C
:103B3800500B00204C1A0020D82100202022002001
:103B480000007A4400C07F44060B0020DBF8002008
:103B5800150442D5D4F89C208E4E8A1A002A3CDBE4
:103B680001F59C422032C6F89C208B4A50798B4A3A
:103B780032F81050A8B2FD7A90FBF5F596F8A0003F
:103B8800013000F00F0286F8A020324482F8A150DC
:103B98001A46804800F1A1055D5D01332A44102BC7
:103BA80092B2F6D112B292FBF3F31BB2642BA8BF08
:103BB800642323EAE37307EE903A9FED797AF8EEEF
:103BC800E77AC7EE877A9FED777A67EE877AFCEE19
:103BD800E77A17EE903AA0F89830DBF80030724E8A
:103BE80013F4807F00F0F780704B714D994203D930
:103BF800AB780BB90123AB70AB78002B00F0EB80EE
:103C08006B4B96F8008093F82170D4F89430781EA6
:103C180047424741002FC8F38008C3F3806914BFA7
:103C28004FF0000A4FF0030A95F82030052B00F2F8
:103C3800CC80DFE803F0034C5175829CB8F1000F8B
:103C480038D0D4F8B400B4F8B81003F04DFE012809
:103C580008D1584A584B12681B68D288642101FB66
:103C680002332B61B9F1000F0CD0524B1B681B7942
:103C780043B107F039FF032385F820304FF47A73F6
:103C8800EB61D1E7002F40F0A0804B4B48491A6800
:103C98002B699A420AD9019107F026FF019903235B
:103CA80081F8203040F6B833CB61BDE7012381F8B5
:103CB8002030B9E74FF48060B9F1000F02D002F06C
:103CC8003FF801E002F02BF800232B617DE0002F84
:103CD80044D107F009FFA7E727B1052385F820306D
:103CE800012100E03946B8F1000F0CD0D4F8B43007
:103CF800DA89324B1A805A809A802E4A1268528882
:103D0800DA804FF0020A2C4B1A686B699A4202D883
:103D1800B8F1000F56D147F23053EB6103231EE090
:103D2800337843F00203337008F026FD224BEA692A
:103D38001B681344AB61042311E01F4B97B11A6849
:103D4800AB699A4241D91E4B1B781BB9D4F8943001
:103D5800D9073AD4337823F002033370052385F862
:103D6800203061E71B68EA691344AB612DE0114A12
:103D7800114B12681B68D288642101FB02332B6146
:103D88004FF48060002385F82030EB7001F0C7FF06
:103D98004AE700BFD80A0020E40D0020F40D0020F7
:103DA8000000C84200C07F44E0220020404B4C0085
:103DB800D8210020FC2100204C1A0020E00C002013
:103DC8001400002000297FF42FAFBAF1000F02D0B1
:103DD800504603F049FFA94D05F5C570B5F85211D5
:103DE80003F082FD074650B907F070FEA44B1F6030
:103DF8005F609F60A34B00221A605A609A60337814
:103E08005A0738D5DBF80030DB0634D594F8BA30D9
:103E1800DFF87C82D8062ED49B4B1B7833B395F8F9
:103E2800E2318FB95BB1994B1A68D8F8BC309B1A4C
:103E3800002B04DA08F0A0FC88F8C0701BE0102002
:103E480003F012FF01230EE03BB1904A12684FF4D1
:103E58007A7101FB0323C8F8BC3094F8C03053B121
:103E680003F0EAFE002384F8C03004E0002FE6D017
:103E780098F8C030F3E7002295F8E09195F8E10151
:103E8800B5F89AE1B5F89CC11346DFF8188238F9FD
:103E980012109B087145C4BF63F07F03DBB2013287
:103EA8006145B8BF43F04003042AEED194F8C1201D
:103EB80077499A4205D191F8C220F92A04D80132EB
:103EC80000E0002281F8C22084F8C1306E4B704AAD
:103ED80019789A46C9B9D2F89430D90706D5A7B93E
:103EE8003378DA0711D508F011FC0EE033785B0758
:103EF8000BD592F82B3043B1664BDB782BB910B158
:103F080008F03AFC01E0002FFAD094F8C230604A79
:103F1800614F142B40F084809AF8003019F10009A1
:103F280018BF4FF001096BB392F8C1305F2B11D164
:103F3800337803F0040303F0FF0113B108F01CFC0D
:103F480008E00B200291019203F08EFE019A02997B
:103F580082F8C210B9F1000F14D094F8C1307D2B4B
:103F680010D1337803F0040303F0FF0213B108F013
:103F780003FC07E00B20019203F076FE444B019A04
:103F880083F8C220337803F0040303F0FF01002B09
:103F980046D194F8C1303E4A572B0BD13F4B4FF4D2
:103FA8007A7119803E4B1B6813F0080338D1A2F8C8
:103FB800C43035E0DBF80000400717D55A2B15D17F
:103FC80092F8C6302BB1012382F8C61082F8C730A8
:103FD80026E092F8C83083F0010382F8C8300BB1AC
:103FE8000C2000E00D2003F03FFE19E05D2B00F0EF
:103FF800D4835B2B00F0D3835E2B01D10320CFE366
:10400800562B01D102F042F99AF80030002B00F04B
:10401800DB8394F8C1306F2B40F0D08308F076FB37
:10402800DBF8003058074DD594F8C830184A93B1DA
:10403800337859070FD5B8F90610B5F89A3199426F
:1040480009DDD2F8943013F0010302BF3221A2F83F
:10405800CC1082F8C830D4F894200D4BD20323D565
:1040680093F8CE202AB993F8C62012B93222A3F8C1
:10407800CC20012384F8CE3024E000BF541A00205D
:10408800E80E00206C0F0020140000204C1A0020BD
:10409800D80A0020D8210020FC110020D8220020B6
:1040A80040220020E00C002093F8C62052B132785C
:1040B80002F0040202F0FF0122B9012283F8C610BF
:1040C80083F8C7203F680023C4F8943007F17B06C3
:1040D80007F1CB093278737816F8010C9A420DD2A1
:1040E800314603F0DBFB48B116F8022C012303FA32
:1040F80002F2D4F894301343C4F8943004364E4591
:10410800E8D1C34B1B783BB1D4F89430C14F13F0BE
:10411800020F40F0FB82F2E207F1CA0607F5897741
:104128003278737816F8010C9A4225D2314603F09A
:10413800B5FB08B3B37896F804E0B74A96F803904D
:10414800B6480C21013B01FB0E4103EB430313442A
:10415800D1F8D4209A420FD0C1F8D430002390F877
:104168000021C1F8D830012303FA0EF322EA030331
:1041780081F8D09080F800310636BE42D0D1A849E7
:10418800A84B0A680192D3F8009094F82B20A64F08
:104198000292002603933868002800F0A98201786B
:1041A800002900F0A5827B68019AD31A002B0ADB4C
:1041B80002F5FA7394F800E17B600123B3402EEA1C
:1041C800030384F80031029B002B00F0918217F85A
:1041D800043C42780433DBB2002A40F04F8238F9BD
:1041E80013E0B5F8983103F1C80CE64502DD90F804
:1041F80002A013E0C83B9E4503DA8378C3F1000AA6
:104208000CE094F800110123B34021EA030384F879
:104218000031019B03F5FA737B6069E294F80001B1
:104228003041C30700F16482BAF1000FCCBF02200D
:104238000120049103F03EFD0499784A481E132892
:1042480000F24F82DFE810F0140020002F00400039
:1042580059006200C10030018F01BE01EB014D021F
:1042680040004D006200C10030019200030160016E
:1042780099F8001001EB0A03FA2BA8BFFA2323EAE6
:10428800E37389F800300AE099F8011001EB0A039A
:10429800642BA8BF642323EAE37389F801304846F6
:1042A80003F0E2FA1DE299F8031001EB0A03642B0C
:1042B800A8BF642323EAE37389F803304846D2F899
:1042C800041103F087FA0CE299F8050050446428B9
:1042D800A8BF642020EAE0700D2989F8050000F0E5
:1042E800008299F8041001EB0A03642BA8BF642329
:1042F80023EAE37389F80430F3E199F8061001EB37
:104308000A0383F3080389F80630EAE1D2F8083192
:10431800187802281FD107EE90AAF8EEE77AB2EED5
:10432800047AC7EE877A93ED097A77EE877AF5EE05
:10433800C07AF1EE10FA09D49FED3D7AF4EE477A8F
:10434800F1EE10FAC8BFF0EE477A01E0DFED397AF6
:10435800C3ED097A07E098785044C828A8BFC82058
:1043680020EAE07098700F2900F0BB81D2F80801AC
:10437800017802291FD107EE90AAF8EEE77AB2EE8B
:10438800047AC7EE877A90ED087A77EE877AF5EEA9
:10439800C07AF1EE10FA09D49FED257AF4EE477A47
:1043A800F1EE10FAC8BFF0EE477A01E0DFED217AAE
:1043B800C0ED087A95E1417801EB0A03C82BA8BF44
:1043C800C82323EAE37343708BE1D2F808311878E5
:1043D800022831D107EE90AA9FED157AD3ED0C6A29
:1043E800F8EEE77AC7EE877A77EEA67AF5EEC07A26
:1043F800F1EE10FA07D4F4EE477AF1EE10FAC8BFDE
:10440800F0EE477A01E0DFED0B7AC3ED0C7A1BE0A2
:10441800DC220020B80E002058080108D80A002025
:104428004C1A002004220020AC0B002000007A4423
:104438000000C84200000000187B5044C828A8BFEC
:10444800C82020EAE0701873102900F04A81D2F8D9
:104458000801017802291DD107EE90AA1FED0C7AF8
:10446800D0ED0B6AF8EEE77AC7EE877A77EEA67A90
:10447800F5EEC07AF1EE10FA07D4F4EE477AF1EED1
:1044880010FAC8BFF0EE477A01E05FED167AC0ED8A
:104498000B7A26E1C17A01EB0A03C82BA8BFC8230F
:1044A80023EAE373C3721CE1D2F8083118780228B2
:1044B8001FD107EE90AA1FED237AF8EEE77AC7EE30
:1044C800877A93ED0F7A77EE877AF5EEC07AF1EE78
:1044D80010FA09D41FED2A7AF4EE477AF1EE10FAB1
:1044E800C8BFF0EE477A01E05FED2E7AC3ED0F7A90
:1044F80007E0987D5044C828A8BFC82020EAE0708B
:104508009875112900F0ED80D2F808010178022988
:104518001FD107EE90AA1FED3B7AF8EEE77AC7EEB7
:10452800877A90ED0E7A77EE877AF5EEC07AF1EE1B
:1045380010FA09D41FED427AF4EE477AF1EE10FA38
:10454800C8BFF0EE477A01E05FED467AC0ED0E7A1B
:10455800C7E0417D01EB0A03C82BA8BFC82323EAA3
:10456800E3734375BDE0D2F80801017802291FD131
:1045780007EE90AAF8EEE77AB2EE047AC7EE877AE9
:1045880090ED0A7A77EE877AF5EEC07AF1EE10FAB6
:1045980009D41FED597AF4EE477AF1EE10FAC8BF44
:1045A800F0EE477A01E05FED5D7AC0ED0A7A98E0B7
:1045B800C17801EB0A03C82BA8BFC82323EAE37319
:1045C800C3708EE0D2F80801017802291DD107EEE8
:1045D80090AA1FED697AD0ED0D6AF8EEE77AC7EE7A
:1045E800877A77EEA67AF5EEC07AF1EE10FA07D45C
:1045F800F4EE477AF1EE10FAC8BFF0EE477A01E020
:104608005FED747AC0ED0D7A6BE0417B01EB0A0334
:10461800C82BA8BFC82323EAE373437361E0D2F829
:104628000811087802281FD107EE90AA1FED817A99
:10463800F8EEE77AC7EE877A91ED107A77EE877A07
:10464800F5EEC07AF1EE10FA09D41FED877AF4EE90
:10465800477AF1EE10FAC8BFF0EE477A01E05FED55
:104668008B7AC1ED107A3CE0C87D00EB0A03C82BB9
:10467800A8BFC82323EAE373CB7532E0012A30D1FF
:1046880090F802E038F91300B0F5617F05DB40F6D9
:1046980033039842A8BF184601E04FF461700C2913
:1046A8001FD16B4A4FF4966393FBFEFE1378A0F577
:1046B800617090FBFEF0C0B2834212D0042834BF70
:1046C80003460223137001FB0351039B049001F27C
:1046D800CA61196001F01CFC04980130C0B203F0F3
:1046E800E9FA94F800110123B3400B4384F8003130
:1046F8000136042E07F10C077FF44DAD04E5DBF815
:104708000030DE0510D5534BDB786BB1524B1B687C
:10471800980709D53B8813F001060AD107F0D6F9A6
:10472800012001F00DFB04E0012001F0F8FA01235B
:1047380000E00023D4F8942051070CD55BB1012088
:1047480001F0EDFA3B889A0708D407F0BFF9022078
:1047580001F0F6FA02E0022001F0E1FA3B8813F0DA
:10476800030F3E4B4FF020020CBF9A611A85D4F814
:1047780094301B054FF4807002D501F0E1FA01E096
:1047880001F0CDFA6B79082B01D00E2B5DD14020BA
:1047980009B0BDE8F04F01F0C2BA012000E00220E4
:1047A8005FFA80F909F1FF3385F8C83601F012FB8A
:1047B80001F0D2FB484603F07DFA31E4B9F1000F6D
:1047C80002D07E2B3FF42AAC94F8C130244A972BB0
:1047D80004D14FF4C873A2F8CA3021E4A72B06D13C
:1047E80092F8BA3043F0040382F8BA3018E4002291
:1047F800BB2B079201D1022303E0B72B04D14FF65C
:10480800FE73ADF81E300AE0BE2B01D1022304E08E
:10481800BD2B7FF405AC4FF6FE73ADF81C303B683A
:10482800BDF81C10B3F858200A44A3F85820BDF866
:104838001E10B3F85A200A44A3F85A2001F026FDA6
:10484800002384F8C230FFF7EBBB09B0BDE8F08F56
:1048580000220020D8210020402200200004004827
:10486800D80A002010B5214A18B9136802221A8202
:1048780010BD1F48146800230380217811F07F01C0
:1048880002460DD1637A990644BF0221017013F0E4
:10489800400F037814BF43F0010323F0010315E030
:1048A800012921D002291ED1637913F0800F03F06A
:1048B8000F034FEA830303F1804303F5B8431B68F2
:1048C80006D003F03003102B07D10123137004E046
:1048D80003F44053B3F5805FF6E7064B1B681B698A
:1048E8009847034810BD184610BD00BF101A002095
:1048F800E80B0020001A002010B5064C18B92368F0
:1049080001221A8210BD044B1B689B6898472068D7
:104918000C3010BD101A0020001A002010B5064CEB
:1049280018B9236801221A8210BD044B1B681B6842
:10493800984720680A3010BD101A0020001A00207D
:1049480003788B4283BF034B03EB41014888002067
:10495800704700BFE80B002070B5002213462449B9
:1049680014180C44A47E83EA0423082413F4004F8B
:104978004FEA430318BF83F4815304F1FF3418BF8F
:1049880083F0010314F0FF049BB2EFD10132192A1E
:10499800E5D100F1190200F11A050A440D44967E8A
:1049A800AA7E02EB062292B29A421FD1104B93F8CC
:1049B8003B50E2B2AA4216D2431C03EB4203DBB2DD
:1049C800CA1801330B44927E9B7E03EB02239BB2F1
:1049D8004FF4AF6253431B13064A03F5487322F89A
:1049E80014300134E5E7012381F83C3070BD00BF85
:1049F800E80B0020EA0B002003788B420BD9074B09
:104A08001A78074B89001944086C02B1400800F570
:104A1800777080B270470020704700BF4C2100209B
:104A2800E80B002007299DBF034B03EB8101B1F878
:104A380070000020704700BFE80B0020034B03EB19
:104A48004101B1F89000C008704700BFE80B002092
:104A58000A4BDFED0B7A03EB810191ED2C7AB8EE6E
:104A6800477AF6EE046AE7EE267A82B0FCEEE77A39
:104A7800CDED017ABDF8040002B07047E80B0020C4
:104A880000005C44024B03EB4101B1F8F8007047A9
:104A9800E80B0020024B03EB4101B1F81C01704701
:104AA800E80B002070B5334C054602F037FFD4F808
:104AB8003431C4F83401C31AB3F5FA5FC4F8383195
:104AC80082BF002384F83C3184F83D3194F83C31AE
:104AD8002BB9A12D02BF274A012182F83D1194F874
:104AE8003D11244A29B1D118EDB201338D7682F8EF
:104AF8003C3194F83C5194F83E31AB4239D11D4BCE
:104B080093F83F31052B02D0062B03D02CE0002070
:104B1800FFF722FFE37E1E2B26D100200246C1B2FA
:104B28006B1E994219DA21448B7E0821DBB283EA95
:104B38000206F60744BF83F01803C3F3460301F1E6
:104B4800FF3154BF5B0843F0800311F0FF01C2F34B
:104B58004702ECD101301A46E1E723449B7E9A4292
:104B680002D10320FFF7F8FE002384F83D3184F8D2
:104B78003C3170BDE80B002010B5044602F0CEFEB3
:104B88000F4BD3F84021C3F84001821A41F2883113
:104B98008A42C3F8442184BF002283F8482193F84D
:104BA8004821074913440F2AE4B218BF013283F899
:104BB800494112BF81F84821012381F8593110BDBC
:104BC800E80B002010B5044602F0A8FE0F4BD3F8FE
:104BD8005C21C3F85C01821A41F288318A42C3F829
:104BE800602184BF002283F8642193F86421074977
:104BF8001344142A18BF013283F8654112BF81F8A3
:104C08006421012381F87A3110BD00BFE80B002030
:104C180038B5044602F082FE274A2749D2F87C318B
:104C2800C2F87C01C31AB3F57A6F84BF002382F8F7
:104C3800803192F8803133B9A82C3BD181F8813189
:104C4800A1F8823106E0022B02D181F8844101E00B
:104C5800242B02D8D11881F8854192F88411164D79
:104C680001330231DBB249008B4282F8803118DA15
:104C7800B5F88231E0B283EA0020082310F4004F2F
:104C88004FEA400018BF80F4815003F1FF3318BF8A
:104C980080F0010013F0FF0380B2EFD1A2F8820187
:104CA80038BD01318B4201BF002385F880310123D3
:104CB80085F8813138BD00BFE80B002010B50446E7
:104CC80002F02CFE104AD2F8AC3140F6AC51C31AAF
:104CD8008B42C4BF002382F8B03192F8B031D118AA
:104CE80081F8B14123B90F2C0DD10749C1F8AC01A6
:104CF8000133DBB2192B044982F8B0310CBF012310
:104D0800002381F8CA3110BDE80B00202DE9F843D3
:104D1800324F3D682A8A2E7AB2B9042E14D1304C0B
:104D280030482378012B0BD12F4B19682F4B89B2B0
:104D38000B445B0019681A6030230380227048E036
:104D480010230380072644E0AC8AAB69A24294BFD3
:104D580004260226944228BF14461FFA84F84046C7
:104D68009847214A13689BB203F1005303F5405357
:104D78005B0004F1010E1B689BB203F1005303F5BD
:104D880040534FEA6E0E5B000021714500F10200AE
:104D980009D010F8019C10F802CC4CEA092C23F831
:104DA80021C00131F1E71268104B92B213445B0045
:104DB8001A681C602B8AC8EB03032B826B8A984401
:104DC800084BA5F8128030221A80094B4FF4405244
:104DD8001A803B681E72BDE8F88300BF101A0020D5
:104DE800DE220020FA190020505C0040023000202A
:104DF800F81900200E4B0F4A1B689BB203EBC0004A
:104E080002443E294FEA420209D94B09C80604BFA9
:104E180003F1FF339BB29B0243F4004304E04B08C9
:104E2800C90748BF01339B0211681360704700BF70
:104E3800505C00400630002010B5454B1A681078C9
:104E480010F07F0004D1537A23F02003537210BD71
:104E580002287AD15388002B78D11379002B75D189
:104E6800537923F08000840004F1804101F5B841B2
:104E780013F0800F096814BF01F0300101F44051AC
:104E8800032862D8002960D0927A002A5DD004F104
:104E9800804404F5B8441906226825D502F030028A
:104EA800102A4CD103F07F039B0003F1804303F5E4
:104EB800B8431A68510641BF196840F60F720A4094
:104EC80042F4004244BF42F0C0021A601A6822F459
:104ED800E04222F0400292B282F0300242F40042F4
:104EE80042F080021A602AE002F44052B2F5805F74
:104EF80025D128B9174B93F82C10FFF77BFF11E049
:104F08009B0003F1804303F5B8431A68520441BF7C
:104F1800196840F60F720A4042F4404244BF42F01A
:104F280080021A60236823F4804323F070039BB245
:104F380083F4405343F4004343F080032360064B5B
:104F48001B685B699847002010BD022010BD00BF98
:104F5800101A0020AC000020001A00208A6803689C
:104F680010B50C6A14430A6914434A6914438A69E0
:104F78001443CA6914434A6A14438A6A23F4FF43F0
:104F880023F070032243134303608B8943600B684B
:104F980083604B68C36010BD02684FF6FE73134010
:104FA80003600023036043608360C360284B98421A
:104FB80001D1284A27E0284B984201D1254A2AE006
:104FC800264B984201D1234A2DE0254B984201D126
:104FD800204A30E0234B984201D11E4A33E0224B4D
:104FE800984204D11B4A536843F470032EE01F4BC8
:104FF800984204D1174A536843F0706326E01C4B6B
:10500800984204D11B4A536843F00F031EE01A4B21
:10501800984204D1174A536843F0F00316E0174B3F
:10502800984204D1134A536843F470630EE0144B5A
:10503800984204D10F4A536843F4704306E0114B79
:10504800984204D10B4A536843F470235360704765
:1050580008000240000002401C00024030000240EC
:1050680044000240580002406C00024080000240A8
:1050780008040240000402401C04024030040240BC
:105088004404024058040240084BDA68D10709D4A6
:10509800DA68D20608D4DB6813F0040F14BF0320C3
:1050A800042070470120704702207047002002400A
:1050B800994A536803F00C03042B2DE9F04105D0FD
:1050C800082B06D095490160B3B916E0934B0360ED
:1050D80012E053685468C3F38343991CE30349BF40
:1050E800D36A8F4B8D4C03F00F0344BF0133B4FBDD
:1050F800F3F34B43036000E000235168894FC1F389
:1051080003117D5C0168EDB221FA05F4446056682C
:10511800C6F30226BE5D24FA06FEC0F808E056680B
:10512800C6F3C226BE5DF6B2F440C460D2F82C8045
:10513800C8F3041808F00F0C07EB4C0C18F0100F0C
:10514800BCF810C01FFA8CFC07D0BCF1000F04D0CB
:10515800B3FBFCFCC0F810C000E00161D2F82CC021
:10516800CCF3442C0CF00F0807EB48071CF0100F89
:105178003F8ABFB204D01FB1B3FBF7F7476100E025
:105188004161176BFF065ABF644F87618161176BD6
:10519800BF065ABF614FC761C161176B7F065ABF0F
:1051A8005E4F07620162176BFF0506D5994204D16D
:1051B800AE4202D14F00476200E04462176BFF0421
:1051C80006D5994204D1AE4202D14F00876200E071
:1051D8008462176BBF0506D5994204D1AE4202D14D
:1051E8004F00C76200E0C462176B7F0506D599427D
:1051F80004D1AE4202D14F00476400E04464176B0B
:105208003F0506D5994204D1AE4202D14F008764CA
:1052180000E08464176BBF0406D5994204D1AE42FE
:1052280002D14B00C36400E08464156B3A4BAD07B0
:1052380001D1046315E01C6B04F00304012C01D1B7
:1052480001630EE01C6B04F00304022C02D14FF43E
:10525800004305E01B6B03F00303032B01D12F4B25
:105268000363146B2C4B14F4403F02D1C0F834E0B4
:1052780018E01C6B04F44034B4F5803F01D141635D
:1052880010E01C6B04F44034B4F5003F02D14FF435
:10529800004306E01B6B03F44033B3F5403F01D1F4
:1052A8001E4B4363146B1C4B14F4402F02D1C0F8FF
:1052B80038E018E01C6B04F44024B4F5802F01D1C9
:1052C800816310E01C6B04F44024B4F5002F02D174
:1052D8004FF4004306E01B6B03F44023B3F5402F63
:1052E80001D10E4B8363146B0B4B14F4401F02D196
:1052F800C0F83CE020E01C6B04F44014B4F5801FB7
:1053080001D1C16318E01C6B04F44014B4F5001F0C
:105318000AD14FF400430EE00010024000127A0058
:1053280000093D00160000201B6B03F44013B3F581
:10533800401F01D1134BC363126B134B12F4400F80
:1053480003D1C0F840E0BDE8F0811A6B02F44002D6
:10535800B2F5800F02D10164BDE8F0811A6B02F446
:105368004002B2F5000F02D14FF4004306E01B6B78
:1053780003F44003B3F5400F01D1024B0364BDE8C9
:10538800F08100BF00127A0000100240F0B500233F
:105398000E681C460125A54005EA060EAE452BD130
:1053A8000F797A1E012A15D8856803229A4025EAC2
:1053B800020282604D7982689D401543856082882B
:1053C80092B222EA0E0282808A798588A2402A4314
:1053D80092B28280032205689A40D2431540056044
:1053E80005689F402F430760C7681740CA7902FACB
:1053F80003F547EA0502C2600134102C03F10203E9
:10540800C8D1F0BD38B52DED048B4A4C0368C4F8FB
:10541800CC318388A4F8D031013A0D46072A42D806
:10542800DFE802F0040A101822292F35B4F8CC312D
:105438000B80B4F8CE3113E0B4F8CE310B80B4F859
:10544800CC3105E0B4F8CC315B420B80B4F8CE31F6
:105458005B4205E0B4F8CE315B420B80B4F8CC3146
:105468006B80B4F8D0311DE0B4F8CC315B420B80CE
:10547800B4F8CE3112E0B4F8CE310B80B4F8CC31A8
:105488000CE0B4F8CC310B80B4F8CE3105E0B4F8B8
:10549800CE315B420B80B4F8CC315B426B80B4F800
:1054A800D0315B42AB80244B93F83030002B3ED197
:1054B800B5F9003094ED780AD4ED757A09EE103A12
:1054C800B5F9023008EE103AB8EEC88AB5F90430DA
:1054D800B8EEC99A28EE000A08EE903AA7EE890AB3
:1054E800F8EEE88AD4ED7B7AA7EEA80A09F078FEF0
:1054F80094ED790AD4ED767A288028EE000AA7EE92
:10550800890AD4ED7C7AA7EEA80A09F069FE94ED21
:105518007A0AD4ED777A688028EE000AA7EE890A1D
:10552800D4ED7D7AA7EEA80A09F05AFEA880BDEC52
:10553800048B38BDE80B002016000020094BD3F877
:10554800F821137844F6FB7103EB431300FB0313B4
:105558005078C0EB0030B3FBF0F39078B3FBF0F079
:1055680080B27047E80B002010B50A4C94F8FD3162
:1055780004EB43030A22B3F80C1204F5067089B24F
:10558800A4F8141201F0E4FB80B2FFF7D7FFA4F8E7
:10559800A00210BDE80B0020F0B50124B0FBF4F523
:1055A8008D4201D34C43F9E70026D4B1B0FBF4F5A2
:1055B80004FB1500B4FBF1F41EB9002D01DC002C2E
:1055C800F3D1092D03F1010EEFB204DD002A14BF57
:1055D8003725572500E030253D441D7001367346B8
:1055E800E3E71C70F0BDF0B50124B0FBF4F58D4283
:1055F80001D34C43F9E70026D4B1B0FBF4F504FB22
:105608001500B4FBF1F41EB9002D01DC002CF3D118
:10561800092D03F1010EEFB204DD002A14BF37256E
:10562800572500E030253D441D7001367346E3E7F9
:105638001C70F0BD2DE9F843089E002B07468846EC
:10564800144614BF4FF030094FF02009334613F8C1
:10565800012B0AB9254603E0002CFBDD013CF6E7E7
:10566800002D04DD38464946C047013DF8E724EAE5
:10567800E4743546A01B284415F8011B11B13846BF
:10568800C047F7E7BDE8F883014B186802F065BB2F
:10569800D003002090ED017A07EE901AB5EE407A1B
:1056A800F1EE10FA01BFF8EEE77A9FED0E7A67EE99
:1056B800877AB7EE007A04BFC7EE277AC0ED017A81
:1056C80090ED017AD0ED007A30EE877A30EE670AF5
:1056D800C0EE870AE0EE807AB0EE670AC0ED007A85
:1056E800704700BFDB0FC94010B50278202A034677
:1056F80000F10100F9D0092AF7D02D2A03D1034679
:10570800BFEE000A04E02B2A08BF0346B7EE000AE2
:10571800DFED387A1A46134612F8010BA0F1300172
:10572800CCB2092C0AD807EE101AB8EEC77AF2EEF6
:10573800046AA7EEA67AF0EE477AECE72E2816D18F
:10574800F2EE046A1146B0EE666A0B4611F8012BB8
:10575800303AD0B209280AD807EE102AB8EEC77A2C
:1057680087EE267A66EE866A77EE877AEDE71A780C
:1057780002F0DF02452A35D15A782D2A02D10233A8
:10578800012004E02B2A14BF013302330020013B1F
:10579800002213F8011F3039CCB2092C03D80A248F
:1057A80004FB0212F5E7B2F59A7F28BF4FF49A720C
:1057B8001346B7EE007A072B05D9DFED0F6A083BD1
:1057C80027EE267AF7E702F007032BB1F2EE046A18
:1057D80027EE267A013BF8E7F0EE476A20B1C7EEDC
:1057E800877A03E0F7EE006A67EEA67A20EE270ACA
:1057F80010BD00BF0000000020BCBE4C30B52DED30
:10580800028B87B0B0EE408A0C220021054603A81F
:1058180009F0D7FAB5EEC08ADFED2A7AF1EE10FA70
:10582800CCBF38EE278A38EE678ADFED277A28EE74
:10583800278A6946FDEEC87A17EE904A84EAE47032
:10584800A0EBE47005F0DAFB002CACBF20232D237D
:1058580068468DF80C3009F0F8FA012807D1302392
:105868008DF80D308DF80E308DF80F300CE00228D1
:1058780005D130238DF80D308DF80E3004E0032863
:1058880004BF30238DF80D30694603A809F0C0FA2B
:1058980003A809F0DAFA0338C4B2224603A9284655
:1058A80009F000FB00232B552846084909F0B0FAF7
:1058B80003AB2846191909F0ABFA284607B0BDEC26
:1058C800028B30BD6F12033A00007A44A721010809
:1058D80070B5064615460846B6FBF2F414B12046E4
:1058E800FFF7F6FF05FB1464024B1B5D00F8013B54
:1058F80070BD00BFA92101080FB42DE9F04F7C4B02
:1059080089B012ACD3F800807A4B54F8046BD3F802
:105918000090049400253178002900F0868025291C
:1059280002D00136404674E07278302A08BFB27857
:10593800A2F1300319BFB71C4FF0000BF71C4FF052
:10594800010B092B4FF0000A19D8A2F13003D9B284
:10595800092905D80A2202FB0A3A17F8012BF4E7AD
:10596800A2F16103052B02D8A2F1570305E0A2F1C9
:105978004103052B03D8A2F137030A2BEADD6C2A71
:1059880030D13A78642A07F1010600F088800AD8F5
:10599800252A3CD002D8002A47D0BCE7582A0CD088
:1059A800632A19D0B7E7732A22D002D86E2A37D0D3
:1059B800B1E7752A62D0782AADD1271D2068A2F1F7
:1059C800580462424FF0100162415BE02CD9582A1A
:1059D80038D0632A34D13E4640462178271DC8472F
:1059E80001350FE0642A6AD00ED9732A14D13E46D5
:1059F800236800934046494652460023FFF71AFEA3
:105A0800271D05443C4686E7252ADFD13E46404609
:105A18002521C84701357EE70ED86E2A10D13E46AB
:105A2800236804341D6076E752B9334B186802F0D6
:105A380091F90028F9D054E0752A28D0782A01D0A5
:105A48003E4668E7A2F1580304F1040C5A42206864
:105A5800CDF80CC04FF010015A4105ABFFF79CFD83
:105A6800DDF80CC03E46644605AB00934046494607
:105A780052465B46FFF7DEFD05444CE72068271DCC
:105A88000A21002205ABFFF7AEFD3C46ECE704F126
:105A9800040CCDF80CC020680A210022DDE720683C
:105AA800002804F1040708DA2D238DF81430404249
:105AB8000DF115030A210022E5E705ABFAE7206896
:105AC800002804F1040C0ADA2D238DF81430404222
:105AD8000DF11503CDF80CC00A210022BEE705AB75
:105AE800F8E7284609B0BDE8F04F04B0704700BF9A
:105AF8007401002070010020D003002080EAE073C8
:105B0800A3EBE0738B4206DB002801DD401A7047E7
:105B180002D00844704700207047FDEEC07A17EEA7
:105B2800903A2033402B43D8DFED237AB4EEE70ACE
:105B3800F1EE10FA04DDDFED217A30EE670AF3E7C3
:105B4800DFED1F7AB4EEE70AF1EE10FA04D5DFEDC7
:105B58001B7A30EE270AF3E7DFED1A7AB4EEE70A8C
:105B6800F1EE10FA04DD30EE670A37EEC00A0AE0FB
:105B78009FED157AB4EEC70AF1EE10FA44BF30EE85
:105B8800270A37EE400A60EE007ADFED106A9FEDD3
:105B9800107AA7EEA67ADFED0F6AE7EE876A9FED27
:105BA8000E7AA7EEA67A20EE276AA6EE070A7047B5
:105BB8009FED0A0A704700BFDB0F4940DB0FC94061
:105BC800DB0F49C0DB0FC93FDB0FC9BF9A7C2E36FC
:105BD800FAAF4FB93587083CA4AA2ABE00000000D6
:105BE80038B52DED068B90ED008ADFED2D9A38EE55
:105BF800290A0C460546FFF790FFB0EE40AAB0EE22
:105C0800480AFFF78AFFD5ED018AB0EE409A38EED0
:105C1800A90AFFF782FFB0EE408AB0EE680AFFF7E4
:105C28007CFFD5ED02AAF0EE408A3AEEA90AFFF70A
:105C380074FFF0EE409AB0EE6A0AFFF76EFF60EE6E
:105C48000A6A69EE297AF0EE665AE7EEA85A29EE52
:105C58008A6A29EE007A69EE889A29EE489A28EE2F
:105C6800400A28EE0A8AC4ED035AF0EE465AE7EED7
:105C7800685AE6EEA87AA6EE687AC4ED009AC4EDF2
:105C8800028A84ED059A84ED088ABDEC068B84EDC2
:105C9800010AC4ED045A84ED067AC4ED077A38BDCA
:105CA800DB0FC93F10B52DED048B8AB090ED009A3B
:105CB800D0ED028A90ED018A0446084601A9FFF753
:105CC8008FFFDDED047A9DED017A68EE277AE9EE23
:105CD800077A9DED077AE8EE877A9DED027AC4EDA2
:105CE800007ADDED057A68EE277AE9EE077A9DED10
:105CF800087AE8EE877AC4ED017ADDED067A28EEB7
:105D0800278ADDED037AA9EE278ADDED097AA8EE68
:105D1800A78A84ED028A0AB0BDEC048B10BD074B3C
:105D28001A8822EA0000904210B518801C4602D05A
:105D3800012001F0BFFF208810BD00BFB80E002071
:105D4800064B1A881043904210B518801C4602D0A2
:105D5800012001F0AFFF208810BD00BFB80E002061
:105D6800024A936823EA000090607047541A0020A2
:105D7800024A936818439060704700BF541A002085
:105D880008B5104B1A780023D9B2914207D20E49B0
:105D980051F823100968002008600133F4E7322025
:105DA80001F0E3FD094B1B685A0309D5084B9B68B2
:105DB8005B0305D440F2DC50BDE8084001F0D5BDD6
:105DC80008BD00BF5B0F0020980F00202422002090
:105DD800541A00202DE9F743474F484A4B233B709C
:105DE800692313704FF4DE635380BE231371EF23CE
:105DF80082F8EE36002382F8EF3619461646F25C32
:105E08000133B3F5DE6F81EA0201F8D13B4B83F829
:105E1800EF163B4B1A69120604D53A4A5A6002F14A
:105E280088325A604FF00408002008F1FF3818F053
:105E3800FF084FD0324B3422DA60002444B10023EB
:105E480056F80490019305F0AAF80428EDD117E05C
:105E580005F0A5F80428E8D1294D2B6943F0020381
:105E68002B61294B6B612B6943F040032B6105F0D3
:105E780096F82B69042823F002032B61DFD0D4E7BE
:105E88001F4D2B6943F001032B6104F1006303F5F7
:105E98007E331FFA89F21A8005F081F8042810D1A0
:105EA8001A4B23440193019B4FEA1949A3F8009028
:105EB80005F075F82B69042823F001032B6105D040
:105EC800B3E72B6923F001032B61AEE70434B4F583
:105ED800DE6FB3D10A4A1369042843F080031361C3
:105EE80002D102F0A0FF10B90A2001F0FBFE022344
:105EF8003B7003B0BDE8F083DD0A0020541A00208F
:105F0800002002402301674500F8030802F803084F
:105F180010B50E4C206801F0A7FC2068047A002216
:105F280002FB02F3193B634303F6C41353431921DD
:105F380093FBF1F3064921F812300132072AEFD119
:105F48000449BDE8104001F045BC00BF0422002010
:105F5800F8020020981B00202DE9F84302F063FFA7
:105F680010B90A2001F0BEFEA94CAA4EAA49AB4DB1
:105F78004B234FF4DE622046337008F017FF94F885
:105F8800C836022B84BF002384F8C83694F8C82684
:105F98004FF4C67101FB02F3E018234400F50970C1
:105FA800286093F8780203F51C73022801FB02426B
:105FB80084BF0020187292F87832994A13700C2224
:105FC80002FB0343974A03F2CA631360A26846F2CE
:105FD800090313401BB94FF40050FFF7C9FEA3682B
:105FE800D80703D54FF40050FFF7BAFEA368590449
:105FF80009D50820FFF7B4FE4FF40050FFF7B0FEB4
:106008000120FFF7ADFEA3681A0706D54FF400502C
:10601800FFF7A6FE0120FFF7A3FEA3689B0402D5A5
:106028004020FFF79DFE94F8E021794B2AB193F8C0
:10603800E42112B1002283F8E4217B4B7B4F1F60DF
:106048004FF00008C64604EB0803B3F8F4C14FEA62
:106058005C0101F077314FEA9C0303F03333C1EB65
:106068000C00C11A4FEADC0303F01133CB1A03EB1F
:1060780023131CF0010903F00F324FF0FF0392FBCA
:10608800F3F3C3EB032318BF0EF1010EA2EB0303D6
:1060980018BF5FFA8EFE012B0ADD022B40F0B58097
:1060A800B9F1000F00F0B1801CF0BC0F00F0AD801A
:1060B80008F10808B8F1200FC5D10EF1FF3EBEF176
:1060C800010F00F2A280FFF723FF00213022584879
:1060D800DFF8B48108F075FE564BD5F80090C3F888
:1060E8000080554B09F17900C3F8009004F048FF8F
:1060F800524B80F001001870514B08F126021A60CB
:1061080099F8000001F060F84E4B94F8D801DFEDE3
:106118004E6A08F194021A6064214C4BC82211FBA4
:1061280000225A6000229A60DA601A615A619A6104
:10613800DA6183F8202083F82120454B08F12C02EE
:106148001A602B68434A93ED187A03F2191111600B
:10615800414A03F289111160404A08F108011160AF
:106168003F4AC2F800803F4A08F1A00111603E4A48
:1061780008F1AA0111603D4967EE266A0F60B4F87C
:106188006611B6EE007A07EE901A87EE267AB4F812
:106198006811101DF8EE677AC2ED027A07EE901AC0
:1061A80093F85C10117193F87810517194F8E31119
:1061B8001174F8EE677AB3F81611C2ED037A07EE98
:1061C800901A2B4908602B49536103F16400086059
:1061D8002949936181ED007AF8EEE77A9FED277AF5
:1061E8002749C2F82480C7EE277A9FED267A67EE02
:1061F800877AC1ED007A03F1680103F21113136283
:1062080002233370D161BDE8F88304F08BFE5AE7AE
:10621800541A0020DD0A002000F80308FC110020B1
:10622800002200200422002020220020DE1B002063
:10623800A80B0020DC0B0020E00B0020140000203D
:1062480028040020FC210020DB0F4940D821002031
:1062580080040020001200208C06002090100020EE
:1062680094100020A0050020900E00206406002055
:10627800B0040020E8040020E40400200000614489
:106288009C0500204C3D0F44981B002008B5FFF7E3
:10629800A1FDFFF761FE0120BDE8084001F00ABD3D
:1062A8002DE9F04F2DED028B87B006460593984BEC
:1062B800B3F800A00AF002081FFA88F39346039384
:1062C800B3B3129B9348DC89B0F900301B1B03F26F
:1062D800F31540F2E632954203D8002BB8BF5B4273
:1062E80001E04FF4FA73B0F90220121B02F2F31422
:1062F80040F2E630844203D8002AB8BF524201E097
:106308004FF4FA729342B8BF1346C3F5FA730522E5
:1063180093FBF2F30A22643B5343327FD210534378
:10632800642293FBF2F3134423EAE373DBB200E045
:106338006423019301F1030937464FF00008B8F1CF
:10634800020F19F8014F06D1714AB2F906201B3421
:106358005443621142E0704A32F91850CBF10002FE
:10636800690091424FEA480003DB59450A46A8BF35
:106378005A466A49059B415E511A33F918208B1811
:1063880008EE103A04F0AEFE70B1B8EEC80A644ADE
:10639800B2EE048A80EE080A12F8080004F0A4FCA1
:1063A80020EE080ABDEEC08A1AF0010F11D11B3485
:1063B800039B6C4322118BB1B17C9DF9040018EE4C
:1063C800103A59434143642091FBF0F102EB21124A
:1063D80004E0347A18EE103A5C4322114C4D05F172
:1063E8000A01042431F9181091FBF4F4141B05F187
:1063F80010024FEA4803049318F802307A7802939F
:1064080062435A43642192FBF1F296F85110D3117A
:1064180008EE103AB9B1B8F1020FB8EEC80A08D1BF
:106428004A0803D09142A8BF114600E001213D4827
:1064380003E005F1140000EBC800D5ED0B0AFFF7E7
:1064480029F9BDEEC08A324B374AFD7A108803F12C
:10645800300C00FB04F25CF82810D21205FB021580
:10646800B5F5001F314AA8BF4FF4001503F13C01F0
:106478009542B8BF154651F8282041F82840A21A7D
:106488004FF6FF7103F154040009B1FBF0F04243E9
:1064980003F148004CF8285054F8281050F828C048
:1064A80044F828C092116144114400EE101A96F87D
:1064B800501040F828206D1359B103F16000B8EE70
:1064C800C00A00EBC800D3ED0B0AFFF7E3F8BDEEF6
:1064D800C00A18EE103A2B44797D029A1D4610EE38
:1064E800103A59434A43049B642108F1010892FB7E
:1064F800F1F10F4A05EB2121B8F1030F995207F189
:1065080001077FF41CAF07B0BDEC028BBDE8F08F2C
:10651800B80E0020E00C0020BA0E0020221A00203D
:1065280094080108DC0E0020542200200000E0FF3F
:10653800300F00202DE9F04F2DED028B87B000259C
:106548000593C14B0491B3F90480B3F90230039267
:10655800B8F1000FB8BFC8F10008002BB8BF5B4204
:106568009845B8BF9846B8F5FA7F0746A8BF4FF4D4
:10657800FA780190AA460295A9462C46B24BB3F880
:1065880000B01BF0030650D00233610033F9142029
:10659800039B52005B429A4203DB039B9342A8BFD2
:1065A8001346AA4A8A5E9B1A059A32F914201344A4
:1065B80008EE103A04F096FD68B1B8EEC80AA44B8C
:1065C800B2EE048A80EE080A185D04F08DFB20EE16
:1065D800080ABDEEC08A397F3A7A18EE103A6FF091
:1065E800040909FB01F95343642293FBF2F24A457B
:1065F80004DB01EB81099145A8BF9146954918EE46
:10660800103A51F82420134442F210729342A8BF62
:106618001346914A9342B8BF1346BA7C41F82430D6
:1066280053431B13012E029339D08C49019B31F936
:1066380014A093F801E001F108032E3133F9140096
:1066480051F8246080EAE073A3EBE073B3F5206FA0
:106658004FEA840516DC0AEB8A031A0192FBFEF363
:10666800042290FBF2F0181A0644B6F57A5FA8BF28
:106678004FF47A567A4B9E42ACBF41F8246041F8F9
:10668800243002E0002341F824304B597D2593FB48
:10669800F5F5019BDB7A6B43402593FBF5F51BF081
:1066A800020F11D0029BC8F5FA7208FB0AF008FB2A
:1066B80005F64FF4FA7102FB090002FB036690FB32
:1066C800F1F096FBF1F606E01BF0010F13BF029EF6
:1066D8002E46504648465C4A02F10A034FEA440BEC
:1066E80033F91410042391FBF3F302F18801615C80
:1066F8004B436FF04F0193FBF1F397F85110C31818
:1067080008EE103A59B102F11400B8EEC80A00EBCD
:10671800C400D2ED0B0AFEF7BDFFBDEEC08A4A4A9F
:1067280002F10A0302F18C003BF803E03BF9003068
:106738002BF800E00FFA8EF102F1900002F1980EAA
:10674800CB1A50F824C0042193FBF1F15EF82430F1
:1067580040F8241063440B4497F850104EF824C0B6
:1067680000EE103A59B102F16000B8EEC00A00EB31
:10677800C400D2ED0B0AFEF78DFFBDEEC00A324A07
:1067880018EE103A02F1A00033441E46005D10EEE8
:10679800103A4343202093FBF0F3F61A019B02F1D1
:1067A800780101332BF8016001930CB90124E5E667
:1067B800049BB2F906109B79B2F90E00946B0F3363
:1067C8005B004B435B11002BA3EB0000B8BF5B429F
:1067D800322B797B0BDC234B01FB00418B42A8BF9A
:1067E8000B4621498B42ACBF9363916301E00023C0
:1067F8009363F97801FB00F392F8A31003294FEA99
:10680800A3130CD9B7F84E10B1F5FA7F07D2484256
:10681800834203DB8B42A8BF0B4600E00346916B23
:1068280041F34F31B1F5807FA8BF4FF480716FF00D
:10683800FF008142ACBF5B181B18A2F87C3007B080
:10684800BDEC028BBDE8F08FB80E0020221A0020A4
:1068580094080108380F0020F0D8FFFFBA0E002076
:1068680080C1FFFFFEFFFF0F020000F02DE9F04F8F
:106878002DED0A8B87B00446049390F850300391AD
:1068880002921BB1322BA8BF322300E0012307EE8E
:10689800903AF8EEE7BADFEDD67AD64B9FEDD6CA36
:1068A8001B88D64AC7EEABBA002B08BF012307EEF8
:1068B800903AF8EEE79A1388009329EE8CCA03F011
:1068C80002077BEE8CBABBB2CCEE2BBA019333B382
:1068D800B2F90230B2F9042083EAE37182EAE27085
:1068E800A1EBE371A0EBE27088420546B8BF0D4604
:1068F800B5F5E17F16DA88429FEDC1BA05DD002AB9
:10690800D8BF524207EE902A04E0002BD8BF5B4262
:1069180007EE903AF8EEE77A87EE8BBA04E09FED3F
:10692800B9BA01E0B7EE00BADFF80CA39FEDB59A4B
:106938000AF108090AF1100B26460AF11C0500277E
:10694800F0EE49AAB04931F917300AEE103AB8EE1C
:10695800CAAAF5EE047A08392AEE27AA31F91730BF
:10696800BDEECAAA08EE103A009BF8EECA7A9FED6F
:10697800A7AA9A074FEA470827EE8AAAB8EEC88A54
:1069880075D078EE087A029BFDEEE77A594217EE49
:10699800900A884203DB8342A8BF034619469C48F5
:1069A800049B38F90000091A33F91700014407EE6F
:1069B800901AF8EEE78A04F095FB48B19549B2EED3
:1069C800049A88EE890AC85D04F08EF960EE098A97
:1069D800237FDFED916A0AEE903A237A07EE903A28
:1069E800F8EE677AF8EE6AAA68EEA77AB1EE047A4A
:1069F80067EEA67A2AEE877AFDEEE77A17EE901A06
:106A0800F1EE477AFDEEE7AA1AEE903A994208DBD2
:106A1800FDEEC7AA1AEE903A8B42A8BF0B460AEEC3
:106A2800903AD5ED007AE8EE8C7ABBEE0E7AF4EE69
:106A3800C77AF1EE10FAF8EEEAAA09D4B3EE0E7AA4
:106A4800F4EE477AF1EE10FAC8BFF0EE477A01E0AB
:106A5800F0EE477AC5ED007AA37C09EE103AB8EE5D
:106A6800499A67EE897A9FED6D9A27EE899A009B7D
:106A7800DB0750D4644938F901100029B8BF4942EE
:106A8800B1F5206F03DD0021CBF8001025E09FED64
:106A9800647A737868EE077A07EE103AB8EE477AA8
:106AA80087EE877ADBED007A37EE4A7AE7EE0C7AE2
:106AB8009FED5C7AF4EEC77AF1EE10FA09D49FEDF7
:106AC8005A7AF4EE477AF1EE10FAC8BFF0EE477A38
:106AD80001E0F0EE477ACBED007AF37ADBED008A3D
:106AE80000EE103AB8EE400A019B20EE280ADFEDCE
:106AF8004F8A60EE288A93B138EE6A8AF0EE6A7A95
:106B0800EBEE087A38EEC90AF0EE498AB0EE678AE9
:106B1800EBEE008A03E0F0EE498AB0EE6A8A374B62
:106B28009FED437A03F18801B0EE480A7A5C94F845
:106B3800511007EE902AF8EEE77A67EECA7AA7EEC8
:106B4800870A39B103F1140000EBC700D3ED0B0A33
:106B5800FEF7A0FDDAED007A2849D9ED006A059123
:106B68007AEE677A01F1A000C7EE8C7A3B5C0BF1F4
:106B7800040B0136043530EE280A77EEE67AAAECE3
:106B880001AAEBEEA76A07EE903AB8EEE77AE9ECCD
:106B9800016A67EE667A9FED277AA7EE870A08F002
:106BA8001FFB059901F1780E2EF8080088460FB9E9
:106BB8000127C7E6039AB1F9063095796D002835A3
:106BC8005D43B1F90E3000EE103ABAEECF0A08F084
:106BD80007FB6D11281A002D07EE900AB8BF6D4209
:106BE800322DF8EEE76A2BDD0023C8F8383050E084
:106BF80083F9223E54220020BD378635B80E002086
:106C08000000E14300000000C20E0020CDCC4C4043
:106C1800221A0020940801086F12033C0AD7A33DEA
:106C28000000A043000040C3000040430AD7233CB3
:106C3800A69B443BF7CC92385C0F002000803B4574
:106C4800FDEEE99A19EE903A23F0030307EE903A25
:106C5800F8EEE79A5FED077A637BC9EEA77A07EE4D
:106C6800103AB8EE477AD8F8383026EE877A67EEC9
:106C7800277AFDEEE77A17EE902A1344314A9342B9
:106C8800A8BF1346304A9342ACBFC8F83830C8F89A
:106C98003820D8F838305B13B3F5807FA8BF4FF49D
:106CA80080736FF0FF029342B8BF134607EE903A25
:106CB800B8EEE78AFDEEE67AE27817EE903A5343AB
:106CC8009B1100EE103A98F8A330032BB8EEC00AD7
:106CD80014D9B4F84E20B2F5FA7F0FD2FDEEC07A7F
:106CE800534217EE901A994204DB914217EE903AFC
:106CF800A8BF134607EE903AB8EEE70A94F8511089
:106D080059B14B0803D09942A8BF194600E00121A8
:106D18000E48D8ED0B0AFEF7BDFC30EE080ABDEEB2
:106D2800C00A8DED000ABDF9003000EE103AB8EE49
:106D3800C00A08F055FAA8F87C0007B0BDEC0A8B29
:106D4800BDE8F08FFEFFFF0F020000F0DC0E002010
:106D58002DE9F84FB0F90230934218BF00232DED0A
:106D6800028B18BF0370057804460E469146002D25
:106D780040F08B8007EE902A9FED770AF8EEE77ACD
:106D8800B6EE008A27EE800ADFED747A20EE270A35
:106D9800A04620EE080A08F069FADFED716A60EE95
:106DA800266AB7EE006AB0EE667AA0EE007A40F284
:106DB800DC536365D0EE006A1023A4F8523037EE36
:106DC800067A76EE866AC6EE077A1823A4F850305B
:106DD800274684ED046A27EE807A27EE007A77EE5C
:106DE800075A84ED017AC4ED025A70EE005A84ED18
:106DF800037AB8EE007AA5EE807A27EE877A67EEF6
:106E0800A67A84ED057AC4ED067ADFED567A98ED18
:106E1800047A27EE277AF0EE678AB5EEC07AF1EEAB
:106E280010FA4CBF77EE487A77EE087A013517EEFC
:106E3800900A05F0E5FCD8ED017A67EEA87AC7E973
:106E48000E01F5EEC07AF1EE10FA4CBF77EEC87A73
:106E580077EE887A08F1040817EE900A05F0D0FC5E
:106E6800032DC7E9080107F10807CED1A6F2DC53C4
:106E78001B042367E3676367C4F88030A367C4F81B
:106E880084300123A4F802902370D4F85490B4F904
:106E98005280636A276A206FE26FD4F840C0D4F842
:106EA8008010C4F88020C9EB060606FA08F64FEAF7
:106EB800E67B734307FB0B332667A7FB06671F4474
:106EC800636C656F60674FEAE27B53430CFB0B3ED4
:106ED800ACFB02237344B61A67EB0307E36AA26AA2
:106EE800C4F884104FEAE07B434302FB0B3EA2FB4D
:106EF80000237344B6185F41E36CA06CB4F95020CA
:106F0800A5674FEAE17B4B4300FB0B33A0FB010174
:106F18001944636B361A206B4FEAE57B05FB03F3D4
:106F280000FB0B3367EB0107A0FB0501194480192F
:106F3800794105F03BFC08F1FF3201239340E067FB
:106F4800C01841EBE371424605F030FCBDEC028B02
:106F58004844BDE8F88F00BF6F12833ADB0F494001
:106F6800F404B53F0000804B2DE9F8430024244B7E
:106F780093F8A360E0B2B0420ED203EB400203EBF9
:106F88008003B2F8C810D3F8E0301BB10B2801D841
:106F9800DB6898470134EAE71A4B1B685B032DD579
:106FA80000242346E2B2B24228D2DFF8549009F115
:106FB800E0074FEA840857F8242055689D4215D009
:106FC800284602F0D7FAEFF31283502282F3128890
:106FD80028216A6A01FB00900132C0F834216A69ED
:106FE80042F001026A61DBB283F3118857F8083076
:106FF8001B6800221A6001342B46D3E7BDE8F883EA
:10700800B80E00202422002008B50E4B1B6813F48C
:10701800805F0D4B14BFD3F8D821D3F8DC2193F847
:10702800A31092880023D8B2884204D2074820F8D7
:1070380013200133F7E7FFF797FF3220BDE8084038
:1070480000F093BC24220020B80E0020800F0020FE
:107058000A4B1A680A4B30B502F48052D3F8D8416B
:10706800D3F8DC5100230AB1A18800E0A9880548BB
:1070780020F8131001330C2BF5D130BD2422002049
:10708800B80E00200822002070B5124D00242146B9
:1070980005F2E110702285F8E04107F092FE2146E2
:1070A800D5F854320B4A0B4493F9020080B102F22E
:1070B800E1141E680E5108199C8884809B7983719D
:1070C80092F8E03107310133702982F8E031E7D1D5
:1070D80070BD00BFB80E0020094B1A680E2303FBD1
:1070E8000020437AFF2B07D0064A12789A4203D928
:1070F800054A32F8130000E0808800B2704700BFEC
:107108000012002048210020E00C002038B52A4C4D
:107118002DED048B94ED968ADFED289A38EE290A36
:107128000546FEF7FAFCF0EE408AB0EE480AFEF794
:10713800F4FC94ED979AB0EE408A39EE290AFEF7EE
:10714800ECFCF0EE409AB0EE490AFEF7E6FC95ED4D
:10715800017AD5ED027A95ED006A68EE676A27EE46
:10716800088AE7EE286A68EE000A67EE807AE6EE9B
:10717800290AB0EE660AE7EEA80A08F003F9DFED7F
:10718800107A20EE270ADFED0F7A80EE270AD4ED79
:10719800987A30EE270AF2EE047A80EE270A08F091
:1071A8001FF8BDEC048B83B21A0444BF00F5B47019
:1071B80083B218B238BD00BFB80E0020DB0FC93F3C
:1071C8000000E144DB0F494001380A4B042804D889
:1071D800DFE800F00507090B0D00074A08E0074A39
:1071E80006E0074A04E0074A02E0074A00E0074AC7
:1071F8001A607047F80000201DB40008A962000852
:1072080015B7000811B100083D6500087568000849
:107218004FF09043202208B19A6170471A85704751
:107228004FF09043202208B11A8570479A61704741
:10723800F8B504460E46174600252046202107F0DB
:10724800F6FD0446D0B10134204607F055FEB0F5EE
:10725800617F05DB40F634039842A8BF184601E079
:107268004FF46170A0F56170192390FBF3F00DB92C
:10727800307000E070703B7801333B700DB9012528
:10728800DBE72046F8BD7FB504780646E4B9364BFF
:107298001B6803EB8403192193F87B0093F87C6047
:1072A80093F8792093F87A304FF4617511FB005008
:1072B80011FB0651009001912C4821460134FEF73C
:1072C8001BFB142CE3D14CE007F016FE13280546EF
:1072D80041DC254B701C1C68202100238DF80F30E1
:1072E80007F0A5FD1E35064670B10136304607F099
:1072F80003FE1A289FBF04EB850358709DF80F30D2
:10730800013398BF8DF80F303046202107F08FFDEC
:10731800064670B10136304607F0EEFD0D289FBFD6
:1073280004EB850398709DF80F30013398BF8DF8F2
:107338000F3004EB85043046E11C0DF10F02FFF716
:1073480077FF9DF80F30042B0BD0601C002104221E
:1073580007F037FD05E00648064900221323FEF72B
:10736800CBFA04B070BD00BFFC110020CE2101088B
:10737800E321010802220108014804F007BE00BF0A
:1073880008220108F0B5047887B006461CBB524BAA
:107398001968062303FB0411192091F8CA5091F8C3
:1073A800CB7091F8CE2091F8C9304FF4617610FB7C
:1073B800056510FB07600095019091F8CC000290DC
:1073C800C83146484979039121460134FEF794FAB9
:1073D8000C2CDCD17DE007F08FFD0B28044672DC15
:1073E8003D4B701C1D68202100238DF8173007F0D5
:1073F8001EFD064680B10136304607F07DFD0328A4
:107408009FBF062303FB045383F8CE009DF8173073
:107418009CBF01338DF817303046202107F007FD57
:10742800074680B10137384607F066FD0D289FBF33
:10743800062303FB045383F8C9009DF817309CBF4B
:1074480001338DF8173006266643A9193846CA3124
:107458000DF11702FFF7ECFE202107F0E8FC0746C4
:1074680070B10137384607F047FD14289FBF9DF8D3
:1074780017307619013386F8CC0098BF8DF817308D
:107488003846202107F0D3FC78B1013007F034FDED
:107498000D289FBF062303FB045383F8CD009DF8F6
:1074A80017309CBF01338DF817309DF81730062B25
:1074B8000FD0062202FB04500021C93007F081FCDE
:1074C800FFF75AFF05E00648064900220B23FEF79E
:1074D80013FA07B0F0BD00BFFC1100201622010806
:1074E800E3210108022201082DE9F3470478064642
:1074F8004CB9204601A903F081FD0134FFF7F4FFE0
:10750800122CF6D17AE007F0F7FCC5B2112D6FD82E
:107518003C4C05F1D00704EB4703701C202193F87D
:107528000280394E07F083FC034630B9A8F1020205
:10753800D2F1000848EB020845E000F1010A597849
:10754800304607F074FC60B1032D8CBF0323002381
:10755800801B334453FA80F090F80490B9F1030F7C
:1075680002D1FFF709FF49E0A9F10203D3F10008AE
:1075780050464FF0200148EB030807F058FCD8B1FB
:10758800B8F1000FEDD0013007F0B6FC40F2ED2362
:1075980080B2984205DD40F6CA039842A8BF184653
:1075A80001E040F2EE2004EB4703A0F2EE2019229E
:1075B80090FBF2F0D87002E0B8F1000FD1D104EBE3
:1075C800470383F8029004EB4704A378F25CB8F110
:1075D800000F08D0E3780D48294640F2EE2419251B
:1075E80005FB034308E029460948FEF785F905E04D
:1075F8000848094900221123FEF77EF902B0BDE8C8
:10760800F08700BF541A00209808010836220108A4
:1076180048220108E32101085F2D010810B5084B35
:107628001968002201EBC20393F90240844201D198
:10763800981C10BD0132042AF4D1002010BD00BFEF
:107648001C110020F0B5027887B08AB94B4C04F1C0
:10765800200694F8F22100234949595650B2814234
:107668006CD00C33302BF7D10834B442F1D183E01D
:10767800002204920592451C07F03EFCC4B260B299
:10768800FFF7CCFF074618B18DF81040012400E041
:1076980004462846202107F0CAFB054638B10135C3
:1076A800284607F029FC0134ADF81200E4B20026A0
:1076B8002846202107F0BBFBA8B3451C284607F045
:1076C8001BFC00222F4951F822108142D3B203D06B
:1076D8000132082AF6D100232B4A02EB8302D26832
:1076E800824220D1022E0FD0032E12D05A1E012E14
:1076F800D2B204D0042A13D88DF814300EE0042A2C
:107708000ED88DF8153009E0052B09D88DF81730FB
:1077180004E09A1E052A03D88DF816300134E4B225
:107728000136042EC4D1052C03D807B0BDE8F040BB
:1077380022E604AB03CB386079601DE094F8F701CA
:10774800114B94F8F651B4F8F42103EB800003EBE5
:107758008505C068009094F8F90103EB8000C068C3
:10776800019094F8F80103EB80030848DB68029362
:10777800EB68FEF7C1F877E707B0F0BD541A0020B0
:1077880020110020A40801089808010857220108C0
:1077980030B50B4B1C6893F834101A4603290BD8E4
:1077A8000B4604EBC3034D1CE9B29D882842F5D073
:1077B80082F83410981C30BD82F83410002030BD97
:1077C8001C110020024B002283F83420E0E700BFA0
:1077D8001C1100202DE9F047877890F803C0214D4F
:1077E800BBB2C7F1640E03EB83065C42C3F17800B9
:1077F8005FFA8EFE7600CCF16408A4B280B2A3B220
:107808000FFA83F9B9F1000F05DC002B14BFBA4653
:107818004FF0010A00E0F24613FB03F303FB0CF2FE
:107828001AFB0AF392FBF3F3434403FB09F30A221E
:1078380093FBF2F333449BB225F8023FB1F8009072
:107848004A880A34C9EB020AA4B21AB202FB0AF245
:107858004FF47A73844292FBF3F34B442B80CED1DE
:10786800BDE8F0875011002010B544780078002258
:1078780002FB02F3193B634303F6C413534340F678
:10788800C411434393FBF1F3034921F81230013249
:10789800072AEDD110BD00BF6A1100200430114B3A
:1078A80033F91000B0F5617F10B506DB40F63303FD
:1078B80098420246A8BF1A4601E04FF461720C785C
:1078C800192340F2833013FB0404944207DA497801
:1078D80013FB01039342B4BF0020012010BD002018
:1078E80010BD00BFE00C00200A4B1B6813F4805F3A
:1078F800094BB3F9063005D0C089421A934207DD17
:10790800084400E0008A8342B4BF00200120704789
:107918000120704724220020E00C002010B50A4AFC
:107928000A4B11689B6800BF12689142F7D1084A58
:10793800D46D4FF47A7000FB04F2D31AB3FBF4F35E
:1079480000FB013010BD00BF4C1A002010E000E021
:107958001C11002038B50446FFF7E0FF0546FFF785
:10796800DDFF401BA042FAD338BD10B504462CB148
:107978004FF47A70FFF7EEFF013CF8E710BD2DE9F0
:10798800F04F87B0824602919DF8444011461A464E
:107998009DF8403000268A4D0C202F1D7043C75794
:1079A800574506D1284490F80CB0BBF1000F04D01D
:1079B80002E10136042EEED1FEE0BAF1010F00F02B
:1079C800E88006DCBAF1000F40F0F68000947D48AC
:1079D800E4E0BAF1020F00F0DF80BAF1140F40F0D2
:1079E800EB80DFF82482D8F8183043F00103C8F898
:1079F8001830D8F814304FF0904443F40033C8F8E6
:107A08001430012703224FF4805904A94FF0904005
:107A18008DF815200392CDF810908DF814708DF81C
:107A280016708DF817B0FDF7B1FCA4F82890C8209F
:107A3800FFF79BFFC4F81890D8F81430039A43F462
:107A48000033C8F8143020464FF4C0538DF8152081
:107A580004A9022204938DF8142003928DF816B01D
:107A68008DF817B0FDF792FC636A23F470436362E4
:107A7800636A43F460436362636A23F47023636256
:107A8800636A43F4602363624F4B4FF480211960AB
:107A980001F18041A1F53F311223C5F89030082348
:107AA80085F895300B6885F8967023F480230B6071
:107AB8004B6823F480234B6095F8943003F180439E
:107AC80003F58233196841F480211960D5F89010C4
:107AD8003E4B21F01F0401F01F01E05807FA01F1A5
:107AE80020EA0101E150D5F89010394821F01F042F
:107AF80001F01F0154F800E007FA01F12EEA010134
:107B08002150D5F8901021F01F0001F01F01C45832
:107B180007FA01F12143C1502E4B2F49C3F800B099
:107B2800D8F81C3043F40003C8F81C302B4B04A8C9
:107B3800D9608DF810A0039A8DF811208DF812B035
:107B48008DF8137003F086F82A238DF810309DF80D
:107B580013308DF811708DF812B01BB104A803F022
:107B680079F804E01E4B4FF48062C3F884201D4A64
:107B78001D4B136002221A721C4A1D4B13601D4ACA
:107B88001D491B68116098470D481C4B40F8603F21
:107B980007E000941A4801E01A48009401F038FE02
:107BA80050B1074B80F804A00C2202FB06369DF862
:107BB80008303373B06000E0002007B0BDE8F08FF4
:107BC8001C11002000380140140401400804014041
:107BD8000C040140D80042420005FA0500ED00E01F
:107BE80000E100E0101A002050210020041A0020B3
:107BF800AC000020001A002048000020C40801083A
:107C0800004400400048004000100240024A136847
:107C180001331360704700BF4C1A0020024BD3F8A1
:107C2800983003B1184770471C110020014B1B689E
:107C3800184700BFC422002010B50020FFF7F6FF48
:107C4800074B00241C7004F0ABF8064B83F89C40EB
:107C5800C3F8A040A3F8A440C3F8A84010BD00BFD3
:107C6800282200201C11002010B510B9BDE81040D2
:107C7800E2E700230C225A430C4C1119125D824290
:107C880003D00133102BF5D110BD094BD3F8A80050
:107C980018B14A784078824206D20022C3F8A81068
:107CA800A3F8A420C3F8A02010BD00BFC411010888
:107CB8001C11002010B540001428A8BF1420002370
:107CC800074A022199540B4499181424834201F855
:107CD800014CF5DBFF21D1540F20BDE81040C3E76C
:107CE8005622002038B5164B202240F2DB151A85A3
:107CF800684310229A61851E0B24013C14F0FF048E
:107D080017D00F4A938A9BB283F020039382938AF9
:107D18009BB283F0100393822846FFF726FE0120CA
:107D2800FFF784FF1920FFF720FE0020FFF77EFFF2
:107D3800E3E7044B044A1A60044B054ADA6038BD8D
:107D480000040048FC9F0020EFBEADDE00ED00E01F
:107D58000400FA0503681B69184703681B6818477D
:107D680038B500240B4D6059254404F00FF96968B3
:107D780011B10948FDF7C0FDA96811B10748FDF721
:107D8800BBFD0748103404F001F9B4F5C07FE9D110
:107D980038BD00BFDC080108482301084E2301084C
:107DA800112C010870B50546284607F04EF806461E
:107DB80058B91A4B1A485A791A4B03EB8203BDE893
:107DC8007040D3F87C11FDF797BD28461649324616
:107DD80007F044F860B91548154C04F0D7F854F882
:107DE800041F19B11348FDF787FDF8E7124805E0AD
:107DF8000024124B53F8241021B91148BDE87040F3
:107E080004F0C4B82846324607F028F801340028A0
:107E1800EFD1024B0B4D5C71C6E700BF541A00202E
:107E280054230108DC0801086023010865230108C0
:107E3800580A010878230108112C01085C0A010876
:107E48007C2301086C200108F0B585B0044606F0D3
:107E5800FCFF082826D1621EE01D1F4912F8013FC9
:107E680009681944497801F00301022908BF203B39
:107E780082421370F1D1254604F1080715F8016B09
:107E88001648314606F0D3FF20B12846314606F0A1
:107E9800CEFF10B1FFF770FA1CE0BD42EED12046CC
:107EA80003F08FF80E4804F071F800230D4A1A44C5
:107EB80004A992F88A210A440849595C02F80C1C62
:107EC8000133082BF2D1002307488DF80C3001A9A3
:107ED800FDF712FD05B0F0BD04010020BB2A010822
:107EE8008B230108541A0020532B01082DE9F04177
:107EF800054606F0AAFF2F4B04469E6888B92E480F
:107F080004F044F82D4B53F8241041B10123A34049
:107F1800334202D02A48FDF7EFFC0134F2E7294842
:107F280021E028462849224606F098FF58B92748F4
:107F3800274C04F02BF854F8041F0029EFD02048F0
:107F4800FDF7DAFCF7E72B782D2B03BF013504F199
:107F5800FF344FF001084FF000080026174B53F884
:107F6800267027B91B48BDE8F04104F00FB8284631
:107F78003946224606F072FFC8B90120B040020611
:107F880001D51548EFE78305FBD4B8F1000F03D0FE
:107F9800FDF7E6FE114802E0FDF7EAFE104803F09F
:107FA800F5FF39460F48BDE8F041FDF7A5BC01369D
:107FB800D4E700BF541A002091230108C40A01081D
:107FC80078230108112C0108602301089B2301086C
:107FD800C00A01087C230108A7230108B52301086A
:107FE800BE230108522B010810B5084803F0CEFF44
:107FF800074B00241C701C63064B1C70FFF728F805
:1080080004F050F9044B1C6010BD00BFC6230108E2
:10801800C8110020DC2200203822002070B5064656
:1080280000240B4BE518AA8816420AD0E1580948E3
:10803800FDF762FC2846002103F035FF064803F0EF
:10804800A5FF143440F618339C42EAD170BD00BF36
:1080580064130108F2230108112C0108F0B5047813
:108068008BB005460CB1002436E04B4B596B0E2300
:1080780003FB041101F58C70B1F91D51B1F91921F7
:10808800B1F91B31009591F82051019591F82151D2
:10809800029590F90700039001F590713F4891F916
:1080A8000210049121460134FDF726FC082CDCD18E
:1080B80070E02D2B14D1072C1BDC284606F01CFF82
:1080C8000AAB661C03EB440424F8100C15F8013FB6
:1080D800303B092BFAD934462B78002BE9D104E040
:1080E800A3F13002092A09D8E5E7082CBDF81820C1
:1080F80009D00BB0BDE8F040FFF73EB9202BF8D10E
:1081080001352646E7E7072AF3D8BDF81A00224BBF
:10811800A0F2EE2189B240F2DC55A9425B6BE8D8A7
:10812800BDF81C10A1F2EE24A4B2AC42E1D8BDF80F
:108138001E6004B237B2A742DBDB0DB2AF42D8DC17
:10814800A542D6DBBDF8247007F16404A4B2C82C9C
:10815800CFD8BDF826E00FFA8EF4112CC9DCBDF893
:108168002050B42DC5D8BDF82240B42CC1D812B2C5
:108178004FF00E0C0CFB0233A3F81901A3F81B11E6
:10818800A3F81D6183F8205183F8214183F81F71FA
:1081980083F822E10BB0F0BDC8110020FC230108D0
:1081A8002DE9F041047806467CB9334DB5F8C6216F
:1081B800B5F8C831314821460134FDF79DFB042C40
:1081C80005F10405F2D1BDE8F0812D4906F002FE63
:1081D800B0B9294B4FF47A714FF4FA62A3F8C6117B
:1081E800A3F8C821A3F8CA11A3F8CC21A3F8CE118B
:1081F800A3F8D021A3F8D211A3F8D421BDE8F081C7
:10820800304606F079FE032805462DD83046202151
:1082180006F00DFE044630B10134204606F06CFE2F
:108228000126074600E006462046202106F0FFFD0D
:1082380018B9BDE8F041FFF79FB8013006F05CFEC1
:10824800012EF6D1A7F2EE2240F2DC539A42F0D882
:10825800A0F2EE229A42ECD8074B703503EB850367
:10826800DF801881BDE8F081064807490022032312
:10827800BDE8F041FDF740BB541A00201C2401085A
:108288002F240108E32101085F2D01082DE9F041A1
:108298002DED048BAB498AB0044606F09BFDAA4934
:1082A800002820460CBF0126072606F093FDA749A3
:1082B8000028204608BF022606F08CFD002808BFCB
:1082C8000426F10740F1E480A148A24C03F05EFEC9
:1082D800002003F031FCA04803F058FE9F4803F04B
:1082E80055FE62799E4B9F4803EB82032546D3F8DF
:1082F8007C11FDF701FB9C48FDF7FEFA4FF00008E2
:10830800274695ED058AB5EE408AF1EE10FA04D1BC
:108318009648FDF7F1FA002570E09548D5ED069AE4
:1083280095ED079AD5ED088A4146FDF7E5FAB5EED1
:10833800C08AF1EE10FA02D5202003F01FFEB0EE3D
:10834800480A06A8FDF75AFA01468A48FDF7D4FA02
:10835800F5EEC09AF1EE10FA02D5202003F00EFED9
:10836800B0EE690A06A8FDF749FA01468148FDF70B
:10837800C3FAB5EEC09AF1EE10FA02D5202003F048
:10838800FDFDB0EE490A06A8FDF738FA014679481E
:10839800FDF7B2FAF5EEC08AF1EE10FA02D5202008
:1083A80003F0ECFDB0EE680A06A8FDF727FA08F11D
:1083B800010801467048FDF79FFAB8F10C0F05F166
:1083C80010059ED1A4E749B294F8D42094F8D5308A
:1083D800009194F8D710019194F9D810029194F96A
:1083E800D910039194F8DA100491644829460135AC
:1083F800FDF782FA102D04F1070403D094F8D61083
:108408000029E0D15E485F4C03F0C0FDD7F8088032
:1084180054F8041F19B15C48FDF76EFAF8E70D46E9
:108428005A4B53F8254054B10123AB4013EA080FC7
:1084380003D057482146FDF75FFA0135F0E7554864
:1084480003F0A4FD21467B180AAA93F88A31134445
:10845800514A8A5C03F8102C01310829F3D1002312
:1084680006A94E488DF82030FDF746FA4C4803F02F
:108478008DFD4C48FFF7E6F84B48FDF73DFA4020E4
:10848800FFF7CCFD494803F081FD4648FFF72CF87B
:10849800B20739D5464803F079FD464803F076FD22
:1084A800404803F087FB444803F070FD3D48FEF761
:1084B800EAFE424803F06AFD3A48FEF763FF404887
:1084C800FDF71AFA3748FFF76BFE3E4803F05EFDEA
:1084D8003448FFF7C3FD00270E257D4300243A4AA0
:1084E800926B2A440123D2F80A20A34013421ED1DA
:1084F80001340E2CF3D10137082FEDD12A48FDF7AE
:10850800FBF98020FFF78AFD730716D52F4803F083
:108518003DFD2F4803F03AFD224803F027FB22488F
:10852800FDF7EAF94FF48070FFF778FD05E039466A
:1085380022462848FDF7E0F9DAE70AB0BDEC048BDB
:10854800BDE8F081352401086C2801083C240108A5
:1085580042240108541A002050240108622401080A
:10856800DC0801086E240108792401088624010822
:108578009324010851230108532B0108AB24010857
:108588009B240108C00A0108CA240108C40A01087A
:10859800D8240108E5240108BB2A0108F1240108B0
:1085A800FA2401086C200108112C0108092501088A
:1085B8001625010829250108372501084125010844
:1085C800502501085E250108C81100206A25010808
:1085D8007B2501088D250108F0B504468FB020469B
:1085E80006F033FCC5B225BBAC48AD4C03F0CEFC5D
:1085F80094F8D61009B9AB4854E049B294F8D4209D
:1086080094F8D530009194F8D710019194F9D810C6
:10861800029194F9D910039194F8DA100491A248C0
:1086280029460135FDF768F9102D04F10704DFD15B
:10863800E1E720469D49052206F010FC0546B8B939
:1086480029469B48702206F0BCFB9A4B596B28467A
:108658000E2303FB001301300022082883F823218E
:1086680083F8242183F8252183F82621F0D113E10A
:1086780020469149042206F0F1FB05462046002DCC
:108688004AD1202106F0D3FB002800F00581461CC2
:10869800304606F0DAFB2C460746884B53F8245040
:1086A8002DB987480FB0BDE8F040FDF725B9304631
:1086B8002946FAB206F0D2FB01340028EDD1784AF7
:1086C80002F170011646002382F8DA3082F8D630BB
:1086D80082F8D53082F8D43007328A42F3D179490A
:1086E80001EBC40191F84022934210DAD1F84472A8
:1086F800C3EBC302B0183A4400F1D4011768C0F8BC
:10870800D4709088888092798A710133E7E7294686
:108718006D48FDF7F1F890E06C49072206F09EFBE2
:1087280005462046002D4AD1202106F080FB06464A
:1087380006F08BFBC4B274BB6548FDF7DDF8214633
:1087480064480134FDF7D8F80E2CF8D15548FDF7E8
:10875800D3F8002460482146FDF7CEF80025554A95
:108768005E48516B0E2202FB04120123D2F823212A
:108778005B49AB4013425B4B05F1010508BF194645
:10878800FDF7BAF80E2DEAD146480134FDF7B4F8E2
:10879800082CDFD180E03046534906F0B1FB2C4667
:1087A80000284CD0022C4FD006F0A6FB06AB4E4951
:1087B80043F82400002006F0A3FB0134F0E74A49FF
:1087C80006F09EFB002460B1082C38D006F094FB1C
:1087D80006AB454943F82400002006F091FB01341C
:1087E800F1E7082C2BD1069B0F2B28D8DDF81CE0CD
:1087F800BEF1070F23D8089F0D2F20D8099E06F138
:108808006402C82A1BD80A9DFF2D18D80B98642823
:1088180015D80C99642912D8884210DA0D9C032CBB
:108828000DD8324AC3EBC303134483F804E05F71E5
:108838009E71DD71187259729C722D4CCFE60FB083
:10884800BDE8F040FEF798BD069B072B20D8079996
:108858000D291DD80278722A0DD06E2A18D1154A12
:10886800526B0E2000FB032301228A40D3F8231108
:1088780021EA020209E00F4A526B0E2000FB032393
:1088880001228A40D3F823110A43C3F8232101E0C7
:10889800FEF772FD0D4CA2E60FB0F0BDAC25010845
:1088A800541A0020112C0108D72501082F2401088B
:1088B800281B0020C8110020F32501085C0A0108C4
:1088C8007C230108DC080108F8250108A425010813
:1088D80052230108042601086B2B01080926010808
:1088E800972E0108372F01080D260108241B0020A8
:1088F8006C2001082DE9FF4104780546002C39D188
:108908007348744D03F042FBD5ED057AF5EE407AD5
:10891800F1EE10FA00F0D98021466F48FCF7ECFF21
:1089280095ED050A6846FCF769FF01466B48FCF7B8
:10893800E3FF95ED060A6846FCF760FF01466748C5
:10894800FCF7DAFF95ED070A6846FCF757FF014682
:108958006248FCF7D1FF95ED080A6846FCF74EFF20
:10896800013401465E48FCF7C7FF0C2C05F11005E1
:10897800CAD1AAE05B49052206F070FA40B9554B06
:1089880003F1C0020021596110339342FAD19CE0EF
:1089980028465549042206F061FA04462846002C68
:1089A80040D1202106F043FA002800F08E80451CB3
:1089B800284606F04AFA07464C4B53F824601EB97D
:1089C8004B4803F0E3FA80E028463146FAB206F055
:1089D80045FA01340028EFD13E4B03F1C0029E4610
:1089E8000021596110339342FAD1424B03EBC40280
:1089F8009846D2F804C0BCF1000F04D131463E4875
:108A0800FCF77AFF57E0002718F834309F42F5DA70
:108A18003B010EEB030563440FCB143585E80F00CB
:108A28000137F1E706F068FA0B28064647DC2846C6
:108A3800202106F0FCF9054650B101352846FCF71F
:108A480053FE244B03EB061383ED050A012400E0D3
:108A580004462846202106F0EAF9054648B10135C2
:108A68002846FCF741FE1B4B03EB061383ED060A71
:108A780001342846202106F0DAF9054648B10135C7
:108A88002846FCF731FE134B03EB061383ED070A68
:108A980001342846202106F0CAF910B9FEF76CFC0B
:108AA80013E00130FCF720FE0A4B032C03EB0616FB
:108AB80086ED080AF2D11148FFF71CFF05E01048BF
:108AC800104901220C23FCF717FF04B0BDE8F08120
:108AD8000F260108541A00202A260108302601080A
:108AE800532B01082F240108F32501085C0A01080B
:108AF8007C23010878220108F82501086C20010868
:108B0800E32101080222010882B01B4B1B4A8DF8A1
:108B180007101968106860B31268052A29D1184A25
:108B2800106810BB9DF808109DF8073043EA012330
:108B380014490B80144B1968144B89B20B445B0021
:108B480019680121196013680B441360104A1368EF
:108B580023F4E04323F040039BB283F0300343F453
:108B6800004343F08003136003E01A68521A312A65
:108B7800D5D902B0704700BF4C1A0020C822002087
:108B8800B022002080610040505C00400A30002084
:108B9800045C0040014B1868C0B270476C2200208A
:108BA8000120704770477047F7B51C4B1A680AB91F
:108BB8001C6800E001241A490E780022D0B2A042B5
:108BC80002F1010207D202AD2F18164D3544285C78
:108BD80007F8040CF2E71A68121B1A600A781D6875
:108BE80022440A709DB903204021FCF703F90E4A7C
:108BF800136823F4804323F070039BB283F440533B
:108C080043F4004343F080031360054B1D70002CB0
:108C1800CBD09DF8040003B0F0BD00BF6C2200204B
:108C280004120020702200200C5C004013B50121C2
:108C38000DF1070204463A2001F0A6FF0520FEF7D1
:108C480089FE9DF8073003B10123237002B010BDDF
:108C580013B50446062143206A4601F095FFA0B1EA
:108C68009DF800209DF8013043EA022323809DF8F7
:108C780002209DF8033043EA022363809DF8042014
:108C88009DF8053043EA0223A38002B010BD13B556
:108C9800044606213B206A4601F076FFA0B19DF804
:108CA80000209DF8013043EA022323809DF802202A
:108CB8009DF8033043EA022363809DF804209DF861
:108CC800053043EA0223A38002B010BD0F4B5A7847
:108CD80013B51C46BAB90E4B1B68A3B11A681AB172
:108CE8000C49486902434A619A88ADF80420022277
:108CF8008DF807209868002201A98DF8062001F058
:108D0800A1F90123637002B010BD00BF0412002056
:108D1800E40200200010024008B5FFF7D7FF8021C9
:108D28006B2001F0D5FE6420FEF71FFE03216B20A7
:108D380001F0CEFE0F20FEF718FE0D4B1920197812
:108D480001F0C6FE0F20FEF710FE0A4B1A20197814
:108D580001F0BEFE18211B2001F0BAFE10211C20D4
:108D680001F0B6FE37200221BDE8084001F0B0BE90
:108D7800E90200200000002008B5FFF7A7FF074B15
:108D88001B7813B1012B03D008BD4FF4006201E03A
:108D98004FF48052024B1A8008BD00BFE802002041
:108DA800020000202DE9F0410369C76805460E4618
:108DB8001F40002F35D0B7FA87F24FF00043D34059
:108DC800DB432B611F40A2F11B03042BF1D8DFE822
:108DD80003F0221F1C190300746A24B1013C00230C
:108DE800A4B2736201E0EC6AA4B2D6F82080B8F1AC
:108DF800000FDED0D8F80030404621469847D8F812
:108E08000480F4E73068696B07E07068A96B04E0D8
:108E1800B068E96B01E0F068296C036889B298478B
:108E2800C7E7BDE8F0810F4B1A78692A16D15A882E
:108E3800B2F5DE6F12D11A79BE2A0FD193F8EE2659
:108E4800EF2A4FF000000BD113F8012B5040064ACF
:108E58009342F9D1B0FA80F040097047002070477A
:108E6800704700BF00F80308F0FE03082DE9F04F33
:108E78002DED028BE74C85B000214FF4DE622046D1
:108E880005F09FFFE44B04F509721A60E34B0025D7
:108E98001D70E34B04F2CA621A60692323704FF411
:108EA800807003236371FCF763FF4FF4167320226D
:108EB800A4F8663184F86A21FA236E22A4F868318E
:108EC80084F87C21BC230A22A4F8643184F87D212B
:108ED8004FF4FA732B22A4F86E3184F87F21012312
:108EE800212284F8623184F87E3184F8802184F864
:108EF80086312322002384F88121C4F818324FF4E4
:108F0800C872C4F81C32052384F8C856A4F87251F4
:108F1800A4F87051A4F8745184F8585184F8595140
:108F280084F85A51A4F85C51A4F85E51A4F8605131
:108F380084F8635184F86B5184F86C51A4F8845117
:108F4800A4F88221A4F8885184F8155284F81452A0
:108F580084F8205284F8233240F2DC53A4F8983184
:108F680040F24C43A4F89A3140F26C73A4F89C3157
:108F780040F27533A4F89E3140F6430384F8215239
:108F880084F8225284F8925184F89351A4F8A031BD
:108F980022462B462546032BCCBF0121002103F195
:108FA800010382F8A21114BF1E217521122B82F829
:108FB800A31102F10202EED14FF4FA63A5F8C83109
:108FC800A5F8CC31A5F8D031A5F8D43140F27E41CE
:108FD800052340F27E5E85F8E231A5F84411A5F834
:108FE8004CE1C82340F23A7140F2EA5EDFF8289279
:108FF800A5F8E631002601274FF47A7A1E201922B7
:109008004FF4C8734FF0320BA5F84611A5F84EE19E
:1090180040F2DC5140F2B45E85F8950185F8E32111
:10902800A5F8EA31A5F84A11A5F850E10390019294
:10903800029185F8946185F89661A5F8C6A1A5F80E
:10904800CAA1A5F8CEA1A5F8D2A185F8D66185F860
:10905800E06185F8E17185F8E47185F8E57185F8D6
:10906800E87185F8EC6185F8EE71A5F848A1A5F8D6
:1090780052B1A5F85431A5F856B101F053FFD9F80B
:10908800003003982F74EF73AE73AE81D8721873E3
:109098005520019AD8700F205871DA7122202122A8
:1090A80098715A740E2053224FF0170E1874DA76FE
:1090B80035200A224FF0280883F815E083F816E0D7
:1090C80098764FF02D0E5A209A740192642283F8F4
:1090D8000DE018721A771E7083F8018083F80280F9
:1090E800DE7583F804B09E731E76DE735E7683F8B1
:1090F800098083F814E04FF4FA7EA3F84EE04FF0AD
:10910800080E83F850E0DFF830E1C3F838E0C3F820
:109118003CE04FF0780CDFF824E183F80AC0C3F88C
:1091280028E0DFF81CC1DFF81CE1DFED3E8AC3F858
:109138002CC0C3F830C0C3F848E0F7EE087ADFF86F
:1091480008C102999F77B7EE008A4FF04B0E83F85B
:10915800526083F85180C3ED087AC3ED097A83ED34
:109168000D8AC3ED108AC3F844C083F84CE085F833
:10917800CA06A5F8D4164120042185F8CB0685F83F
:10918800CCB685F8CD6685F8D16685F8D26685F8BF
:10919800CE6685F8CF6685F8D066A3F85860A3F840
:1091A8005A60A3F8566083F85C10152183F868109C
:1091B8001D49D9661D4919671D495967C3F860C01B
:1091C80083F8648083F8658083F87870194801F023
:1091D800F8FED9F80010019A81F811614FF448732C
:1091E800A1F81631C82381F8126181F8138181F83A
:1091F800147181F8186185F8D931642385F8D8216C
:10920800A5F8DAA185F8DC61A5F8DE3118EE105A68
:109218000A461BE0541A0020FC11002000220020FE
:1092280004220020000000009A99193FF6287C3F8C
:109238003D0A773FA52A01088FC2F53C000060402F
:10924800CDCCCC3E000040400000A0400E2303FBE4
:1092580006136FF0170083F81901032083F81A0129
:109268006FF02F0083F81B01072083F81C016FF0B3
:10927800230083F81D01052083F81E01642382F86A
:109288001F3101365A2382F8203182F82131082E05
:109298004FF0FF0382F8223102F10E02D6D10023EB
:1092A80081F889314A4BC4ED058A10349C42FAD1C1
:1092B8000820484CDFF83081FCF75AFD1020FCF7F5
:1092C80057FD4023A4F80432052384F893314FF462
:1092D8007A73A4F844314FF4FA63A4F846314FF492
:1092E800FA43A4F85431D9F8003014220126002199
:1092F800032084F87C21A18184F892612674187077
:10930800242058709870D8F8003084F8D9110227B2
:1093180084F8D87182215A711A71642219709A716D
:109328002D4801F04EFE6561E56165622563656360
:10933800E5632564656465656566A5662567656793
:10934800C4F88050C4F88450C4F88850D9F8005044
:109358002249234A234BA161A162A263A264E16569
:10936800E166E267C4F88C20294604F56C704FF476
:10937800C6722362E362E3642365A3652366A36779
:10938800C4F8903005F012FD04F23C5029464FF421
:10939800C67205F00BFDD8F800301A68C4F8D62656
:1093A8005A68C4F8DA269A68C4F8DE261A68C4F837
:1093B800E2265A68C4F8E6269A68C4F8EA2684F8C9
:1093C800046484F8907505B0BDEC028BBDE8F08F9D
:1093D800141B0020541A0020AE2A0108240FD4BE02
:1093E800240FD43E000080BF042200201549D1F884
:1093F800883043F47003C1F88830134B1A6842F080
:1094080001021A605868114A02405A601A6822F02C
:10941800847222F480321A601A6822F480221A6058
:109428005A6822F4FE025A60DA6A22F00F02DA62FF
:10943800186B074A02401A6300229A604FF00063D3
:109448008B60704700ED00E0001002400CC07FF810
:10945800CCFC00FF07B52320FEF787FA7520012111
:109468000DF1070201F090FB28B19DF80700A0F16B
:1094780068035842584103B05DF804FB01480249AB
:1094880090E400BF004801406810002001480249EC
:1094980088E400BF00400140401000200148024914
:1094A80080E400BF00040040181000204FF0804006
:1094B800004977E4F00F00200148024972E400BF38
:1094C800002C0140C80F0020014802496AE400BF8F
:1094D800002C0140C80F0020224B10B5224C5A43E3
:1094E800224BB3FBF2F203880139013AA04289B258
:1094F80092B29BB20ED004F50064A0420AD0B0F13B
:10950800804F07D0A4F59834A04203D004F58064B6
:10951800A04202D123F070039BB2154CA04206D0A2
:1095280004F58064A0421CBF23F440739BB20380FF
:109538000D4BC162984202850FD003F50063984233
:109548000BD003F54063984207D003F58063984237
:1095580003D003F58063984201D1002303860123D9
:10956800436110BD40420F00002C014000A24A0494
:10957800001000400E4B800A984216D007D8B0F56C
:10958800801F0CD04A3B98420DD102207047094BEE
:10959800984206D00233984205D104207047012032
:1095A800704703207047FE2070470020704700BFB7
:1095B8004B00100050001000F8B50468064620461D
:1095C8000F461546FFF7D6FF04284BD8B27A910804
:1095D80047B902238B40D4F80CE0DB439BB203EA83
:1095E8000E03E3600A23204A03FB001342F82370AA
:1095F800043342F8235015463FB1B17AE26889082E
:1096080002238B409BB21343E360282202FB0052E3
:109618002032EFF31286502383F3128803B203EB50
:109628008303DB0003F10C011C3329442B4451F85C
:10963800047F17B117600A6804329942F7D10023F2
:109648001360F3B283F31188282303FB0050036AE5
:109658001BB1E36843F0010303E0E2684FF6FE73D1
:109668001340E360F8BD00BFC80F0020014800F0B8
:1096780077B800BF08120020014800F071B800BF99
:109688005C120020014800F06BB800BFB012002047
:10969800026BC168034610B5406942B11A6C8C1A56
:1096A800013A005D08BF0A46C0B21A6410BD1A6AC2
:1096B800805C01328A4228BF0022C0B21A6210BD03
:1096C800436B13B190F844007047836A406A1B1AD1
:1096D800584258417047036B13B15B68016C01E055
:1096E800C369016A8B423CBFC2689B18581AC0B252
:1096F8007047836A8169426B1944D160416A994213
:109708009DBF0169CB1A5360CB1A96BF00235360E3
:1097180083624FF0000380F84430136888BF816289
:1097280043F0010313607047436A8269D154436A66
:1097380002690133934228BF00234362436B1BB184
:109748001B68DB0705D4D4E7026D136843F0800378
:1097580013607047417100F013BB816000F010BBCB
:10976800026D036B70B50446D5699BB9A90611D57E
:10977800C36A1BB1908C80B298470BE0E169928C68
:1097880040694E1CD2B2E6614254E169E2689142F6
:1097980028BFE361616BA1B92A0612D5636AA26A80
:1097A8009A42236D09D0501CA669A062B25C1A8542
:1097B8002369984205D3A16203E01A6822F0800267
:1097C8001A602B0742BF236D08221A6270BD0D4B29
:1097D8000D484FF400525A600C4A11684FF6FE7358
:1097E8000B401360426B11684FF6FE730B40136019
:1097F800426A836A9A4200D07BE7012380F84430AA
:10980800704700BF00000240B01200204400024030
:109818002DE9F0471E46A14B8CB0984289469046E8
:109828009DF850507ED19E4B9E4A1A609E4A5A61BE
:1098380002F580729A614FF48072DA601A619B4A6D
:109848001A63143A5A63A2F54842203ADA64043299
:109858009A64C3F808801865954B9A6942F4804267
:109868009A615A6942F001025A6102238DF8083060
:10987800032315F0010A8DF809304FF000038DF825
:109888000A3014BF022301232C078DF80B3017D59B
:10989800884C402701978AF001038DF80A30236A23
:1098A80023F070632362236A43F0E0632362204657
:1098B80001A9FBF76BFDBAF1000F23D1A76121E0E5
:1098C800B0070ED50CA9402341F82C3D7948036A0E
:1098D80023F070630362036A43F0E0630362FBF7FB
:1098E80055FDF1070ED50CA9802341F82C3D714890
:1098F800036A23F070430362036A43F0E0430362A0
:10990800FBF744FD0E238DF8003000220123684642
:109918008DF801308DF802208DF80330604C01F08D
:1099280099F908E1644B984274D1644B5D4A1A6016
:109938004FF48072DA601A61614A5A6102F58072E6
:109948009A615B4AC3F808801865D36943F4003309
:10995800D36102238DF80830032315F0010A8DF82E
:1099680009304FF000038DF80A3014BF0223012399
:109978002A078DF80B3019D54FF09044042701972A
:109988008AF001038DF80A30236A23F47063236296
:10999800236A43F4E063236220460DEB0701FBF7DB
:1099A800F5FCBAF1000F25D1A76123E0B3070FD565
:1099B8000CA9042341F82C3D4FF09040036A23F48E
:1099C80070630362036A43F4E0630362FBF7DEFC3F
:1099D800F7070FD50CA9082341F82C3D4FF090400C
:1099E800036A23F470430362036A43F4E0430362A7
:1099F800FBF7CCFC26238DF80030002201236846B3
:109A08008DF801308DF802208DF803302B4C01F0D1
:109A180021F990E02B4B984240F006812A4B214ACD
:109A28001A604FF48072DA601A61284A5A6102F5A6
:109A380080729A611E4AC3F808801865D36943F496
:109A48008023D36102238DF80830032315F0010A1F
:109A58008DF809304FF000038DF80A3014BF022347
:109A680001232C078DF80B3032D5124C4FF4806748
:109A780001978AF001038DF80A30636A23F4706352
:109A88006362636A43F4E0636362204601A9FBF7FB
:109A98007DFCBAF1000F3FD1A7613DE000380140DD
:109AA800B01200206C110108041300205800024075
:109AB8000010024000040048004400405C120020EE
:109AC8000415002000480040081200200417002058
:109AD800B0070FD50CA94FF4806341F82C3D5448CA
:109AE800436A23F470634362436A43F4E063436266
:109AF800FBF74CFCF1070FD50CA94FF4006341F8B4
:109B08002C3D4B48436A23F470434362436A43F451
:109B1800E0434362FBF73AFC27238DF8003000222C
:109B2800012368468DF801308DF802208DF8033046
:109B380001F090F83F4CC4F82C900027012384F8DA
:109B480044302762E761A76267626671C4F80880DB
:109B5800A571204600F014F9F2072FD5206B30B319
:109B6800E36C01934FF480530A9380230693E368D0
:109B7800ADF8103020230993636902930397059782
:109B8800079708970B97FBF707FA01A9206BFBF7D4
:109B9800E5F9236B216D1A6842F001021A608A68A0
:109BA80042F040028A605B689BB2236406E0236D42
:109BB80020221A621A6842F020021A60B3072CD5D4
:109BC800606B28B3A36C01934FF480530A938023EE
:109BD80006932369ADF810300025102303930295EE
:109BE80005950795089509950B95FBF7D5F9606BD1
:109BF80001A9FBF7B3F9636B1A6842F002021A6015
:109C0800226D5D605D60936843F08003936004E0BB
:109C1800226D136843F080031360226D136843F0CC
:109C280001031360204600E000200CB0BDE8F08777
:109C3800000400480812002010F80A3C0133DBB287
:109C48000A2B84BF10F8131C044A00F80A3C82BF90
:109C5800002322F8113000F80A3C7047040D002058
:109C6800334A136C90681944081A40F68C239842BA
:109C780070B513469160D06051603BD9127893F962
:109C880045108A4210460BD1111F082908D893F8AD
:109C98004610182901D8013103E083F8442002E076
:109CA800002183F8461093F944402149A24219D172
:109CB80091F84740B4B10C310024944206DA1D4DA6
:109CC80051F8046F25F814600134F6E70C2805D024
:109CD8001849002421F810400130F7E716480178A8
:109CE8000131017083F84520002201211A7083F8A0
:109CF800471070BD92F84710C9B1A0F2EF2440F2A6
:109D0800DA518C4208D811780B2905D80B1D01317E
:109D1800117042F8230070BD002283F84720074BDA
:109D280003F13002002143F8041F9342FAD170BDB9
:109D380098010020040D00201C040020A40100202C
:109D4800024A136C013319441164704798010020CA
:109D5800024B53F820301B6819607047980F002099
:109D6800064B53F820301A681B89A1F57A715943BC
:109D78004FF47A7391FBF3F111607047980F00204C
:109D8800F0B5046D8668236823F0010323608379A6
:109D9800054613F0020F40790CBF4FF0000E4FF448
:109DA800005E13F0040F14BF4FF48067002710F013
:109DB800010F14BF042100218307206820F001004F
:109DC8002060626822F440524EEA02026260226811
:109DD80022F4B05323F00C0348BF41F008013B4381
:109DE8000B432360A36895B023F44073A3606846CF
:109DF800FBF75EF9284B9C4201D10C9B0EE0274BE8
:109E08009C4201D10D9B09E0254B9C4201D10E9B40
:109E180004E0244B9C420CBF0F9B109B2268A8793E
:109E2800170448BF5B00B3FBF6F206FB1233B3EB33
:109E3800560F236828BF01321E0441BF4FF6F07346
:109E4800C2F34201134041EA03026B7992B213F064
:109E5800020FA28100F0010114BF4FF4003200226A
:109E6800DC0748BF42F480322B6D11B159680A43B0
:109E780002E0596821EA02025A609A6801074CBF59
:109E880042F0080222F008029A601A6842F00102C1
:109E98001A6015B0F0BD00BF003801400044004012
:109EA80000480040004C00403D4B1B78012B30B56A
:109EB80014BF00240324B1B9036A23F00103036229
:109EC8008169036A21F0F30123F00A0341F00101DB
:109ED80042F001021A4341EA041181610262836976
:109EE80023F00C031BE004291DD1016A4FF6EF7320
:109EF8000B4003628169056A120121F473414FF630
:109F08005F7342F0100241F480712B4092B2134308
:109F180041EA043181610362836923F44063836108
:109F28008369836130BD0829016A1AD14FF6FF633E
:109F38000B400362C169036A9BB289B223F42063B0
:109F480043F4807321F0F30143EA022241F0010156
:109F580092B241EA0411C1610262C2694FF6F37319
:109F680019E04EF6FF730B400362C369056A40F6B9
:109F7800FF41194045F6FF732B4043F4805343EAF1
:109F8800023241F4807192B241EA0431C161026245
:109F9800C2694FF2FF331340C361C369C36130BD67
:109FA8009401002038B510F80E2C50F8043C0446F3
:109FB80052B9012200F80E2C20F80C1C997A186866
:109FC8000222BDE838406FE730F80C2C20F80A1C54
:109FD800891A89B220F8081C074A10F80F0C0025C6
:109FE80022F8101004F80E5C1868997A2A46FFF7D0
:109FF8005BFF04F8065C38BD040D0020044B53F8E1
:10A0080020301BB107289CBF1B681960704700BF30
:10A01800C0020020084A13689B050BD5074B002196
:10A028001970074908684FF6FE7303400B604FF438
:10A0380000735360704700BF00000240DD2200201B
:10A048003000024073B506460D46002401232A88D5
:10A05800A34013421AD0AA78009302F003038DF8A4
:10A068000430EB78022B03D0032B0CBF032301230E
:10A078008DF805303046C2F301136946C2F38102F8
:10A088008DF806308DF80720FBF780F90134102C85
:10A09800DCD102B070BD2DE9F743DFF8149299F8CE
:10A0A800004005468E464F461146006816469846BB
:10A0B8007246631C07F8043BFFF70EFA2B89ADF8CC
:10A0C800043001A9022368688DF806308DF807303E
:10A0D800FFF7B8FFAB7A2A682401274449460C2BBE
:10A0E80000F2B780DFE803F007B5B5B53EB5B5B502
:10A0F8006AB5B5B59300136ADFF8B8C123F0010358
:10A108001362136AD2F804E0906920F4803020F0DA
:10A118007300624540F0700012D00CF5006C624587
:10A128000ED00CF5406C62450AD00CF5806C624587
:10A1380006D00CF5806C624502D043F0030307E0BB
:10A1480023F00E032EF4407E43F003034EF4807E8A
:10A15800C2F804E09061C2F834801362936943F056
:10A16800080329E0136ADFF84CC123F010031362D7
:10A17800136AD2F804E0906920F0807020F4E64079
:10A18800624540F4E04006D00CF5006C624502D010
:10A1980043F0300307E023F0E0032EF4406E43F071
:10A1A80030034EF4806EC2F804E09061C2F8388043
:10A1B8001362936943F4006393614AE0136ADFF81A
:10A1C800F4C023F480731362106AD2F804E0D369F0
:10A1D800624523F0730343F0700306D00CF5006C5E
:10A1E800624502D040F4407007E020F460602EF42D
:10A1F800405E40F440704EF4805EC2F804E0D361E3
:10A20800C2F83C801062D36943F0080320E0136A67
:10A21800DFF8A0C023F480531362106AD2F804E078
:10A22800D369624523F4E64343F4E04340F44050E5
:10A2380003D00CF5006C624501D14EF4804EC2F893
:10A2480004E0D361C2F840801062D36943F400632C
:10A25800D3612B7B1BB1536C43F4004353641388C5
:10A268009BB243F001031380AB7A0C2B18D8DFE8BC
:10A2780003F0071717170B1717170F1717171300E0
:10A288000B1902F134000AE00B1902F1380006E05C
:10A298000B1902F13C0002E00B1902F14000586072
:10A2A8000C443846A681A26003B0BDE8F08300BF25
:10A2B80004190020002C0140054B98420CBF054AA8
:10A2C800054A138801339BB213800020704700BFF2
:10A2D800005400405022002052220020704708B548
:10A2E8000B4B002093F82C10FAF784FD094B1B68E0
:10A2F800187A082801BF084B4FF480521A801022A0
:10A3080008BF5A80A0F109035842584108BD00BF50
:10A31800AC000020101A0020F81900207047704780
:10A328007047FEE7FEE7FEE7704730B50024E3B26A
:10A3380093420DD2030F092B94BF3033373301F802
:10A34800143001EB4403002500015D700134EEE791
:10A3580030BD30B5002202F1805303F5B8539B009D
:10A3680042F400441D6840F60F7144F0800429400F
:10A3780001322143042A1960EDD1024B40F08000DC
:10A38800186030BD4C5C00402DE9F347884D894C7E
:10A398002B68894E9BB2A380A28831880A40970512
:10A3A80007D54FF6FF53854A2B6013780133DBB28C
:10A3B8001370A3880B40180440F100830023ADF804
:10A3C80002302B687B4F9AB21804A28040F1F682C3
:10A3D800BB8803F00F03BB71002B40F0C182784AA1
:10A3E80013689BB23B803B8803F030037B803B883B
:10A3F80003F440533B8011684BF6BF730B4083F462
:10A40800005383F0200343F4004343F080031360B8
:10A41800BB88D90621D4116848F60F730B406949E7
:10A4280013600B681A7A022A884601D0042A02D1DE
:10A43800FAF76CFC5AE2062A40F06B825A78052A31
:10A4480008D11A78520605D1D878FFF782FFBB6881
:10A458001B6A9847E3689B685AE213689BB2ADF899
:10A468000230BDF802301F0540F1D0811168554F08
:10A4780040F68F730B40544913600A68534B92B2ED
:10A4880013445B0088461A683B68187A092817D075
:10A4980092B2520002F1804202F5C042117819705E
:10A4A800517859709188C8B2090A41EA0021598047
:10A4B8001189C8B2090A41EA002199809289DA8093
:10A4C80001221A72DA8893F80190002A40F0DC80A1
:10A4D8001A7812F07F024AD1B9F1090F0FD1DA7850
:10A4E800012A00F2B8809978002940F0B480998850
:10A4F800002940F0B0809A72A3685B68A9E0B9F1BE
:10A50800050F10D193F90320002A01DA0823B9E0D6
:10A518009A78002AFAD19A88002AF7D19B7A002BD8
:10A5280000F0A280F2E7B9F1030F0ED1DA78012A20
:10A5380040F091809A88002A40F08D805A7A42F043
:10A5480020025A72A368DB6983E0B9F1010F40F079
:10A558008280DA78012A7ED19A88002A7BD15B7AB8
:10A56800980678D5FAF768FC00287DD073E0012AB0
:10A578002ED1B9F10B0F6ED1E26858799269D9786A
:10A5880090473B689A7A002A65D0002863D11A79E7
:10A59800002A60D19B78002B5DD1064B9B68DB6855
:10A5A8009847084B1B685A79DA72DA781A735BE0B5
:10A5B800445C0040F8190020B4220020DF2200206B
:10A5C800005C0040101A0020505C0040043000205D
:10A5D800022A40D1B9F1010FC4D0B9F1030F3AD121
:10A5E800587920F0800E4FEA8E0202F1804101F581
:10A5F800B84110F0800F096814BF01F0300101F470
:10A608004051BEF1030F26D8B3F802E0BEF1000FA7
:10A6180021D101B39B7AF3B102F1804202F5B8422D
:10A62800010613684BBF23F4E04323F4804323F06F
:10A63800400323F070034BBF9BB29BB283F010031F
:10A6480083F4805343F4004343F080031360A3680A
:10A658009B69984708E0E36848465B699847032880
:10A668000FD000287FF452AFD8F80020A14B92B247
:10A6780013445B001A6800221A60302363800623A3
:10A6880000E009233A6847E1B9F1060F12D11A78B8
:10A69800520678D19B78012B02D1E368DB6967E029
:10A6A800022B02D1E3681B6A62E0032B6BD1E368DB
:10A6B8005B6A5DE0B9F1000F38D15988002962D191
:10A6C8005A6822F47F42B2F5003F5CD11A7812F042
:10A6D8007F0204D19B88002B00F0D58153E0012A2A
:10A6E80008D1E26858799269904700284BD13B68B5
:10A6F8009B7A17E0022A46D15A7902F00F010BB271
:10A708009B0003F1804303F5B84312F0800F1B68E8
:10A7180014BF03F0300303F44053032933D812F075
:10A72800700F30D1002B40F0AE812CE0B9F1080F4A
:10A7380004D11B785B0600F0A88124E0B9F10A0F68
:10A7480021D11A7802F07F02012A1CD19A7AD2B15B
:10A758005988C1B95A6822F47F42B2F5803F12D1B4
:10A76800E268587992699047002800F090810AE0E1
:10A778004BB13A684FF00008A2F812809361404646
:10A78800984740460BE0E3683A681B695078984759
:10A79800032804D1584B1B6809221A72BDE03A6895
:10A7A800138A4FF6FF718B4201D10923B4E00228C6
:10A7B80000D00BB90823AFE092F9001000291FDA86
:10A7C800D18801910198834202D9019B138210E03C
:10A7D8008B420ED2E16891F82C00834201D200210D
:10A7E80005E093FBF0F100FB113313B90121434B52
:10A7F8001970E36893F82C309382FAF787FA8CE0A3
:10A80800032313724FF44053238086E0BDF80230CF
:10A818001BB2002BBFF6D5AD116840F68F730B4005
:10A828001360354A17683B7A022B904671D0042B87
:10A838006FD0032B01D0052B66D1BB693A8A8BB93F
:10A84800398A00293BD04FF4405323802C4B1A6897
:10A85800284B92B213445B001A6800221A60302316
:10A8680063802CE0002AEBD0B7F81490914528BFFC
:10A8780091461FFA89FA504698473B8ACAEB030368
:10A888003B827B8A53447B821D4B1A681D4B92B2D4
:10A8980013445B0009F101021B689BB203F10053EA
:10A8A80003F5405352105B004FF0000E9645C7D099
:10A8B80053F82E1020F81E100EF1010EF6E7BB8A91
:10A8C8008B42D8F8003001D8032201E011B10522EB
:10A8D8001A720BE006221A72094B1A68054B92B2DB
:10A8E80013445B001A68196030236380D8F800307D
:10A8F8001B7A0FE002300020101A0020DE22002010
:10A90800505C004004300020072B02D1E368DB686C
:10A9180098470823D8F800201372FFF7E0FC5E4B35
:10A928001A684BF6BF7313402288D704228848BFA1
:10A9380083F480539004628848BF83F40053D1069F
:10A94800628848BF83F01003920648BF83F0200353
:10A9580043F4004343F080034F4A9BB213602DE059
:10A968009A0002F1804202F5B842116889B2ADF846
:10A978000210BDF8021009B2002909DA106840F681
:10A988008F7101401160013B444A52F823309847C7
:10A99800BDF802301F067FF514ADA1798B0003F1D5
:10A9A800804303F5B84348F60F72186802401A60EE
:10A9B8003A4B03EB81039B69984702E5A2883388E9
:10A9C8001340590505D54FF6FF332B60344B5B68B0
:10A9D8009847A28831880A40920444BF4DF6FF7315
:10A9E8002B60A3882F4A0B40DB0452D54EF6FF7329
:10A9F8002B6000231374137C052B41D8DFE803F088
:10AA0800030D1418222D6369264D1BB900F04CFB69
:10AA1800062300E005232B743BE000F045FB0423EC
:10AA280023740123636134E002236374032328E061
:10AA3800637C013BDBB26374637C53BB194B042218
:10AA48001A7426E0184A13689BB243F01003136087
:10AA5800052323740A2363741BE0637C114A013BBA
:10AA6800DBB26374637C03F0FF0093B90E490C6892
:10AA78004FF6EF7323400B6006231374506108E010
:10AA88000623237405E0094B73E6094B71E6094B6D
:10AA98006FE602B0BDE8F087005C00408411010851
:10AAA800AC000020F8190020405C00406D48000808
:10AAB800254900080149000820B9034B1B680822F2
:10AAC8001A82704701487047101A00206C00002055
:10AAD80038B5294B05464FF4204298685A60846976
:10AAE800240404D51446013A002CF8D10FE042683A
:10AAF800224C1440224A224342604FF420425A60BA
:10AB08008469A4070AD41446013A002CF8D15A6083
:10AB1800FFF7D2FB003018BF012038BD4FF42042A8
:10AB280085625A608469250604D41446013A002CCB
:10AB3800F8D1ECE74268114C1440124A22434260B3
:10AB48004FF420425A608469A40704D41446013A99
:10AB5800002CF8D1DBE74FF4204281625A6081690A
:10AB6800890604D41146013A0029F8D1CFE75A6082
:10AB78002023C361012038BD101A0020009800FC72
:10AB8800D0200101D00001022F4B70B505464FF4CB
:10AB9800204498685C608669360404D52646013CE2
:10ABA800002EF8D111E04668284C344044F4903423
:10ABB80044F0D00444604FF420445C608669B607D2
:10ABC80016D42646013C002EF8D15C600AE098684D
:10ABD8005C6022468169890631D41146013A002910
:10ABE800F8D15A60FFF768FB003018BF012070BD2C
:10ABF8004FF4204485625C6085696E0604D425465E
:10AC0800013C002DF8D1E0E75C60104D4468254018
:10AC18000F4C2C4344EA014444604FF4204400297B
:10AC2800D5D0986885696D0703D414F1FF34F9D23B
:10AC3800CBE7406A02F8010B0139C9B2EDE75A6067
:10AC48002023C361012070BD101A0020009800FC69
:10AC5800D02400020C4B0D49DA684378D243C2F382
:10AC68000222C2F10402934002781B010A44DBB2BB
:10AC780082F8003303780122580903F01F0302FA0F
:10AC880003F341F82030704700ED00E000E100E0F8
:10AC980073B50546002100680122FEF71DFC2A68ED
:10ACA80013889BB243F001031380EB7A8DF80430CC
:10ACB8000124002601A88DF805408DF806608DF85E
:10ACC8000740FFF7C7FFEB7A1B2B0BD1192301A80D
:10ACD8008DF804308DF805408DF806608DF8074032
:10ACE800FFF7B8FF02B070BD864B1A7B013A012A04
:10ACF80030B500F20681597B814240F002819A7B8F
:10AD0800022A00F0FE80804A1C7C505CD8734900FF
:10AD1800B2EE047A1CB15A18B2F9122009E05A1896
:10AD2800D3ED067AB2F91220F1EE677AC3ED067A0E
:10AD3800524207EE902AD3ED076A724AF8EEE77A94
:10AD4800F5EE406AF1EE10FAC7EE877A49D1D2EDF6
:10AD5800086AF4EEE67AF1EE10FA04DD9069C2EDC5
:10AD6800087A5062B9E0F5EEC06AF1EE10FA40F3E5
:10AD7800B48092F8285045B1022D00F2AE80D06B15
:10AD8800C2ED077AFA301064A7E0D2ED066A77EED2
:10AD9800E67AF7EE006AF4EEE67AF1EE10FAD2ED12
:10ADA8000C7A0DDBDFED596A67EEA66ADFED587A9B
:10ADB800F4EEE76AF1EE10FA58BFF0EE667A03E0B7
:10ADC800DFED546A67EEA67AC2ED0C7A012283F8A9
:10ADD80028209A6B024484F001040020D0721C746D
:10ADE80078E0F4EEE67AF1EE10FA48BFC2ED077AA1
:10ADF8001C6CDA6B93ED086AD3ED075A121B002A14
:10AE080076EE656A0BDAB7EE005AF4EEC56AF1EE33
:10AE180010FA62DDF4EEE57AF1EE10FA5DDDD3EDBD
:10AE2800097A384AB4EEE76AF1EE10FA0CDDD2ED91
:10AE38000B7ADFED366A67EEA67ADFED366AC2ED89
:10AE48000B7AD2ED0D7A0AE0F0EE007AF4EEE76ABA
:10AE5800F1EE10FA08DDD2ED0D7ADFED2C6A67EE1F
:10AE6800A67AC2ED0D7A07E0D2ED0B7ADFED296AFA
:10AE780067EEA67AC2ED0B7AD3ED0B7A9A6B214C6A
:10AE880067EE877A0244FCEEE77A17EE900A507074
:10AE9800D3ED0D7AFCEEE77A17EE900A507593F829
:10AEA8002800022801BFD4ED0C7ADFED1B6A67EE9B
:10AEB800A67A002003BFFCEEE77A84F8280017EE94
:10AEC800900A02220CBFD07284F828201A7C82F0E3
:10AED80001021A740022DA611A62187C094A08B160
:10AEE8000E4800E00E4890611944D3ED067AB1F996
:10AEF800122000EE102AB8EEC00A80EE070A37EEDC
:10AF0800C00A30BD101A0020C0110108EC51783F6A
:10AF18006F12833A0AD7833F00007A440000A041A9
:10AF28000000A0C108B522221148002103F049FF02
:10AF3800104B002210490420515C83F8F2110132B1
:10AF4800052183F8F701042A4FF0000083F8F61171
:10AF580083F8F90183F8F81103F10803EAD1074BE4
:10AF68000122A3F83822522283F8342208BD00BFF8
:10AF7800441C0020541A0020B72A0108101A002087
:10AF880000F1500302781AB98178C278914204D34B
:10AF980004309842F6D1002070470120704710B560
:10AFA800FAF772F84FF43024012806D11CB1FAF7E9
:10AFB8006BF8013CF8E7052010BD002C08BF052000
:10AFC80010BD70B50646441E14F8011F89B1094D1D
:10AFD800284603F02CFF0028F6D005F10803984214
:10AFE8003FBF054B401BC018A31B38BF80F8CE31AC
:10AFF800EAE770BDBB2A0108101A0020031EB8BF7B
:10B008002D2210B5B8BF58420C46B8BF01F8012B25
:10B018000A22FAF75DFC00230370204610BD07B52D
:10B028001B4B03F5E762C3F8342793F8D6215AB1CE
:10B03800012A14D1032183F83A17072183F83C2702
:10B0480083F83B170C2208E0022183F83A17032102
:10B0580083F83C2783F83B17072283F838270D4BE2
:10B068000D4A9A604020FCF7ADFB70B10122002325
:10B0780090F9000040218DE80C00084A4FF4E133B4
:10B08800FCF77DFC003018BF012003B05DF804FB1D
:10B09800101A00206C000020014A0008814B0008AB
:10B0A8000120002100F0CCBE0B4B10B519684FF6FB
:10B0B800FB720A401A60094A92F84A271C46084B54
:10B0C8000AB1052200E001221A60FEF78FF94FF459
:10B0D8003643236010BD00BF405C0040101A0020BA
:10B0E800C8220020064B1B7803F0040303F0FF007E
:10B0F8001BB1044B1888C0F3C01000F00100704762
:10B10800E0220020B80E00202DE9F04F2DED028B33
:10B1180085B083460293AC4B01911C88009204F0E1
:10B128000204A4B294B1A94BB3F90240B3F90030B8
:10B13800002CB8BF6442002BB8BF5B429C42B8BF2A
:10B148001C46B4F5007FA8BF4FF40074D94600250B
:10B158009E4B9F4833F915109E4B50F8256033F9E4
:10B16800153083EAE37EAEEBE37EBEF5206F4FEA4F
:10B1780045084FEA41074FEA850A12DC4FF0040EF2
:10B1880093FBFEF3FB1A1E44B6F57A5FA8BF4FF493
:10B198007A56914B9E42ACBF40F8256040F8253066
:10B1A80002E0002340F8253050F80A6099F80B3087
:10B1B800F6115E4399F801305F43834B1B889B0768
:10B1C8004FEAA6164FEAA71751D0009B49005B42E9
:10B1D800994203DB009B8B42A8BF0B467F4938F995
:10B1E8000110591A029B33F91530CB1808EE103AA2
:10B1F800FFF778FF68B1B8EEC80A794BB2EE048A57
:10B2080080EE080A585DFFF76FFD20EE080ABDEED4
:10B21800C08A744874495AF8003018EE102A42F26D
:10B22800107E13447345A8BF73468B42B8BF0B46C4
:10B238004AF800309BF808109BF81C00514300EBBB
:10B248008000C911C0F1000E714503DB8142A8BF1F
:10B2580001468E469BF812104B431B13F61ACEEB91
:10B2680007076643674303EB66260EEB6727594BD0
:10B27800042138F9030090FBF1F15C48405D41433B
:10B28800A7EBA1129BF8511008EE102A69B1584893
:10B29800584F0393B8EEC80A00EBC500D7ED000A73
:10B2A800FAF7F8F9039BBDEEC08A534933F8083022
:10B2B80038F9010028F801300FFA83FEC0EB0E0EB2
:10B2C80004209EFBF0F001F1040E0C315AF80E70C8
:10B2D8005AF801304AF801703B449BF850104AF87C
:10B2E8000E00034400EE103A59B1424B4348D3EDE7
:10B2F800000AB8EEC00A00EBC500FAF7CBF9BDEEBC
:10B30800C00A3F4A10EE103A575D3E4A18EE101A2E
:10B318007B433144A1EB631628F8026009F1010967
:10B328000DB9012514E7294B2948B3F90410019BED
:10B3380084689B790F335B004B4326495B11B1F955
:10B3480004509BF80D10002BA3EB0505B8BF5B421A
:10B35800322B0BDC01FB05442B492C4BA142A8BF27
:10B3680021469942ACBF8160836001E0002383607D
:10B378009BF8031001FB05F32549097803294FEAD7
:10B38800A3130CD9BBF84E10B1F5FA7F07D24C4283
:10B39800A34203DB8B42A8BF0B4600E0234681682B
:10B3A80041F34F31B1F5807FA8BF4FF480716FF042
:10B3B800FF008142ACBF5B181B18938005B0BDEC41
:10B3C800028BBDE8F08F00BFB80E0020BA0E002037
:10B3D800E80E0020C20E002080C1FFFF221A0020C4
:10B3E80094080108380F0020F0D8FFFF400F002014
:10B3F800CC0E0020E40E00206C210020180F002045
:10B40800580F0020300F0020FEFFFF0F020000F051
:10B418005B0F00202DE9F04F2DED028B85B0002544
:10B428000393A94B0292B3F90270B3F9003000906C
:10B43800002FB8BF7F42002BB8BF5B429F42B8BF06
:10B448001F46B7F5FA7F8146A8BF4FF4FA77A8469A
:10B458000195AA462C469D4E338813F0030F4FEAF8
:10B46800440B54D0022C52D0974B33F90B20029B3B
:10B4780052005B429A4203DB029B9342A8BF1346E9
:10B48800934A32F90B209B1A039A32F91420134479
:10B4980008EE103AFFF726FE68B1B8EEC80A8D4BE1
:10B4A800B2EE048A80EE080A185DFFF71DFC20EE54
:10B4B800080ABDEEC08A18EE102A99F8083099F8E3
:10B4C8001C105343642293FBF2F36FF0040202FB57
:10B4D80001FA534505DB01EB81029342A8BF1346ED
:10B4E8009A467D4818EE103A50F824100B4442F260
:10B4F80010718B42A8BF0B4678498B42B8BF0B46E8
:10B5080099F8121040F824304B431B1301933388E9
:10B5180003F00301012901D1022C41D1704D6A4980
:10B5280035F90B50009A6F4831F90B80567850F86E
:10B53800242085EAE57CACEBE57CBCF5206F4FEA7E
:10B54800840120DC022C17D008EB8800000190FB56
:10B55800F6F6042095FBF0F5761B02EB060EBEF519
:10B568007A5F6048604DA8BF4FF47A5EAE45ACBFC5
:10B5780041F800E00D5008E088EAE87CACEBE87C94
:10B58800BCF1640FE0DD002545505648009A095883
:10B598007D2591FBF5F5D17A6943402591FBF5F5B9
:10B5A8009A0713D5022C11D0019AC7F5FA7307FB35
:10B5B80005F607FB08F103FB0A114FF4FA7003FBC9
:10B5C800026391FBF0F193FBF0F608E0DB0704D58A
:10B5D800022C02D0019E514601E02E464146404BC6
:10B5E800042033F9143093FBF0F34048205C4343C4
:10B5F8006FF04F0093FBF0F3CB1899F851104FEA16
:10B60800440B08EE103AB1B1022CB8EEC80A384B18
:10B6180008D1480803D08142A8BF014600E00121B3
:10B62800344802E0344800EBC400D3ED000AFAF7CE
:10B6380031F8BDEEC08A2A4B30493BF803E03BF9AC
:10B6480001002BF801E00FFA8EF301F1080E143116
:10B658001B1A5EF82420042093FBF0F051F82430E4
:10B6680041F82420134499F850104EF8240003445C
:10B6780000EE103A59B11E4B2148D3ED000AB8EE3E
:10B68800C00A00EBC400FAF705F8BDEEC00A18EED0
:10B69800103A1C493344095D1E4610EE103A4B43DC
:10B6A800202193FBF1F3F61A174B2BF80360009B4C
:10B6B80001340133032C00937FF4CDAE05B0BDEC0B
:10B6C800028BBDE8F08F00BFBA0E0020B80E002034
:10B6D800221A002094080108380F0020F0D8FFFF34
:10B6E800C20E0020E80E002080C1FFFF400F00209E
:10B6F800E40E0020DC0E0020CC0E0020802100206B
:10B70800180F0020580F0020300F00202DE9F04FAF
:10B7180099462DED088BD54B09EE902A1A8883B0EF
:10B7280012F0020F04460193B7EE009A4CD0149B16
:10B73800CF48DD89B0F900305B1B03F2F31640F205
:10B74800E632964203D8002BB8BF5B4201E04FF4C3
:10B75800FA73B0F90220521B02F2F31540F2E630F8
:10B76800854203D8002AB8BF524201E04FF4FA726A
:10B7780094F84C0058B39342B8BF1346C3F5FA7314
:10B7880007EE903A9FEDBB7AF8EEE77A6423C7EEAE
:10B79800877A93FBF0F307EE103A77EEC97AB8EEA2
:10B7A800C77AF0EE498AE7EE878AF7EE006AF5EE87
:10B7B800C08AF1EE10FA0AD4F4EE668AF1EE10FAB5
:10B7C800C8BFF0EE668A04E0F0EE498A01E0DFEDDA
:10B7D800AA8ACF1C25464FF0000ABAF1020F17F8C3
:10B7E80001BFDFF8DC824FEA4A06B2EE04AA0ED1A6
:10B7F800B8F904209FEDA17A0BF10A0B02FB0BF3B9
:10B8080007EE903AF8EEE77AC7EE877A5FE038F904
:10B818001A30DFED986A07EE103AF8EEC77AB8EEFC
:10B82800697A19EE903A87EE267A5B4227EE877A94
:10B8380007EE903AF8EEE77AB4EEE77AF1EE10FA0E
:10B8480008D4F8EEE97AB4EEE77AF1EE10FAD8BF48
:10B85800F0EE477A8A4B9B5F08EE103A39F91A30B6
:10B86800B8EEC88A77EEC87A08EE103AB8EEC88AF9
:10B8780037EE888A88EE0A8AFFF734FC40B1814B9C
:10B8880013F80A00B0EE480AFFF72EFAB0EE408A25
:10B89800019B1A88D10704D5D4ED117A68EE277A6E
:10B8A80015E038F906309FED757A0BF1140B03FBA0
:10B8B8000BF307EE903AF8EEE77A9307C7EE877A2C
:10B8C80042BF94ED127A28EE078AE8EE287A6E4B8A
:10B8D800DFF8F0B19B5FD5ED08AA94F85110DFF8B6
:10B8E800E88107EE103A694BB8EEC77AD3ED116AD2
:10B8F8001AF80B30E7EE667AB0EE678A67EEAA7A36
:10B908000AEE903AF8EEEAAA67EEAAAADFED607AA4
:10B91800CAEEA7AAB0EE67BAC1B1BAF1020F0AD14E
:10B928004A0803D09142A8BF114600E00121B0EEB9
:10B938006A0A584804E05848B0EE6A0A00EBCA00A0
:10B94800D8ED000AF9F7A6FEF0EE40AAD8ED000AF5
:10B95800524995ED0B7A4FEA8A0268EE207A114433
:10B9680067EE877A91ED000AA7EE8A0ADFED4C7A36
:10B97800B4EEE70AF1EE10FAB0EE40AA09D4DFED12
:10B98800497AB4EE670AF1EE10FAC8BFB0EE67AABA
:10B9980001E0B0EE67AAC9EE207A434B81ED00AA18
:10B9A800991891ED007A81ED008A38EE477A03F113
:10B9B8000C011144183327EE277A1A44D1ED007A86
:10B9C80092ED000A81ED007AC2ED007A37EE800A26
:10B9D80094F8501030EE070A21B1344800EBCA0041
:10B9E800F9F758FEB0EE087A80EE070A1BF80A301D
:10B9F800D5ED0E7A20EE277A07EE903AF8EEE77A40
:10BA080067EE277A9FED2A7AC7EE8B7AF4EEC77A2B
:10BA1800F1EE10FA09D49FED277AF4EE477AF1EEA9
:10BA280010FAC8BFF0EE477A01E0F0EE477A3AEE36
:10BA38008A0A0AF1010A30EE270A03F0D1FB1E4BED
:10BA4800B0F57A7FA8BF4FF47A709842B8BF18460D
:10BA58001A4BBAF1030F985305F104057FF4BDAEF4
:10BA680003B0BDEC088BBDE8F08F00BFB80E002016
:10BA7800E00C00200000FA430000000000004842EB
:10BA8800221A002094080108C20E00206C21002010
:10BA98000000C842DC0E0020CC0E00206C0F0020F5
:10BAA80000007AC300007A43B4210020180F002058
:10BAB800000096C30000964318FCFFFF300F0020DB
:10BAC800BA0E0020C80E0020E40E0020044B00220D
:10BAD8001A605A60034B00221A605A60704700BF10
:10BAE800380F0020780F002010B50D4C012384F882
:10BAF8006F304FF48060022384F88C30FAF720F915
:10BB0800D4F89020074B51781B68642212FB01334C
:10BB1800C4F88030B4F86C300133A4F86C3010BD30
:10BB28006C2100204C1A0020014B33F8110070479B
:10BB3800040D00200020704707B5064B0093064B04
:10BB480001930649064A074B0748F9F7D5FE03B0A3
:10BB58005DF804FBB1200108BA200108F02A0108A9
:10BB6800FB2A0108A5200108D02A010808B5037896
:10BB780033B90C4B0C481978BDE80840F9F7BCBE3E
:10BB880003F0BAF902280BD8064B084A18700C21A2
:10BB980001FB002002305860FAF7BAF90448E6E7DA
:10BBA80008BD00BF00220020022B01081C21002034
:10BBB8006C20010808B503783BB90B4B0B4893F888
:10BBC800C816BDE80840F9F797BE03F095F90228B2
:10BBD80008D8054B83F8C806FAF7FCF8FAF7BCF959
:10BBE8000348E8E708BD00BF541A0020062B0108E7
:10BBF8006C20010838B5037803BB214B1B6801335F
:10BC08000F2B07D81F490C2202FB03121C4695680C
:10BC18002DBB00E01C4601340F2C01DD002400E0A0
:10BC280005D818490C2202FB04129568BDB99C423C
:10BC3800F1D11548BDE83840F9F75EBE03F05CF96C
:10BC48000F28044605D80F4A0C2303FB00239D68E0
:10BC58002DB921460D48BDE83840F9F74DBE084BCF
:10BC68001C60FBF7E9FF21462A460948F9F744FE1C
:10BC78000C235C43034B185DBDE83840FBF7F4BF69
:10BC880078000020C4110108132B0108292B010892
:10BC9800412B010873B5037813B9FBF76DFB3FE03F
:10BCA80001AA204903F089F90024024626462546C0
:10BCB8009AB134B1012C08D1104603F01DF906469B
:10BCC80003E0104603F018F9054601AA00201549BB
:10BCD80003F073F901340246EAE70B2D03D9124841
:10BCE80012490C230CE0022C11D1A6F57A73B3F596
:10BCF8007A7F08D90C480E494FF47A724FF4FA63E8
:10BD0800F9F7FAFD0CE00B4B03EB45031E81094BD9
:10BD1800094803EB45032946B3F90820F9F7ECFD78
:10BD280002B070BD0D260108E321010802220108B6
:10BD3800C627010800220020582B0108104910B519
:10BD48000B6A03EB4002147E14B1022C0FD00AE0F8
:10BD5800022804D9032806D14A6AD20401D5D88911
:10BD680010BD988A10BD074B33F8100010BD507EE7
:10BD780000EB800000EB800000F2EE2080B210BDE6
:10BD880000220020E00C0020044B5B6A42F2010212
:10BD98001A420CBF01200020704700BF002200207B
:10BDA8000F4B93F82820012A10B51C460DD008D354
:10BDB800022A0DD10B4A938A9BB283F01003938217
:10BDC80006E0084B10229A6102E0064B10221A8501
:10BDD800FBF7A4FD00F5F42000F59070E06210BDBB
:10BDE8000022002000040048034B1A6BD379591C29
:10BDF8001344D171187A70470022002010B5FFF75C
:10BE0800F3FF84B2FFF7F0FF04EB002080B210BD0F
:10BE180010B5FFF7F3FF0446FFF7F0FF04EB00400F
:10BE280010BD38B5054D04462146686BFBF795FFF4
:10BE38002B6B98796040987138BD00BF00220020B4
:10BE480038B5044624200D46FFF7EBFF4D20FFF7D9
:10BE5800E8FF002C084C14BF21203E20FFF7E1FF2B
:10BE6800236B002228469A71FFF7DBFF236B93F8B8
:10BE78004900BDE83840D4E70022002001460020F0
:10BE8800DEE710B50446C0B2FFF7CBFF200ABDE8D5
:10BE98001040C6E710B5044680B2FFF7F2FF200C49
:10BEA800BDE81040EDE737B5828883680446100680
:10BEB8000D4641BF2B4991F8C8164FF4C67000FBD8
:10BEC8000133D10544BF2849097802F03F0244BF35
:10BED80001EB410103EB8103042A12D006D8012AA1
:10BEE8000DD0022A32D193F9001030E0102A0AD07E
:10BEF800202A0AD0082A29D1B3F9001027E0197896
:10BF080025E0198823E0196821E093ED000A6846C6
:10BF1800F9F774FC01461548F9F7EEFC05B3D4EDC2
:10BF2800037A6846B8EEE70AF9F768FC0146104854
:10BF3800F9F7E2FC94ED040A6846B8EEC00AF9F78E
:10BF48005DFC01460A48F9F7D7FC09E000210948D9
:10BF5800F9F7D2FC25B10848E1682269F9F7CCFC69
:10BF680003B030BD541A00200022002051230108DC
:10BF78004A2301086B2B0108672B0108024B014675
:10BF8800986BFBF7EABE00BF0022002010B5441EE4
:10BF980014F8011F21B1034B986BFBF7DEFEF7E79E
:10BFA80010BD00BF002200202DE9F3412B4C2C4B83
:10BFB80094F83C002B4E1D682B4B06EB80001A882A
:10BFC8002A4BD0F8C0101B78294800914FF47A7199
:10BFD800B5FBF1F1F9F790FC26484821F9F78CFCFC
:10BFE800D4F840800027FBB206EB8302D2F8D010C9
:10BFF800E9B101259D4015EA080F16D02A0714D08B
:10C008001D4AD25C0B2000FB0323164A1B4802EB97
:10C018008303D3F8F020F9F76FFC022D05D194F8CB
:10C028004C1011B11648F9F767FC0137DBE71548E2
:10C03800FFF7ACFF144B15481A68154BB4F85410A9
:10C048009A420CBFB4F85020B4F852204FF4DE6383
:10C0580092B202B0BDE8F041F9F74EBC00220020D0
:10C068004C1A0020C4110108880E0020000100208D
:10C078006E2B0108B12B0108FC000020C12B010820
:10C08800C92B0108112C0108181A0020CD2B010812
:10C09800005400402DE9F0410024804625460F4E0B
:10C0A800A7594146384602F00FFF58B139460C48A7
:10C0B800F9F722FC30190021FFF7F5FE0948FFF7D0
:10C0C80065FF0135143440F618339C42E7D11DB999
:10C0D8000548BDE8F04159E7BDE8F081641301085F
:10C0E800F6230108112C01087C2301082DE9F04FE3
:10C0F8002DED028B83B0054602F0A7FE064620B15F
:10C10800012818D12B782A2B15D15C48FFF73EFF60
:10C1180000245B4D5B486159F9F7EEFB281931465D
:10C12800FFF7C1FE5848FFF731FF143440F61833C3
:10C138009C42EED19CE028463D2102F078FE002882
:10C1480000F08F800346994613F8012D202AFAD073
:10C15800441C204602F0D0FE80462046F9F7C4FA77
:10C16800C5EB0909B0EE408A0026DFF834A1142295
:10C1780002FB06F40AF5D07B54F80B70384602F03F
:10C1880064FE03461A4628463946019302F066FEC5
:10C19800019B00285BD15FFA89F29A4257D10AEBDA
:10C1A8000402D2ED6B7AF8EEE77A0BEB0405B4EEF5
:10C1B800E78AF1EE10FA48DBD2ED6C7AF8EEE77A0E
:10C1C800B4EEE78AF1EE10FA3FD8B2F8A431D2F80B
:10C1D800A82113F0200F08BF08EE108A1C0641BFE3
:10C1E8002A4991F8C8164FF4C67404FB0122D905F0
:10C1F80044BF2749097803F03F0344BF01EB4101DD
:10C2080002EB8102042B18EE100A0BD004D8013B74
:10C21800012B0ED810700CE0102B05D0202B06D067
:10C22800082B06D1108004E082ED008A01E082ED3F
:10C23800008A39461748F9F75FFB2846002103B002
:10C24800BDEC028BBDE8F04F2DE6134803E0013644
:10C258008E2E8AD1114803B0BDEC028BBDE8F04F99
:10C2680094E6284603B0BDEC028BBDE8F04F11E719
:10C2780003B0BDEC028BBDE8F08F00BFFF2B0108B7
:10C2880064130108F6230108112C0108541A002030
:10C2980000220020142C01081F2C01087C2301080F
:10C2A800C411010810B50A48FFF770FE094B9C6BD2
:10C2B8002046FBF74FFD18B90A20FBF756FBF7E7B6
:10C2C800FAF7A2FEF9F75CFD034B044ADA6010BDE9
:10C2D8003F2C01080022002000ED00E00400FA05D0
:10C2E80008B50548FFF752FEFCF7C0FDF9F772FDE7
:10C2F800BDE80840D6E700BF4B2C010808B5044844
:10C30800FFF744FEF9F766FDBDE80840CAE700BF3D
:10C31800612C010820B9034B1B6808221A82704758
:10C3280001487047101A00206C00002021B901282C
:10C338008CBF0220002070470220704710B50A4BBE
:10C348001968CA78042A0CD84C8A084B28B903EB18
:10C35800C2039B881B1B0B8210BD53F8323018197F
:10C3680010BD002010BD00BF101A00207C00002066
:10C37800054B1968054B4A8A18B99B8C9B1A0B8286
:10C388007047186A10447047101A00207C0000207B
:10C39800054B1968054B4A8A18B99B8D9B1A0B8265
:10C3A8007047986A10447047101A00207C000020DB
:10C3B800074B1B681B7803F07F03212B06D100F085
:10C3C800DF00022814BF02200020704702207047B7
:10C3D800101A0020212810B508D1114B1B681B78B2
:10C3E80003F07F03212B10D0022010BD2028FBD1A1
:10C3F8000B4B0C4A1B6810701B7803F07F03212B32
:10C40800094B18BF00230BB9EEE7084B044A126822
:10C4180000249361548220469847204610BD00BFEF
:10C42800101A0020E1220020C1AA00081DC300083C
:10C438007047034B1A78202A04BF00221A707047ED
:10C44800E1220020014B04221A607047C822002014
:10C45800034B9B7A13B1034B05221A60704700BF48
:10C4680050210020C82200200D4B0E491A680E4B9F
:10C4780092B213445B000D4A1B68C3F3090310B55D
:10C48800136013689BB201335B1000229A4206D0F6
:10C49800074851F8044B20F812400132F6E710BD66
:10C4A800505C0040206200401E3000206C220020BA
:10C4B80070220020014B00225A6470476C22002031
:10C4C8002DE9F843664B674E1B68DFF8B881664A6A
:10C4D80000254FF0C0099D7283F80990DD72356020
:10C4E800D8F8003023F4EC4323F0700343F40073CE
:10C4F8009BB2C8F80030D8F8003023F4E04323F0AA
:10C5080040039BB248F2800483F010032343C8F829
:10C518000030336812FA83F35B0040271A681F6003
:10C5280033689BB203F1005303F540535B00284680
:10C538001A6880221A60D8F8003023F4F8731B05B3
:10C548001B0D2343C8F80030484B93F85C10F8F7EC
:10C5580051FCD8F80030464A464923F4804323F07A
:10C5680070039BB283F440532343C8F80030136828
:10C5780023F4EC4323F070039BB21360336811FA81
:10C5880083F35B0003201968C3F8009013683A49E5
:10C5980023F4E04323F040039BB283F020032343BA
:10C5A8001360136823F4804323F0700323439BB282
:10C5B8001360536823F4EC4323F0700343F4C0631F
:10C5C8009BB25360336811FA83F35B0019684FF428
:10C5D80080711960536823F4804323F07003234368
:10C5E8009BB25360536823F4E04323F040039BB2AB
:10C5F80083F0200323435360D8F80C301F4A23F4F8
:10C60800EC4323F070039BB2C8F80C30336812FA7D
:10C6180083F35B0039461A684FF488721A60F8F79A
:10C62800E9FBD8F80C3023F4804323F070039BB265
:10C6380083F440532343C8F80C30D8F80C3023F463
:10C64800E04323F040031C43A4B2C8F80C4028463A
:10C65800FDF77FFE0A4B01221A60BDE8F88300BF90
:10C66800101A0020505C0040043000207C0000209C
:10C67800045C004008300020103000201C300020EE
:10C68800C8220020005C0040134A144B50681B6805
:10C69800181810B5146808D011490822FDF745FE8E
:10C6A800204610490422FDF740FE0F4B1A6800236C
:10C6B80093720E4A012111600D4913604FF4E05046
:10C6C8000B6010600B480B604FF43641A0F848101F
:10C6D8001160094A136010BDB0F7FF1FACF7FF1FC8
:10C6E800DE000020EE000020101A0020405C004010
:10C6F800445C00406C220020C8220020024B4FF40A
:10C7080080221A60704700BF1404014013490B7857
:10C7180013F0010F03F004021BD0F2B910480068AF
:10C7280040011AD4980714D443F004030B700D4B3E
:10C738001A880D4B1A800D4B0D4A1B6892F8E2219E
:10C748004FF47A7101FB02330A4A05201360FBF7A4
:10C758008BBA12B90120FBF7ADBA7047E02200206E
:10C768006C0B00209C0B0020B82200204C1A0020E3
:10C77800541A0020940B0020054A1378590705D550
:10C7880023F0040304201370FBF76EBA704700BF50
:10C79800E022002008B5044B1B7803F00503052BA5
:10C7A80001D1FAF731FCFEE7BA220020D0400B1C79
:10C7B8001141203A03D49C46134118436346524220
:10C7C80093401843704700BF7BB972B90029BEBFB8
:10C7D80000204FF0004106E008BF00281CBF6FF0A2
:10C7E80000414FF0FF3000F073B882B0EC462DE9FD
:10C7F800005000F03DF8DDF804E002B00CBC7047D2
:10C8080007EE900AF5EEC07AF1EE10FA01D400F0C6
:10C8180009B808B580F0004000F004F8404261EB28
:10C82800410108BDD0B500F0B9F900220E4B06460B
:10C838000F4600F007FA00F017FC044600F08CF9E8
:10C8480000220A4B00F0FEF902460B4630463946F4
:10C8580000F044F800F008FC2346002242EA0002F7
:10C8680010461946D0BD00BF0000F03D0000F04161
:10C878002DE9F041069C154606460F46984600F0FD
:10C8880013FC05FB01F300FB0838A5FB0023B21AD3
:10C89800434467EB0303C4E90023BDE8F08100BF0C
:10C8A8002DE9F041069C904606460F461D4600F0CD
:10C8B80049FD00FB05F5A0FB082308FB0155B21A4A
:10C8C8002B4467EB0303C4E90023BDE8F08100BFF4
:10C8D800704700BF81F0004102E000BF83F00043D1
:10C8E80030B54FEA41044FEA430594EA050F08BF03
:10C8F80090EA020F1FBF54EA000C55EA020C7FEAC7
:10C90800645C7FEA655C00F0E2804FEA5454D4EB43
:10C918005555B8BF6D420CDD2C4480EA020281EA0D
:10C92800030382EA000083EA010180EA020281EA45
:10C938000303362D88BF30BD11F0004F4FEA013197
:10C948004FF4801C4CEA113102D0404261EB4101A6
:10C9580013F0004F4FEA03334CEA133302D052422C
:10C9680063EB430394EA050F00F0A780A4F10104E8
:10C97800D5F1200E0DDB02FA0EFC22FA05F2801822
:10C9880041F1000103FA0EF2801843FA05F3594108
:10C998000EE0A5F120050EF1200E012A03FA0EFC87
:10C9A80028BF4CF0020C43FA05F3C01851EBE371B1
:10C9B80001F0004507D54FF0000EDCF1000C7EEBCE
:10C9C80000006EEB0101B1F5801F1BD3B1F5001F0C
:10C9D8000CD349085FEA30004FEA3C0C04F101042B
:10C9E8004FEA445212F5800F80F09A80BCF1004F54
:10C9F80008BF5FEA500C50F1000041EB045141EAD6
:10CA0800050130BD5FEA4C0C404141EB010111F4D6
:10CA1800801FA4F10104E9D191F0000F04BF014681
:10CA28000020B1FA81F308BF2033A3F10B03B3F15F
:10CA380020020CDA0C3208DD02F1140CC2F10C02EF
:10CA480001FA0CF021FA02F10CE002F11402D8BF4D
:10CA5800C2F1200C01FA02F120FA0CFCDCBF41EA19
:10CA68000C019040E41AA2BF01EB0451294330BDE8
:10CA78006FEA04041F3C1CDA0C340EDC04F11404C5
:10CA8800C4F1200220FA04F001FA02F340EA03009C
:10CA980021FA04F345EA030130BDC4F10C04C4F1E2
:10CAA800200220FA02F001FA04F340EA03002946C2
:10CAB80030BD21FA04F0294630BD94F0000F83F40C
:10CAC800801306BF81F480110134013D4EE77FEAEF
:10CAD800645C18BF7FEA655C29D094EA050F08BF3B
:10CAE80090EA020F05D054EA000C04BF194610461C
:10CAF80030BD91EA030F1EBF0021002030BD5FEA60
:10CB0800545C05D14000494128BF41F0004130BD87
:10CB180014F580043CBF01F5801130BD01F00045DB
:10CB280045F0FE4141F470014FF0000030BD7FEA4E
:10CB3800645C1ABF194610467FEA655C1CBF0B4649
:10CB4800024650EA013406BF52EA033591EA030F60
:10CB580041F4002130BD00BF90F0000F04BF002158
:10CB6800704730B54FF4806404F132044FF000058B
:10CB78004FF0000150E700BF90F0000F04BF002104
:10CB8800704730B54FF4806404F1320410F000456A
:10CB980048BF40424FF000013EE700BF42004FEA65
:10CBA800E2014FEA31014FEA02701FBF12F07F43E2
:10CBB80093F07F4F81F06051704792F0000F14BFDF
:10CBC80093F07F4F704730B54FF4607401F0004523
:10CBD80021F0004120E700BF50EA010208BF70477A
:10CBE80030B54FF000050AE050EA010208BF70476F
:10CBF80030B511F0004502D5404261EB41014FF4D8
:10CC0800806404F132045FEA915C3FF4DCAE4FF0DB
:10CC180003025FEADC0C18BF03325FEADC0C18BFC2
:10CC2800033202EBDC02C2F1200300FA03FC20FA13
:10CC380002F001FA03FE40EA0E0021FA02F1144460
:10CC4800C1E600BF70B54FF0FF0C4CF4E06C1CEA75
:10CC580011541DBF1CEA135594EA0C0F95EA0C0FEA
:10CC680000F0DEF82C4481EA030621EA4C5123EA5D
:10CC78004C5350EA013518BF52EA033541F480118C
:10CC880043F4801338D0A0FB02CE4FF00005E1FB3F
:10CC980002E506F00042E0FB03E54FF00006E1FB89
:10CCA80003569CF0000F18BF4EF0010EA4F1FF04CC
:10CCB800B6F5007F64F5407404D25FEA4E0E6D410C
:10CCC80046EB060642EAC62141EA55514FEAC5201D
:10CCD80040EA5E504FEACE2EB4F1FD0C88BFBCF599
:10CCE800E06F1ED8BEF1004F08BF5FEA500E50F14A
:10CCF800000041EB045170BD06F0004646EA010110
:10CD080040EA020081EA0301B4EB5C04C2BFD4EB41
:10CD18000C0541EA045170BD41F480114FF0000E3A
:10CD2800013C00F3AB8014F1360FDEBF002001F0A8
:10CD3800004170BDC4F10004203C35DA0C341BDC22
:10CD480004F11404C4F1200500FA05F320FA04F0F4
:10CD580001FA05F240EA020001F0004221F0004128
:10CD680010EBD37021FA04F642EB06015EEA430E9B
:10CD780008BF20EAD37070BDC4F10C04C4F12005CB
:10CD880000FA04F320FA05F001FA04F240EA02007E
:10CD980001F0004110EBD37041F100015EEA430E4F
:10CDA80008BF20EAD37070BDC4F1200500FA05F26F
:10CDB8004EEA020E20FA04F301FA05F243EA0203EE
:10CDC80021FA04F001F0004121FA04F220EA0200FD
:10CDD80000EBD3705EEA430E08BF20EAD37070BD43
:10CDE80094F0000F0FD101F00046400041EB010123
:10CDF80011F4801F08BF013CF7D041EA060195F005
:10CE0800000F18BF704703F00046520043EB0303BE
:10CE180013F4801F08BF013DF7D043EA06037047AB
:10CE280094EA0C0F0CEA135518BF95EA0C0F0CD0B6
:10CE380050EA410618BF52EA4306D1D181EA0301FC
:10CE480001F000414FF0000070BD50EA410606BFF6
:10CE58001046194652EA430619D094EA0C0F02D13B
:10CE680050EA013613D195EA0C0F05D152EA033680
:10CE78001CBF104619460AD181EA030101F000419E
:10CE880041F0FE4141F470014FF0000070BD41F0E7
:10CE9800FE4141F4780170BD70B54FF0FF0C4CF4C1
:10CEA800E06C1CEA11541DBF1CEA135594EA0C0FE0
:10CEB80095EA0C0F00F0A7F8A4EB050481EA030E2D
:10CEC80052EA03354FEA013100F088804FEA033314
:10CED8004FF0805545EA131343EA12634FEA0222E2
:10CEE80045EA111545EA10654FEA00260EF00041A3
:10CEF8009D4208BF964244F1FD0404F5407402D2F5
:10CF08005B084FEA3202B61A65EB03055B084FEA85
:10CF180032024FF480104FF4002CB6EB020E75EB82
:10CF2800030E22BFB61A754640EA0C005B084FEAAA
:10CF38003202B6EB020E75EB030E22BFB61A754627
:10CF480040EA5C005B084FEA3202B6EB020E75EB72
:10CF5800030E22BFB61A754640EA9C005B084FEAEA
:10CF68003202B6EB020E75EB030E22BFB61A7546F7
:10CF780040EADC0055EA060E18D04FEA051545EAE6
:10CF880016754FEA06164FEAC30343EA52734FEA8F
:10CF9800C2025FEA1C1CC0D111F4801F0BD141EA08
:10CFA80000014FF000004FF0004CB6E711F4801F6D
:10CFB80004BF01430020B4F1FD0C88BFBCF5E06F4D
:10CFC8003FF6AFAEB5EB030C04BFB6EB020C5FEA5D
:10CFD800500C50F1000041EB045170BD0EF0004EB2
:10CFE8004EEA113114EB5C04C2BFD4EB0C0541EAE4
:10CFF800045170BD41F480114FF0000E013C90E6E1
:10D0080045EA060E8DE60CEA135594EA0C0F08BFA4
:10D0180095EA0C0F3FF43BAF94EA0C0F0AD150EAA3
:10D0280001347FF434AF95EA0C0F7FF425AF104636
:10D0380019462CE795EA0C0F06D152EA03353FF45E
:10D04800FDAE1046194622E750EA410618BF52EADB
:10D0580043067FF4C5AE50EA41047FF40DAF52EAAF
:10D0680043057FF4EBAE12E74A0011D212F5001225
:10D0780011D20DD56FF47873B3EB62520ED44FEA28
:10D08800C12343F0004343EA505323FA02F07047A8
:10D098004FF00000704750EA013002D14FF0FF30E6
:10D0A80070474FF00000704700292DE9F043C0F2A7
:10D0B800A6800026002BC0F29C80884694469E4697
:10D0C800154604460F46002B3DD18A4259D9B2FA7B
:10D0D80082F33BB1C3F120029F4020FA02F29D4047
:10D0E80017439C40290C220CB7FBF1FEA8B201FBA8
:10D0F8001E7742EA074700FB0EF3BB420AD97F19A5
:10D108000EF1FF3280F00581BB4240F20281AEF1A0
:10D11800020E2F44FF1AA4B2B7FBF1F301FB1377F9
:10D1280044EA074700FB03F0B84208D97F1903F126
:10D13800FF3280F0F080B84240F2ED80023B43EAD3
:10D148000E43002203E08B420FD900221346341C01
:10D1580018BF012460424FF0000565EB45015840B7
:10D16800514000196941BDE8F083B3FA83F2002AFF
:10D1780040F086808B4202D3844500F2DB80012395
:10D18800E5E712B90123B3FBF2F5B5FA85F00028FB
:10D198003BD1781B4FEA154E1FFA85FC0122B0FBE4
:10D1A800FEF8210C0EFB180741EA07470CFB08F3B1
:10D1B800BB4207D97F1908F1FF3102D2BB4200F206
:10D1C800BD808846FF1AA4B2B7FBFEF30EFB1377A7
:10D1D80044EA07470CFB03FCBC4507D97F1903F158
:10D1E800FF3102D2BC4500F2A7800B4643EA084350
:10D1F800ADE752426FEA060663EB43035DE7404240
:10D2080061EB41014FF0FF3654E7C0F1200224FAE8
:10D2180002F107FA00F385404FEA154ED74019434B
:10D22800B7FBFEF20B0C0EFB12771FFA85FC43EAE4
:10D2380007430CFB02F79F4204FA00F407D95B1975
:10D2480002F1FF3074D29F4272D9023A2B44DF1B9D
:10D2580089B2B7FBFEF80EFB187341EA03430CFBD7
:10D2680008F79F4208D95B1908F1FF315CD29F4249
:10D278005AD9A8F102082B44D81B48EA02428EE783
:10D28800C2F120032CFA03F10EFA02FE20FA03F78A
:10D2980041EA0E0E08FA02F028FA03F14FEA1E4599
:10D2A8003843B1FBF5F8030C05FB18111FFA8EF78C
:10D2B80043EA014107FB08F38B420CFA02FC09D947
:10D2C80011EB0E0108F1FF3930D28B422ED9A8F1AB
:10D2D80002087144C91A80B2B1FBF5F305FB1311BA
:10D2E80040EA014107FB03F78F4208D911EB0E0111
:10D2F80003F1FF3016D28F4214D9023B714443EA3E
:10D308000843C91BA3FB0C89494509D305D0002252
:10D318001DE79646FEE6134611E794404445F6D2CB
:10D32800013BF4E70346EAE78846A5E7C846D1E7A4
:10D3380002468CE713460AE7023B57E7A8F10208C2
:10D348002F443FE72DE9F041002B44D18A4215468E
:10D3580004464FD9B2FA82F70E464FB1C7F12003FF
:10D36800B94020FA03F602FA07F50E4300FA07F46B
:10D378004FEA154E230CB6FBFEF0AFB20EFB106160
:10D3880043EA014307FB00F1994209D95B1900F10F
:10D39800FF3280F0EC80994240F2E98002382B4459
:10D3A8005A1AA4B2B2FBFEF30EFB132244EA02425D
:10D3B80007FB03F7974208D9521903F1FF3180F0B0
:10D3C800D880974240F2D580023B43EA00400026CD
:10D3D8003146BDE8F0818B4247D8B3FA83F6002E78
:10D3E80048D18B4202D3824200F2CD8001203146DF
:10D3F800BDE8F08112B90125B5FBF2F5B5FA85F85B
:10D40800B8F1000F77D14A1B4FEA154EAFB201268B
:10D41800B2FBFEF0230C0EFB102143EA014107FB8F
:10D4280000F38B4207D9491900F1FF3202D28B422F
:10D4380000F2BA801046C91AA4B2B1FBFEF30EFB83
:10D44800131144EA014407FB03F7A74208D96419FA
:10D4580003F1FF3280F08F80A74240F28C80023BBC
:10D4680043EA00403146BDE8F081002630463146A7
:10D47800BDE8F081C6F1200422FA04F5B3402B433D
:10D4880020FA04FC01FA06F721FA04F54FEA134ED4
:10D498004CEA0707B5FBFEF8390C0EFB18551FFAC6
:10D4A80083FC41EA05450CFB08F1A94202FA06F2A1
:10D4B80004D9ED1808F1FF3467D3A0466D1ABFB23E
:10D4C800B5FBFEF40EFB145547EA05410CFB04FCC2
:10D4D8008C4504D9C91804F1FF355CD32C4644EABD
:10D4E8000844CCEB0101A4FB0223994248D344D061
:10D4F800204600266CE7C8F1200401FA08F305FA73
:10D5080008F520FA04F7E1404FEA154E1F43B1FB36
:10D51800FEF63A0C0EFB16111FFA85FC42EA01438F
:10D528000CFB06F29A4200FA08F407D95B1906F1D7
:10D53800FF3137D29A4235D9023E2B449B1ABFB2EB
:10D54800B3FBFEF00EFB103347EA03430CFB00F17C
:10D55800994207D95B1900F1FF3221D299421FD9AC
:10D5680002382B445A1A40EA0646674650E71046E6
:10D5780016E70B4629E7134672E7B0409042B7D248
:10D58800601E002624E7304622E7A94295D9A8F173
:10D5980002081D4492E78C45A0D9023C19449EE735
:10D5A8001046DFE70E46C9E70238294443E700BFC3
:10D5B8004FEA4102B2F1E04324BFB3F5001CDCF1AD
:10D5C800FE5C0DD901F0004C4FEAC0024CEA5070E5
:10D5D800B2F1004F40EB830008BF20F00100704714
:10D5E80011F0804F21D113F13872BCBF01F0004017
:10D5F800704741F480114FEA5252C2F11802C2F149
:10D60800200C10FA0CF320FA02F018BF40F00100C9
:10D618004FEAC1234FEAD32303FA0CFC40EA0C007B
:10D6280023FA02F34FEA4303CCE77FEA625307D1B8
:10D6380050EA01331EBF4FF0FE4040F440007047EF
:10D6480001F0004040F0FE4040F40000704700BF89
:10D6580011481249026800608A4218D0002103E08C
:10D668000F4B5B58435004310E480F4B42189A42F7
:10D67800F6D30E4A02E0002342F8043B0C4B9A42D0
:10D68800F9D3FBF7B3FE00F019F87047FEE7094835
:10D69800D0F800D040680047FC9F0020EFBEADDE08
:10D6A800943A010800000020700100207001002059
:10D6B800E822002000D8FF1FFEE700002DE980487F
:10D6C80095B0F2F75DFDAC4DDFF810A32B78DAF8D2
:10D6D800004033B1A94B1B68E31A002BA4BF0023F9
:10D6E8002B70FEF751FB10B1A54B00221A70A54B09
:10D6F80019680F0740F18281A34B1B681B7A062B20
:10D7080000F27081DFE813F0070007003200CC0058
:10D718000501300130019D4B1A78002A00F0628122
:10D7280000221A709A4B1F789A4B1B6893F800E0F6
:10D73800994B93F800C00222984EB35C3B4103F02A
:10D748000F03734502F101080CD20B2B9FBFB05C8D
:10D7580016F8086000EA0C0006EB00209CBF904E0B
:10D7680046F823000232102AE6D102E18D4B1A78DE
:10D77800002A00F0378100221A708B4B8B4A93F8ED
:10D7880002E0DF7858780EF0070640EA062007F036
:10D798003F06760146EADE061060187956605E7923
:10D7A80093F806E0800040EA971006F0010740EA87
:10D7B80087209060DF790EF00F00C00140EA560024
:10D7C80007F07F06D0603601187A46EA1E1693F8ED
:10D7D80009E0166140000EF0030640EAD71040EA5F
:10D7E80046209F7A5061D87A07F01F06B601C0001C
:10D7F80046EA9E0640EA571093F80DE09F7BD061F9
:10D80800187B96610EF0070640EA062007F03F06EF
:10D81800760146EADE061062D87B56621E7C93F8D3
:10D8280011E0800040EA971006F0010740EA8720DF
:10D8380090629F7C0EF00F00C00140EA560007F08E
:10D848007F06360146EA1E16D062D87C166393F826
:10D8580014E0400040EAD7100EF003065F7D40EA6E
:10D868004620506307F01F06987DDB7DB60146EA27
:10D878009E06C00040EA57109663DE07D0634CBF8F
:10D8880040F21470AD20106498074CBF40F2147039
:10D89800AD2013F0080F506414BF03230123A2E046
:10D8A800434A1378002B00F09D8000231370414AEF
:10D8B800414F1678414807EB460EB0F800C09EF875
:10D8C80003809EF8040040EA0820844540F08A80DE
:10D8D8007878012804D0812840F08580032300E06F
:10D8E8000346102E84BF1020107035481778002288
:10D8F800D6B2BE4200F1020075D210F802EC10F860
:10D90800016C46EA0E26DFF8D8E02EF812600132E4
:10D91800EEE72C4B1A78002A64D000221A702A4BA2
:10D928001A78A82A1E465DD1DA7C002A5AD106EB5D
:10D9380042009FED267AC778037903EB072307EEA9
:10D94800903AF8EEE77A224BC7EE877A9FED217A74
:10D9580077EEC77AFCEEE77A17EE900A43F82200D2
:10D968000132082AE3D104E01B4B1A78D2B3002213
:10D978001A70012337E000BF030B002018040020B1
:10D98800040B00202422002020220020410D00202A
:10D998004A210020442100204B210020310D002085
:10D9A800280C0020B20D0020990D0020980C0020B2
:10D9B800690D00206C0D00206D0D00206A0D0020FF
:10D9C800700D0020620D00204D0D0020CDCCCC4004
:10D9D800580C00200080BB43240C0020C0220020EB
:10D9E800780C00200023DF0741BF83F002038A4A36
:10D9F8000120C3F3400344BF10702B704E0406D5BA
:10DA0800864A13780BB100201070834A137044F2D1
:10DA180008030B403BB1804B1B7823B104F5C3339B
:10DA28007F4AA0331360C8070CD57D4B5A79187903
:10DA380082421FBF01222A7004F5C332A0321CBFE4
:10DA48001A605871890407D50023764A32F81320E2
:10DA580082BB01330C2BF8D16F4B714D1B7823B966
:10DA6800714B1B68E41A002C04DBF5F721FF012336
:10DA7800AB7104E0AB68013303EAE373AB60DFF832
:10DA8800C881F9F74BFF98F80F30CAF80000EC6826
:10DA980063B1664B0DA8DB6898479DF834308BB9A5
:10DAA800634B1868001B96280CD50CE6001B002851
:10DAB80008DA08E601232B70594A04F5C333A0336A
:10DAC8001360C9E7D5F8EC20DAF8003059485A4F06
:10DAD800534C1344EB60594B1E68544B5B68984792
:10DAE800544895F8B9260146F7F78CFC3B88394627
:10DAF800002B74D023691B7808EE103A04F114093E
:10DB08004FF0000B2034B1F800E04A48BEF57A7FA8
:10DB180002BF0023C9F80030236130F91BC0D9F8CF
:10DB280000306344C9F80030236907EE90CA013316
:10DB3800012B4FEA4B02F8EEE77A236106D1002366
:10DB4800C4ED017AC4ED007AA3601BE0D4ED006A4D
:10DB580007EE103A37EEE66AB8EEC77A86EE077A2D
:10DB680036EE877AD4ED026A84ED017A77EEC77AC9
:10DB780084ED007AE6EE276AF0EE667AC4ED036A71
:10DB8800C4ED026A002383522D48BEF1010F1352DF
:10DB980030D123690491012BC3BF03F1FF3300EE99
:10DBA800103AD4ED037A9FED270A0390C8BFB8EE68
:10DBB800C00A0292C8BF87EE800A01F0E5FB029A0C
:10DBC8000398049918EE103A5BB1F8EEC87AB4EEEF
:10DBD800E70AF1EE10FA04DD4FF47A733B80002374
:10DBE80034E0D9F800304FF47A7E03F5FA7393FBEA
:10DBF800FEF383520BF1010BBBF1030F09F104098A
:10DC080004F114047FF47FAF3888012801D1FAF7B2
:10DC18002BF83B88013BE1E7040B00200A040020B5
:10DC280018040020040D0020D80A0020A02100209C
:10DC3800C0220020C20E0020D8220020FC110020A3
:10DC48007404002000000000541A0020C04CC14990
:10DC580004F15C0031F8132030F81300121A21F88F
:10DC680013200133032BF1D1BB4B1B6813F00203C4
:10DC780000F0C282B94B04F162005B689847B84B68
:10DC880004F162001A780146F7F7BCFBB54B1B8814
:10DC9800002B3FD0A06E0023B24AB3491288AC4F84
:10DCA800B2F5C87F04BF002241F823204FEA830C55
:10DCB80007F1620E51F80C203EF91340224441F856
:10DCC8000C2000212EF8131020F813100133032B19
:10DCD800E2D1A44C2388012B19D1FB6E4FF4C87EE6
:10DCE800C83393FBFEF303803A6FC83292FBFEF20F
:10DCF80042809E4A7B6F1288C83393FBFEF39B1ABF
:10DD08008380A6F85810A6F85A10F8F7BFFA2388A7
:10DD1800013B2380964B1B685A0777D5954B1B8888
:10DD2800322B12D1AB6E1A88A5F878205A889B88B6
:10DD3800A5F87C30B6F85830A5F87E30B6F85A30D9
:10DD4800A5F87A20A5F8803001E0002B3FD0D5F85F
:10DD580068E00023874A7E4C1288322A864A04BF2C
:10DD6800002142F823104FEA830C04F1620752F8AD
:10DD78000C1037F91300014442F80C10002227F860
:10DD880013202EF813200133032B1146E2D1794FCB
:10DD98003B88012B18D1794A1170794A0C201370ED
:10DDA800F9F762FFA36EB4F878201A80B4F87A20E5
:10DDB8005A80B4F87C209A80B4F87E30A6F858309F
:10DDC800B4F88030A6F85A303B88013B3B806D4B55
:10DDD8001A78DAB1A96E002232201A70D5F8843088
:10DDE80093FBF0F30B80D5F8883093FBF0F34B806E
:10DDF800D5F88C3093FBF0F35C4800881B1A8B80B5
:10DE0800A6F85820A6F85A20F8F740FAAA6EB5F8EE
:10DE1800623011885B1AA5F862305188B5F8643011
:10DE28005B1AA5F864309288B5F866309B1AA5F895
:10DE38006630F9F773FDD5F8903095ED256AD5F879
:10DE48009860C5F89000C3EB000B07EE90BAB8EEE7
:10DE5800678A002428EE066A96F800E04A484B498B
:10DE680007AF22463B4B33F9123007EE903AF8EEF3
:10DE7800E77A474B67EE867AE7EC017ABEF1000F46
:10DE88001CD007EE90EAF8EEE76AB7EE007AC7EE24
:10DE9800266A33F9123007EE903AF8EEE77A37EE51
:10DEA800667A67EEA67AD1ED006AE6EE877AC1ED6A
:10DEB800007AFDEEE77A17EE903A01E033F8123077
:10DEC800438030F8023F0132032A13FB034401F177
:10DED8000401C7D1254F2F48642363433C8864431A
:10DEE80093FBF4F4493C07A9A4B2F7F7DBFE3B2CFB
:10DEF800D6ED016A11D9B5F9B430D5ED2C0A07EE83
:10DF0800903AF8EEE77A244BF4EEE70AF1EE10FACD
:10DF180046DD1A7842F0080245E0F7EE007A36EE60
:10DF2800A77A1C4A87EE877A00231C4931F9131017
:10DF38000133032B07EE901A92ED006AF8EEE77AA8
:10DF4800E6EE267A67EE877AE2EC017AEDD1D2E73F
:10DF580018040020C20E0020402200204422002085
:10DF6800DB220020A20B00208404002002000020F5
:10DF780024220020A40B00209C040020A60B0020D3
:10DF88009E0B00209F0B0020EE030020B40400200D
:10DF98007A040020C0040020920B0020F003002027
:10DFA8001A7822F0080295ED2B0A1A7001F0EAF9A6
:10DFB800DFF8C493D5ED2B7A89ED000A95ED2C0A8C
:10DFC800D5ED2A8ADB4C20EE000AF1EE688AA7EE2E
:10DFD800A70A01F0D9F9F0EE400AB0EE680A01F09C
:10DFE800D1F9DFEDD58A89ED010A99ED000A20EE15
:10DFF800280A01F0F5F899ED010A208020EE280A98
:10E0080001F0EEF8CD4B60801B681B0721D5CC488A
:10E0180007A9F7F747FED6ED026AC94AF7EE007A74
:10E0280036EEA77A002387EE877AC64931F91310AE
:10E038000133032B07EE901A92ED006AF8EEE77AA7
:10E04800E6EE267A67EE877AE2EC017AEDD1BC48F3
:10E058002AE0BD4C07A92046F7F724FE94ED010AF3
:10E0680094ED007AD4ED027A20EE000AA7EE070AB2
:10E07800A7EEA70A01F088F9B5EE400AF1EE10FA0A
:10E0880011D0D4ED007AC7EE807AC4ED007AD4EDD1
:10E09800017AC7EE807AC4ED017AD4ED027A87EE70
:10E0A800800A84ED020AA848F9F730F8DFEDA77A6C
:10E0B800A74B9FEDA87A188028EE278AD9ED007A19
:10E0C800A34BF1EE677ACDED0A7AD9ED017AB3F96F
:10E0D8000030F1EE677ACDED0B7A07EE903A9E4B61
:10E0E800F8EEE77AB3F9002067EEC77A0DA8CDED10
:10E0F8000C7A07EE902AB3F90220B3F90430F8EE4F
:10E10800E77A0AA9CDED0D7A07EE902AF8EEE77ABC
:10E11800CDED0E7A07EE903AF8EEE77ACDED0F7A6C
:10E12800F7F7C0FD73789DED0F7A012B19D18B4B52
:10E138001B785C070FD4D5F8C430402293FBF2F269
:10E148009B1A07EE903AF8EEE77A77EE877AFDEEBB
:10E15800E77AC5ED317AD5F8C430402293FBF2F363
:10E1680000E03B889DED0D0A07EE903AF8EEE77A5D
:10E1780037EE677AD5ED327A8DED0F7A95ED337AF1
:10E1880038EE077A88EE078A9DED0F7A37EE677AC0
:10E19800E8EE077AB0EE678AC5ED327A01F020F82A
:10E1A800D5F8D0402178F7F7A9FCD5F8D4309DED03
:10E1B8000E0A1844C5F8D40001F012F82178F7F7D0
:10E1C8009DFCD5F8D830B0EE480A1844C5F8D800F8
:10E1D80001F006F86178F7F791FCD5F8DC30604A71
:10E1E80018441368C5F8DC005B441360D5F8E030C8
:10E1F8000133C5F8E03005E0A4F86230A4F86430D3
:10E20800A4F86630F9F78AFBD5F8E430CAF80000BC
:10E21800C31A9BB207EE903A524EDFF860A19FED09
:10E228004B7AAAF80030F8EE677A3368DFF8509135
:10E2380093F852304C4AC5F8E40067EE877AB34643
:10E24800C9ED007A2BB998F81030002B00F0BD808A
:10E258002DE0D2ED3A7AF5EE407AF1EE10FA04BFED
:10E26800D2ED3B7AF8EE677A4FF0000404BF67EE10
:10E27800877AC2ED3A7A3D4F3D4837F91430D5EDEB
:10E288003A0A00EE103ADBF8003000EBC40093F8CD
:10E298005210B8EEC00AF7F7FDF9FDEEC07A17EE96
:10E2A800903A27F814300134032CE4D1CBE7BAF8BC
:10E2B80000302D4FD9ED000AB5F8084100EE103AAC
:10E2C80007F58670B8EE400A0121F7F7E3F9BCEECE
:10E2D800C00AAB798DED020ABDF80800B4FBF0F076
:10E2E800441CA4B2A5F81441002B4BD0B7F816B1C2
:10E2F80000231D491F4A01F5907E01F58C7932F8FB
:10E3080013C03EF8137039F813202EF813C0C7EB6A
:10E318000C0712FB0BF20FFA84FA92FBFAF217447D
:10E3280029F813700133042BE3D100238B71A1F872
:10E3380016012CE0221A00204C3D0F4440220020F8
:10E34800D00400200E04002004000020BD378635CC
:10E358009C0B002035FA8E3CF0030020E0220020C0
:10E36800BC220020FC11002018040020C20E00204E
:10E3780008050020E00C0020101100205422002085
:10E38800E40E0020B7F81631013BA7F81631B5F8AE
:10E398001601B24A03B2002B4FF0000313DDB2F9A5
:10E3A8001441AF4931F81320083112FB00F231F85B
:10E3B800131092FBF4F28A1AAA4921F813200133A8
:10E3C800042BEED101E0A2F81631A74FDFF8FCA22A
:10E3D800DFF8FC92F3F7C4F93B6813F4801300F0FC
:10E3E8009280B9F80030180600F1DA809F4B1B784C
:10E3F80003F0040303F0FF0B002B71D09C4A9D4BE4
:10E40800117811B195F8281139B19B49002008609D
:10E4180001211973002185F828111B7BDAF80040C7
:10E428001370032B05D120469449542200F0BEFCFA
:10E438004FE0012B06D154229048214600F0B6FC4B
:10E44800002202E0022B02D101228D4B1A708D4A64
:10E45800012313708C4A13708C4A002313608C4A72
:10E4680013608C4B1C608C4B22781A70844B8B4A3F
:10E478001B78D05C8A4B8B4A18707F4B20441A60FB
:10E488004278894B07EE902AF8EEE77AB2EE047AE2
:10E49800C7EE877AC27A9FED857AC3ED007A07EED8
:10E4A800902AF8EEE77A427DC7EE877A9FED807A68
:10E4B800C3ED017A07EE902AF8EEE77A67EE877ADD
:10E4C800C3ED027AFCEEE77A17EE903A4375002323
:10E4D800C3728020F7F734FC012385F880315FE0B0
:10E4E800654CD4ED007AF5EE407AF1EE10FA57D08B
:10E4F800F7F7CCFE002323605D4B83F800B05D4B3B
:10E5080001221A734CE0B9F8002011063DD5584A8B
:10E518001078411E012957492CD8634C5D4BD4ED26
:10E52800017A9FED627A1A685D4B67EE877A1878F0
:10E538009FED607AFCEEE77A104417EE903AC372CA
:10E54800D4ED027A67EE877AFCEEE77A17EE903A16
:10E558004375537807EE903AF8EEE77A77EEA77AA4
:10E56800FCEEE77A17EE903AD370D37A5373537D63
:10E57800D37504E0032802D11370012301E00B7B5B
:10E58800013380200B73F7F7CAFB384B1B785A0707
:10E5980006D495F880311BB1304B012283F828212D
:10E5A800454B464C1B78ABB12E4B454AB3F9061088
:10E5B800B2F89A3199420DDC5379012B01D0192B0D
:10E5C80002D192F8E8212AB90E2B03D0082B1CBFE0
:10E5D8000023A380DAF8003093F818A1BAF1000FED
:10E5E8007CD0B9F800309B0778D095ED2B0AD5ED93
:10E5F8002A7A95ED2C8A20EE000AA7EEA70AA8EE43
:10E60800080A00F0C1FE88EE000ADFED2E7AB4EEAB
:10E61800E70AF1EE10FA5DD900F056FE0F4BD3ED84
:10E62800617A20EE270A00F0DBFDB0F5617FA8BF14
:10E638004FF4617007EE900AB8EEE70ADFED227A30
:10E6480080EE270AF7F769FA07EE90AAF8EEE77A5C
:10E6580027EE800A00F0C4FD80B23CE018040020D8
:10E6680030050020E00C00206C0B0020E022002088
:10E678001C1A002004000020281A0020440500204D
:10E688001D1A0020201A0020381A00202C1A0020F9
:10E69800301A0020481A00201E1A0020C011010854
:10E6A8001F1A00200000A0413C1A002000007A44F4
:10E6B8005555553F9A99993F14000020BA0E0020ED
:10E6C800541A00208FC2753CEFB6B044FC110020EC
:10E6D800B80E00200020E3881844E080894B306899
:10E6E800B8F86E210093884B1E68884B196800F1B2
:10E6F8005803B047864B87491E78032E1AD9D5F898
:10E708008831B3F802E0BEF5FA7F13D2B4F90400F9
:10E71800B1F904C080EAE078A8EBE078CEF1000215
:10E72800C8EB02039C4504DB0EEB08036345A8BF56
:10E7380063468B80E488B1F802E0B1F800C0D5F8F0
:10E748008881B1F90490744A0020B04202F11002A5
:10E7580033D298F9013052ED045ADFF8C8A15B4270
:10E7680009FB03F307EE903A0FFA8CF306EE903AA2
:10E7780023B206EE103A0FFA8EF3B8EEE77A07EEF8
:10E78800903AF8EEE77AB8EEC66A67EEA57A52EDE7
:10E79800065AE6EE257AF8EEE66A12ED056AE6EE26
:10E7A800867A52ED036AE7EE267AFDEEE77A17EEEF
:10E7B800903A2AF810300130C7E7584B1A7802F01F
:10E7C800040202F0FF03002A7BD0554B554ADB7840
:10E7D8000393138801209646B0421AB207D23EF935
:10E7E80010309A42B8BF1A4693B20130F4E74E4847
:10E7F800D5F84C8200684488A242C8BF1C1B4B4B0A
:10E808001B6803F480520492494AB2F906C0494A87
:10E81800D2F80090434A03F0100BD5F888310293E0
:10E8280002EB4603CCBFA4B200240593059B9A4291
:10E838003ED01388049E1B1B9BB222F8023B1BB2DE
:10E8480066B1B8F80EE0F445C7BFB9F802E0B0F811
:10E8580002A0B0F804E0B9F800A005E0039EB0F803
:10E8680002A056B1B0F804E0734503DB5345A8BFD6
:10E8780053469E4622F802ECD8E7B0F800E073450C
:10E8880003DB5345A8BF53469E4622F802ECB8F86E
:10E8980010309C45CADABBF1000F01D0838804E030
:10E8A800029B1B78002BC1D1038822F8023CBDE7EC
:10E8B80095F85032204C013BDBB2182B00F2448112
:10E8C80009E0B342F4D21D4A32F81300154A22F87F
:10E8D80013000133F5E701229A40194B1340002B2E
:10E8E80000F03281174B1B8813F4807F104B2DD01A
:10E8F800154A1188ADF834105188ADF83610928851
:10E908003AE000BFDE1B0020F800002004220020AF
:10E918005B0F0020300F0020AC050020E022002013
:10E92800D8210020800F00209410002024220020ED
:10E93800E00C002090100020F603002008220020A0
:10E9480099209801B80E0020BA0E00200A88ADF868
:10E9580034204A88ADF836208A88AF49ADF8382087
:10E968000968C8040AD5AD49B3F90600D1F84C12B4
:10E97800C989884202DA5242ADF83820A84EB6F961
:10E9880002204FF47A7102F5E1624A434FF4616064
:10E9980092FBF0F2A2F5FA72ADF84C20B6F900201D
:10E9A80002F5E16251439F4A91FBF0F11288A2F20D
:10E9B800DC52A1F5FA71ADF83A20D5F84C22ADF841
:10E9C8004E10D2891988891AADF83C105988891ACD
:10E9D800ADF83E109988891AADF84010D988891A7F
:10E9E800ADF842101989891AADF844105989891A65
:10E9F800ADF846109989DB89891A9A1AADF848103A
:10EA0800ADF84A200023002224F813200133082BF4
:10EA1800F9D13A68844B0292844A1B781268844977
:10EA28000392844E072202FB031B594572D00B78D0
:10EA380033B103F1150201239340029A134065D0C4
:10EA480011F806CC039B11F805AC11F8035C11F81A
:10EA5800018CCCEBCC0E03EB4E0E6420BEF90020EB
:10EA6800BEF902309B1A9BB211F9022C4FEA5309E6
:10EA78005A434FEA4A0792FBF0F214A8C9EB020284
:10EA880092B2074415B937F81C0C0CE0B6F900002F
:10EA980037F91C7CB84208DA0544854203DBAF42EB
:10EAA8003846A8BF2846308008E007DD451BBD4230
:10EAB80003DB8542A8BF05462F463780DEF80A509B
:10EAC80011F9047C012000FA0AF02842308812B2B9
:10EAD80017FB00F014BF4FF0FF350125642790FBAA
:10EAE800F7F090420ADB4FFA88F25A4392FBF7F2AA
:10EAF800C9EB020212B28242A8BF02464E4B33F85B
:10EB08001C9002FB059523F81C5000E03380023668
:10EB180007318AE7454B494FD3F8008000260E227B
:10EB280002FB068237F8023F92F90650F0B215FB55
:10EB380003F3642593FBF5F53D80F8F7CDFA01362C
:10EB48002844082E3880EAD1334E384D336813F004
:10EB5800200F32D00020F8F7BFFA2080804601202D
:10EB6800F8F7BAFA364B344F1B686080190624D57B
:10EB78002A4BD5F800C0D3F87432294A1B78012BE8
:10EB88001FD113889CF91410B2F9022011FB03F36A
:10EB98004FF0320E93FBFEF399B29CF906305B42BC
:10EBA80053436FF0310293FBF2F20A44424493FB61
:10EBB800FEF30B443A8018447880D5F800E000232F
:10EBC80018E09CF9061053884FF0320E11FB03F33E
:10EBD80093FBFEF308EB0301398011889CF914209C
:10EBE80012FB01F292FBFEF21044E5E70133082B19
:10EBF800E25327D00E2101FB03E134F91300B1F9E8
:10EC08000020B1F9021090424FEA4307EEDB0AB246
:10EC18008242A8BF0246E9E7242200201804002007
:10EC2800221A0020800F00209810002000120020D7
:10EC38009F1000206A060020F6030020F40300203D
:10EC48006C0B0020544FD7F888A19AF90830A3B963
:10EC580097F8508208F1FF33182B72D8DFE803F0D9
:10EC68003571714F7171714871717171715971712B
:10EC78007171714F657171593500DFF82C914FF042
:10EC88000008464B39F9021FBAF90620882000FB14
:10EC98000830F8F75DF82A680E2380B203FB0822D3
:10ECA800A9F80000B2F90030B2F9022000B2984287
:10ECB80003DB13B28342A8BF034608F10108B8F189
:10ECC800080FA9F80030DCD1C2E79AF8043013B174
:10ECD8000020618908E0324B1B7803F0040303F03D
:10ECE800FF00002BF4D10146FBF788F9012529E044
:10ECF8000020E188FBF782F90120218905E0002046
:10ED08002189FBF77BF961890120FBF777F9022557
:10ED180018E00225A81E34F81510C0B20135FBF71B
:10ED28006DF9082DF6D106250CE00325E81E34F808
:10ED38001510C0B20135FBF761F9072DF6D104258E
:10ED480000E0002533689A0602D4B8F1050F0AD10D
:10ED580028462188FBF752F9681CC0B26188FBF786
:10ED68004DF90235EDB23368DB0208D497F8B836AE
:10ED7800002B3EF4A8ACF8F7F7F8FEF7A4BC094E50
:10ED880000242819C0B236F8021FFBF737F90D2CFA
:10ED9800ECD00134F5E700BF1804002090060020ED
:10EDA800E0220020E60C0020F403002010B5431EEA
:10EDB8000A44914204D011F8014B03F8014FF8E7D7
:10EDC80010BD02440346934202D003F8011BFAE740
:10EDD800704700000D4B30B51D6810F8013BEA186C
:10EDE800527802F00302012A11F8012B05EB020404
:10EDF80008BF2033647804F00304012C08BF2032D4
:10EE08009B1A01D1002AE8D1184630BD0401002020
:10EE180010B50246134601321C78002CFAD1013B8A
:10EE280011F8012B03F8012F002AF9D110BDC9B23E
:10EE3800034610F8012B1AB18A42F9D118467047D7
:10EE480000290CBF184600207047034613F8012B11
:10EE5800002AFBD1181A013870470000104B70B512
:10EE68001E680A44914217D010F8013BF4186478E0
:10EE780004F00304012C11F8014B06EB040508BF4C
:10EE880020336D7805F00305012D08BF20341B1BC6
:10EE980003D1002CE6D100E00023184670BD00BF66
:10EEA8000401002010B5034632B111F8014B03F8F4
:10EEB800014B013A002CF7D11A44934203D00021A8
:10EEC80003F8011BF9E710BD30B5037823B90B78B7
:10EED800002B18BF002030BD034601301A783AB124
:10EEE80000228C5C34B19D5CA542F5D10132F8E773
:10EEF800104630BD184630BD00210A2200F0E6B8A1
:10EF0800174B2DE9F0411D68AC6D06460F46FCB95C
:10EF1800502000F0E9F8A8658460AB6D0460446097
:10EF28001C61DC60AB6D9C615C61AB6DDC629C62FA
:10EF3800AB6D5C631C63AB6DDC639C63AB6D5C6445
:10EF48001C64AB6DDC649C64AB6D1C77AB6D5C6260
:10EF580030463946AA6D0123BDE8F04100F002B8F9
:10EF680068010020F0B548B9106838B9F0BD17F845
:10EF7800016B5EB1B542FAD12BB1204604460F466B
:10EF880014F8015BF3E714600370F0BD4DB9156028
:10EF98002846F0BD17F8016BAE4207D0002EF9D114
:10EFA8001C4623460F4613F8015BF3E715B1002111
:10EFB800217000E02B461360F0BD0123FFF7D2BF9C
:10EFC8002DE9F047404CD4F800900F463D4615F81F
:10EFD80001EB09EB0E04667806F0080404F0FF065E
:10EFE8000CB12F46F2E774462D2C03D1BD1C7C785A
:10EFF800012603E02B2C04BF7C78BD1C13B1102B19
:10F008000AD15AE0302C56D12C7804F0DF04582C61
:10F018004CD16C7810230235002E14BF4FF00048F5
:10F028006FF000480027B8FBF3FABE4603FB1A88C6
:10F0380009EB040C9CF801C01CF0040F01D0303C13
:10F048000BE01CF0030C1BD0BCF1010F0CBF4FF000
:10F05800370C4FF0570CCCEB04049C4210DAB7F194
:10F06800FF3F0AD0D64506D801D1444503DC03FB4F
:10F078000E4E012701E04FF0FF3715F8014BD7E797
:10F088007C1C73460AD1002E4FF0220114BF4FF0AA
:10F0980000436FF0004301602AB911E00EB1CEF1D0
:10F0A80000036AB107B1691E116009E03024002B22
:10F0B800B2D10823B0E70A23AEE7302CACD1A3E7DE
:10F0C8001846BDE8F08700BF0401002030B513469C
:10F0D800044A05460C46106829462246BDE83040D9
:10F0E800FFF76EBF68010020024B0146186800F068
:10F0F80003B800BF6801002070B5CC1C24F00304DD
:10F1080008340C2C38BF0C24002C064603DA0C23D8
:10F118003360002070BD8C42F9D3204A1368104632
:10F128001946A1B10A68121B0ED40B2A03D90A602A
:10F138008B188C501FE08B420DBF5A684A685A6082
:10F14800026018BF0B4616E00B464968E9E7144D04
:10F158002B681BB9304600F025F828603046214658
:10F1680000F020F8421C0346D1D0C51C25F0030549
:10F1780085420AD11C6003F10B001A1D20F007001C
:10F18800821A0AD05142995070BD3046E91A00F0EF
:10F1980009F80130BBD02B46ECE770BDD022002027
:10F1A800CC22002038B5064C0023054608462360CB
:10F1B80000F008F8431C02D1236803B12B6038BD66
:10F1C800E4220020044A05491368002B08BF0B46B7
:10F1D8001844106018467047D4220020E822002006
:10F1E80084B08DED010A019BC3F3C750A0F17F01E4
:10F1F8001E2927DC4A1C22DB16294FEAD3720ADDB6
:10F20800C3F3160343F40003963883405042434047
:10F21800981804B07047144BDDED017A03EB8203B4
:10F2280093ED007A77EE277ACDED037ADDED037A58
:10F2380077EEC77A17EE901A21F0004353B90020F1
:10F2480004B07047DDED017AFDEEE77A17EE900A1B
:10F2580004B07047C1F31603C1F3C75143F4000368
:10F26800C1F19601CB40D1E78036010800B510EE18
:10F27800103A134A23F00043934283B018DDB3F1E8
:10F28800FF4F04DB30EE400A03B05DF804FB68462C
:10F2980000F0AEFA00F001004000C0F101009DED61
:10F2A800000ADDED010A00F02FFF03B05DF804FB52
:10F2B800DFED040A012000F027FF03B05DF804FB2E
:10F2C800DA0F493F0000000010B52DED028B2A4CE3
:10F2D8008AB0F0EE408A00F0B3F894F900300133B8
:10F2E800B0EE408A04D0B0EE680A01F02DF928B9D2
:10F2F800B0EE480A0AB0BDEC028B10BDB0EE680A49
:10F3080001F0D2F8F7EE007AB4EEE70AF1EE10FA5F
:10F31800EEDD0123194A009318EE900A00230192AA
:10F328000893FDF73BFC02460B461548CDE904233C
:10F33800CDE9022300F0D4FF94F90030022B8DEDC3
:10F34800060B0FD0684600F0C7FF58B1089B73B989
:10F35800DDE90601FEF72CF900EE100A0AB0BDEC53
:10F36800028B10BD01F080F921230360EEE701F064
:10F378007BF9089B0360EBE76C01002088360108E5
:10F388009036010800F07EB910B52DED028B2A4C9D
:10F398008AB0F0EE408A00F073FB94F90030013334
:10F3A800B0EE408A09D0B0EE680A01F0CDF820B17D
:10F3B800F5EEC08AF1EE10FA05D4B0EE480A0AB0AC
:10F3C800BDEC028B10BD01231C4A009318EE900A75
:10F3D800002301920893FDF7E1FB2478CDE90401AD
:10F3E800CDE902019CB900220023CDE90623684635
:10F3F80000F072FFA8B1089BC3B9DDE90601FEF76A
:10F40800D7F800EE100A0AB0BDEC028B10BD002040
:10F41800002102460B46FDF73FFD022CCDE906010F
:10F42800E5D101F021F921230360E4E701F01CF99B
:10F43800089B0360E1E700BF6C01002094360108D7
:10F4480008B510EE102A22F00043B3F17E5F2DEDCF
:10F45800028B12D00ADCB3F17C5F19DAB3F10C5FCE
:10F468006ADCBDEC028B9FED760A08BD30EE400ADF
:10F4780080EE000ABDEC028B08BDBDEC028BDFED0F
:10F48800717A9FED710A002AC8BFB0EE670A08BDFD
:10F49800002AC0F28C80F7EE008A38EEC00AB6EE79
:10F4A800008A20EE088AB0EE480A00F0E9FADFED9B
:10F4B800677A9FED673A9FED674ADFED672ADFEDD0
:10F4C800673A9FED675ADFED674ADFED676ADFED60
:10F4D800675A9FED677AA8EE273AE8EE223AA3EE3C
:10F4E800084AE3EE884AA4EE085A10EE103AE5EE10
:10F4F800086A23F47F6323F00F03E4EE885A07EECB
:10F50800903AA6EE887AF0EE486AE5EE888AE7EE49
:10F51800E76AB0EE406A27EE088A30EE270A88EEDE
:10F52800288A86EE800AA8EE060ABDEC028B37EE22
:10F53800800A30EE000A08BD60EE007ADFED431A5B
:10F548009FED433A9FED434A9FED432ADFED433A4F
:10F558009FED436ADFED434A9FED435ADFED435A7F
:10F568009FED437ADFED436ADFED432AA7EEA13A28
:10F57800BDEC028BA3EE274AE7EE823AA4EE276A97
:10F58800E3EEA74AA6EE275AE4EEA75AA5EE277A95
:10F59800B7EE006AA5EEA76A67EE277AC7EE867A05
:10F5A800E0EE676A30EE660A32EEC00A08BDB7EED2
:10F5B800008A30EE080AF6EE007A60EE277ADFED70
:10F5C800232ADFED233A9FED243ADFED224A9FED0F
:10F5D800234ADFED235A9FED235ADFED236A9FED7F
:10F5E800236A9FED237AE7EEA23AA7EE834AE3EE79
:10F5F800A74AA4EE275AE4EEA75AA5EE276AE5EE35
:10F60800A76AA6EE278AA6EEA77AF0EE488A27EE22
:10F61800278AB0EE670A00F033FAC8EE287ADFEDE1
:10F62800176A9FED177AE7EE806AF0EE667A37EE92
:10F63800800AF0EE006AA0EE667AB0EE470A19E793
:10F64800DB0FC93F00000000DB0F494008EF11380D
:10F65800047F4F3A461124BD2EC69D3D613330BF0D
:10F66800A80A4E3E2D57014090B0A6BE39D119C008
:10F67800ABAA2A3E6821A233DA0FC93F6821A2B398
:10F68800DA0F494010B582B0CDED010A019B23F095
:10F698000042B2F1FF4FF0EE407A19DC10EE100A8A
:10F6A80020F00041B1F1FF4F12DCB3F17E5F49D089
:10F6B8009C1704F0020444EAD07479B9022C3ED0B5
:10F6C8009FED400A032C18BFB0EE670A02B010BDC8
:10F6D8009DED017A37EE270A02B010BD12B3B2F1E0
:10F6E800FF4F34D0B1F1FF4F1CD08A1AD2153C2AF3
:10F6F80022DC002B4BDB9DED017A87EE870A00F0B8
:10F70800D3FE00F0F5FD012C3AD0022C2FD0002CAE
:10F71800E2D09FED2D7ADFED2D7A30EE070A30EE3C
:10F72800670AD9E7DFED2A7A9FED2A0A0028A8BFE1
:10F73800B0EE670A02B010BD9FED250AE3E79FED22
:10F74800230AC9E702B0BDE8104000F0D1BDB1F10D
:10F75800FF4F21D0022CF2D0032C2AD0DFED1E7AE5
:10F768009FED1E0A012C08BFB0EE670AB4E79FEDB3
:10F77800167ADFED167A30EE070A37EEC00AABE7E5
:10F7880010EE103A03F1004300EE103AA4E73C32C1
:10F79800B1DA9FED120AB6E7022C10D0032C0BD079
:10F7A800DFED0F7A9FED0F0A012C08BFB0EE670A54
:10F7B80092E79FED040A8FE79FED0B0A8CE79FED18
:10F7C8000B0A89E7DB0F49C02EBDBB33DB0F49406D
:10F7D800DB0FC93FDB0FC9BF00000080000000003D
:10F7E800DB0F49BFDB0F493FE4CB16C0E4CB164023
:10F7F80070B510EE103A944A23F00044944286B053
:10F8080010EE106A054666DD904A94421ADC002B19
:10F81800DFED8F7A8F4A24F00F0440F3DD809442A5
:10F8280070EE677A66D09FED8C7A77EEC76A012012
:10F8380077EEE67AC5ED006A77EEC77AC5ED017A0C
:10F8480006B070BD854A944266DDB4F1FF4F49DACF
:10F85800E215863AA4EBC25307EE103AFDEEC76AEA
:10F86800DFED7F7AF8EEE66A37EE667ACDED036A69
:10F8780027EE277AFDEEC76AF8EEE66A37EE667A73
:10F88800CDED046A67EE277AF5EE407AF1EE10FACC
:10F89800CDED057A40F0B380F5EE406AF1EE10FA4E
:10F8A80014BF022301236F4902208DE8030003A837
:10F8B800294600F037F9002E12DA95ED007AD5EDD9
:10F8C800017AB1EE477AF1EE677A404285ED007A27
:10F8D800C5ED017A04E0002285ED000A42600020AF
:10F8E80006B070BD70EE407A0020C5ED017AC5ED16
:10F8F800007AF5E7DFED5C6A9FED5C7A77EEE67AF1
:10F90800012077EEC76A77EEE67AC5ED006A77EEF2
:10F91800C77AC5ED017AE3E700F0C6FDDFED546A6A
:10F92800DFED4B5A9FED4C7AF6EE007AE0EE267A40
:10F93800FDEEE77A17EE900AF8EEE76A1F28B1EEB7
:10F94800666AA6EE250A66EE877A1DDC494A411EDC
:10F9580024F0FF0352F82120934215D030EE677A45
:10F9680085ED007A30EE470A002E30EE670A85ED05
:10F97800010AB5DAB1EE477AB1EE400A85ED007AB0
:10F9880085ED010A4042ABE730EE677AE41517EEE1
:10F99800103AC3F3C753E31A082BE1DDDFED327ADF
:10F9A8009FED327AF0EE405AE6EE275A30EE650ABD
:10F9B800A6EE270AF0EE407AD6EE877A35EEE77A99
:10F9C80017EE103AC3F3C753E41A192C2CDC85ED53
:10F9D800007AB0EE650AC5E7944270EE277A10D037
:10F9E8009FED1D7A77EE876A4FF0FF3077EEE67A63
:10F9F800C5ED006A77EE877AC5ED017A70E70323D3
:10FA080051E7DFED196A9FED197A77EEA67A4FF084
:10FA1800FF3077EE876A77EEE67AC5ED006A77EE13
:10FA2800877AC5ED017A5BE79FED137A9FED135A4C
:10FA3800B0EE650AA6EE070A75EEC07AE6EE077A1A
:10FA4800D6EE857A8AE700BFD80F493FE3CB164048
:10FA5800800FC93FD00FC93F43443537800F494312
:10FA6800000080431C3701080044353708A3852E61
:10FA780084F9223F9C36010800A3852E32318D245B
:10FA880010EE103A23F00042B2F1FF4F70B430D2BA
:10FA98006AB3002B3DDBB2F5000F4FEAE3512CD3DC
:10FAA800A1F17F02C3F31603D10743F4000348BF53
:10FAB8005B00002456105B00254619214FF0807228
:10FAC800A818984202DC1B1A8518144401394FEA19
:10FAD80043034FEA5202F3D113B104F001031C446B
:10FAE800641004F17C5404EBC65300EE103A70BC69
:10FAF8007047A0EE000A70BC704713F400020DD1E5
:10FB08005B00180202F10102FAD5C2F101021144A8
:10FB1800C6E730EE400A80EE000AE8E70122114409
:10FB2800BEE700BF2DE9F04F2DED048BD7B05F1E67
:10FB3800D74C649D0293D31E48BF131D54F825600B
:10FB48000191DB1023EAE3736FEA030BB9190393FE
:10FB5800824602EBCB0BA3EB070314D41944659838
:10FB680001311AAA002BAABF50F82340DFEDCC7A46
:10FB780007EE904A03F10103A8BFF8EEE77A8B423B
:10FB8800E2EC017AEED1002E1ADB029B1AA9741C52
:10FB980001EB840442A89D00002FC0F2BA81DFED7A
:10FBA800C07A52464B1933ED017AF2EC016A994258
:10FBB800E6EE877AF7D10431A142E0EC017AEBD185
:10FBC800029ADFEDB48A9FEDB48A06F18043013BC7
:10FBD8009B00C2EB827906AA03F1040813449044FF
:10FBE80004934FEA89093446A50056AB2B44002CF0
:10FBF80013ED140A18DD42A94B1905AA60EE287AFC
:10FC0800B0EE407AFDEEE77A73ED016AF8EEE77A36
:10FC18008B42A7EEC87A37EEA60ABDEEC77A17EE72
:10FC2800100A42F8040FE9D1584600F0A9FCB0EEDA
:10FC3800409AB4EE000A29EE000A00F03DFCF2EE0C
:10FC4800007AA0EE679ABBF1000FFDEEC99AF8EEB4
:10FC5800E97A39EE679A40F34181601E06AACBF132
:10FC6800080352F8201041FA03F202FA03F30DF1E7
:10FC7800180EC91A4EF8201019EE900A1044CBF14C
:10FC8800070309EE900A1941002939DD19EE903A67
:10FC9800002C03F1010309EE903A40F3CB810022D6
:10FCA80010460DF1140E08E0C3F5807C13B1CEF8B0
:10FCB80000C00120013294420CDD5EF8043F0028A8
:10FCC800F2D00132C3F1FF039442CEF800304FF076
:10FCD8000100F2DCBBF1000F10DDBBF1010F00F0F9
:10FCE8000481BBF1020F09D1621E06AB0DF1180E9B
:10FCF80053F8223003F03F034EF82230022959D03E
:10FD0800B5EE409AF1EE10FA66D1631E9E420BDC06
:10FD180006AA1544002255F8040D454542EA00029A
:10FD2800F9D1002A40F07081731E06AA52F82330D8
:10FD3800002B40F07C81049B4FF0010E53F8042DFA
:10FD48000EF1010E002AF9D0A644631C73452FDC7E
:10FD5800039A9D18029A05F18045A0180EEB020C33
:10FD6800659A013D02EB85051AAA02EB800002EBB9
:10FD78008C0C42AA02EB830455F8043F07EE903A34
:10FD8800F8EEE77A002FE0EC017ADFED457A0BDB3D
:10FD9800524600EB0901034633ED017AF2EC016AA1
:10FDA8008B42E6EE877AF7D16045E4EC017AE3D13D
:10FDB800744619E7B7EE000A30EE499A00289FD03A
:10FDC8005846059100F0DCFB39EE409A0599B5EEEE
:10FDD800409AF1EE10FA98D0B0EE490ACBF1000043
:10FDE800029100F0CDFB9FED2C7A0299B4EEC70A80
:10FDF800F1EE10FAC0F27E81DFED267A60EE277A06
:10FE080006A8FDEEE77A631CF8EEE77A0BF1080B1B
:10FE1800A7EEC70AFDEEE77ABDEEC00A10EE102A7B
:10FE280040F8242017EE902A40F823205846B7EED1
:10FE3800000A0393029100F0A3FB039B0299002B95
:10FE4800C0F2C78003F1010E4FEA8E0242AC06A849
:10FE58009FED107A1044A71870ED017AF8EEE77A52
:10FE680067EE807A20EE070A67ED017AA742F3D1A0
:10FE7800043A17440025002EC0F2A880002DC0F2D5
:10FE8800A580064CDFED067A384600220CE000BF5C
:10FE9800343A01080000803B00008043403A0108E2
:10FEA80000000000AA4208DCF4EC016AB0EC017A18
:10FEB80001329642E6EE877AF4DA56AA02EB850218
:10FEC80001357545A7F1040742ED287AD3D1649A24
:10FED800032A5FD8DFE802F0673737B010D1631E16
:10FEE80006AA52F823100912CEE6621E06AB0DF1DF
:10FEF800180E53F8223003F07F034EF82230FDE647
:10FF0800F6EE007AB4EEE79AF1EE10FA0ADA00217A
:10FF1800F6E65FED1D7A0431A142E0EC017A7FF448
:10FF28003BAE4DE619EE903A002C03F1010309EEC1
:10FF3800903AC8BF02213FF7B2AEF7EE007A37EE2B
:10FF4800C99A0221DCE62EAA5FED2B7A02EB8E0E0F
:10FF58003EED017A964577EE877AF9D1002943D0AC
:10FF6800DDED2E6A019AB1EE677A002B76EEE77A1C
:10FF780082ED007A09DD2FA80122B0EC017A013266
:10FF8800934277EE877AF8DA09B1F1EE677A019B46
:10FF9800C3ED017A19EE903A03F0070057B0BDECB3
:10FFA800048BBDE8F08F2EAA5FED437A02EB8E0E2C
:10FFB8003EED017A013B5A1C77EE877AF8D109B1F8
:10FFC800F1EE677A019BC3ED007AE3E75FED4C7AC7
:10FFD80073E7649A032ADDD8DFE802F0130202808F
:10FFE8005FED517A0029BBD19DED2E7A019A002B45
:08FFF800C2ED007A77EE677A92
:020000040801F1
:10000000BDDC019BC3ED017AC8E75FED597ADAE701
:1000100006AAABF1080B52F82320002A7FF40AAF9E
:1000200006AA02EB830252F8040D013BABF1080B68
:100030000028F8D0FEE64FF0010E89E600204DE6DC
:10004000002B4FDD9A0056A810442EAD141D10ED64
:10005000287A2C44A81870ED017A77EE276AA84216
:1000600077EEE67A77EE277AB0EE667A64ED017A7B
:10007000C0ED006AEFD1012B34DD131D56AC1444E2
:10008000034414ED287A02442FAC184672ED017A2D
:1000900077EE876AA24277EEE67A77EE877AB0EE5D
:1000A000667A60ED017AC2ED006AEFD15FED827A87
:1000B00030AA33ED017A934277EE877AF9D1A9B16C
:1000C000DDED2E6A9DED2F7A019AF1EE677AF1EE61
:1000D000666AB1EE477AC2ED027AC2ED006A82ED3D
:1000E000017A5BE75FED907A0029E9D101982E9AB9
:1000F0002F9BC0ED027A026043604FE7BDEEC00A5D
:1001000006A810EE102A234640F8242092E600BFED
:1001100008B510EE103A23F00042B2F1465F2DED23
:10012000028BB0EE407A12DAFDEEC07A17EE901A2A
:1001300019BB431C134300F0AA80012800F08480FF
:10014000BDEC028BBFEE000A80EE070A08BD5349E2
:100150008A4212DD002BB8BFB1EE407ADFED507A53
:100160009FED500AB8BFF1EE600A77EEE07A30EE0C
:10017000477ADFED4D0A37EE277A67EE076A9FED83
:100180004B8A9FED4B2ADFED4B8ADFED4B1A9FED3B
:100190004B3ADFED4B2A9FED4B4ADFED4B3A9FED9B
:1001A0004B5ADFED4B4A9FED4B6ADFED4B5A9FED0B
:1001B0004B0A3A4966EEA67A26EE871AA7EE882AF7
:1001C0008A42E7EEA81AA2EE273AE1EEA72AA3EEAA
:1001D000274AE2EEA73AA4EE275AE3EEA74AA5EE95
:1001E000276AE4EEA75AF0EE467AE5EEA67AB0EE7C
:1001F000606AA7EE816AE6EE260AE1EE000A37EEB3
:10020000200A24DC01281FD0FFEE006AC6EE806AB7
:1002100010EE103A16EE902A23F47F6322F47F62E8
:1002200023F00F0322F00F0200EE102A06EE103A20
:10023000F7EE007AE6EE007A36EE477A70EEC70AFD
:10024000E0EE807AA7EEA60ABDEC028B08BD07EEB1
:10025000900AB8EEE76A60EE006A70EE067A9B17C5
:10026000C6EEA77A03F00203C3F10103BDEC028BD3
:10027000F0EE005A77EEE00A00EE103A37EE607AC0
:10028000F8EEC06AA7EE656A26EE860A08BD00F0A1
:100290000FF9B7EE007A87EE000AD5E73FA12C3FB1
:1002A00068212233DA0F493F000000005FAE9BB7A0
:1002B00045F4A3388453D9377AC09538C8261A3AFA
:1002C000B937813916696B3B48DEBE3AA427B33C87
:1002D0001F37113C8988083ED10D5D3DABAAAA3E6F
:1002E00000207047000000009FED010B704700BF29
:1002F000000000000000F87F38B510EE105A25F01D
:100300000044B4F1A14FF0EE407A0BDBB4F1FF4FA3
:1003100058DCDFED547A9FED540A002DC8BFB0EED3
:10032000670A38BD514B9C425DDCB4F1445F4CDB45
:100330004FF0FF3367EEA75A9FED4D1A9FED4D2A00
:100340009FED4D3ADFED4D1ADFED4D2A9FED4D4A01
:10035000DFED4D3A9FED4D5ADFED4D4A9FED4D6A71
:10036000DFED4D6A25EEA57A5A1CA7EE012AE7EECD
:10037000212AA2EE073AE2EE873AA3EE074AE3EE1D
:10038000874AA4EE075AE4EE876AA5EE076A26EECE
:10039000877A66EE256A3ED0404A41499B001A445E
:1003A00076EE876A92ED007A96EEA77A0B44002DDE
:1003B00093ED000A77EE677A70EE677A28DBB0EE8D
:1003C000670A38BD30EE000A38BD9FED367A30EE50
:1003D000077AF7EE006AB4EEE67AF1EE10FAA7DDDE
:1003E000B0EE670A38BD00F063F82F4B9C4219DC71
:1003F000A3F5D0039C422ADCF0EE007ABFEE007A2F
:10040000A0EE277A002370EE277AC7EE277A91E7CD
:10041000B1EE670A38BD76EE876AB0EE670AA6EEDF
:10042000E70A38BD214B9C420BDCF7EE087AB7EEA9
:10043000007AA0EE277A022370EE677AC7EE877AF9
:1004400078E7FFEE007AC7EE807A032372E7F7EED3
:10045000007A30EE677A70EE277A0123C7EE277AAA
:1004600068E700BFDB0FC93FDB0FC9BFFFFFDF3EFF
:10047000D769853C59DA4B3D356B883D21A215BDC6
:100480006BF16EBD6E2EBA3D95879DBD2549123E1E
:10049000388EE3BDABAAAA3ECDCC4CBE6C3A010867
:1004A0007C3A0108CAF24971FFFF973FFFFF1B40EA
:1004B00010EE103A23F0004300EE103A704700BFF0
:1004C00010EE102A22F00041CB0D7F3B162B17DCDB
:1004D000002B10EE100A19DB1A491941114222D0E3
:1004E000DFED197A70EE277AF5EEC07AF1EE10FAA8
:1004F00019DD002A18DB20EA010300EE103A7047EC
:10050000B1F1FF4F0FD330EE000A7047DFED0E7AE6
:1005100070EE277AF5EEC07AF1EE10FA03DD002ACC
:1005200008DB9FED0A0A70474FF4000242FA03F31A
:100530001844E0E70029FFEE007A18BFB0EE670A22
:10054000704700BFFFFF7F00CAF249710000000042
:1005500010EE103A33F0004001D102207047A0F5B0
:100560000003B3F1FE4F01D204207047054B421E39
:100570009A4201D803207047A0F1FF40B0FA80F002
:1005800040097047FEFF7F0008B510EE103A33F0C7
:1005900000422DED028B11D0B2F1FF4F11D2B2F516
:1005A000000F13D3D20D0244FE2A2EDC002A1ADDDE
:1005B00023F0FF4343EAC25300EE103ABDEC028B36
:1005C00008BDBDEC028B30EE000A08BD1D4BDFED0F
:1005D0001E7A984220EE270A22DB10EE103AC3F36F
:1005E000C752193ADFE712F1160F1EDA4CF25033F8
:1005F00098420ADC9FED158AF0EE400AB0EE480AF8
:1006000000F02AF820EE080AD8E79FED118AF0EEF4
:10061000400AB0EE480A00F01FF820EE080ACDE7C5
:10062000DFED0A0A20EE200AC8E7193223F0FF4363
:1006300043EAC253DFED077A00EE103A20EE270AB4
:10064000BCE700BFB03CFFFF0000004C6042A20DC1
:10065000CAF249710000003310EE103A23F0004254
:1006600010EE903A03F00043134300EE103A704747
:10067000014B1868704700BF680100200004004863
:1006800010000102000400482000010200100402D2
:1006900008001102C0060108A8060108A606010804
:1006A000A4060108FFFFFFFF0A0100030103020384
:1006B0000303040305030603070308030903FFFFFD
:1006C00000030103020303030403050306030703F6
:1006D00008030903FFFF0000524F4C4C3B504954A4
:1006E00043483B5941573B414C543B506F733B503F
:1006F0006F73523B4E6176523B4C4556454C3B4DD9
:1007000041473B56454C3B0000000000C220010819
:100710000000000001000000C720010801000000E7
:1007200002000000CE2001080200000003000000CB
:10073000D72001080300000004000000DD200108AC
:100740000500000005000000E2200108060000008E
:1007500006000000EC200108070000000700000070
:10076000F52001080800000008000000FE20010834
:100770000900000009000000072101080A0000002C
:100780000A000000112101080B0000000B0000000E
:100790001B2101080C0000000C00000025210108AD
:1007A0000D0000000D0000002D2101080E000000CA
:1007B0000E000000352101080F0000000F000000AE
:1007C0003D21010810000000100000004621010832
:1007D00011000000110000004D210108120000006E
:1007E0001200000057210108130000001300000050
:1007F0005F21010814000000140000006A210108B4
:10080000150000001500000074210108160000000A
:10081000160000007B2101081700000017000000EF
:100820008321010818000000180000008B21010836
:100830001900000019000000932101081A000000AF
:100840001A0000009D2101081B0000001B00000091
:1008500000000000FF000000010001020001030091
:100860000104000105000106000107000108000164
:100870000900010A00010B00010C01030D00010E2B
:1008800000010F000110000111000112000113000E
:1008900001140001000100006168730000010303FE
:1008A000010200000000000080250000004B000055
:1008B0000096000000E1000000C201000084030077
:1008C00090D00300118B00089D8B0008B18B0008AD
:1008D000AF8B0008A98B0008AD8B00080327010827
:1008E0000C270108000000008D730008282701086C
:1008F0002C270108000000008F720008582C010806
:100900003C27010800000000E9C20008592701083F
:100910005E270108712701089582000882270108D7
:100920000000000000000000F17F00088727010898
:100930008F270108A2270108F57E0008B5270108C6
:10094000B9270108AE2701089DC00008CC2701087F
:100950000000000000000000697D0008D1270108A8
:10096000D5270108F0270108517E00080228010858
:10097000F827010808280108AD7D0008162801089D
:100980001B28010800000000FD8800083628010827
:100990002E2801083C2801089DBC00084E280108AB
:1009A0000000000059280108FDBB00086C28010860
:1009B0006528010874280108BDBB00087E280108CD
:1009C0008A2801087428010875BB00089E280108C0
:1009D000A628010800000000A9810008C22801081B
:1009E000C928010800000000F1740008E728010888
:1009F000EC2801080000000005C30008FC280108DD
:100A000003290108000000004D7600087F3101082D
:100A10001A2901080000000065800008312401083F
:100A20002B2901083A290108F5C000084B290108C3
:100A3000502901085C290108E1850008D029010836
:100A4000CB29010800000000B1BF0008DC29010823
:100A5000D72901080000000041BB0008A12A0108B5
:100A6000E4290108EA290108F0290108F32901080D
:100A7000FA290108FD290108022A01080E2A0108A5
:100A8000112A0108172A01081E2A0108282A01082C
:100A9000922A0108322A0108402A01084C2A01083A
:100AA000532A0108592A0108662A0108712A0108F7
:100AB0007E2A0108852A01088C2A01089B2A010840
:100AC00000000000342601083B26010840260108EA
:100AD000512601085B2601086626010871260108D7
:100AE0007C26010880260108892601088F26010836
:100AF00099260108A7260108AA260108BA26010896
:100B0000C1260108CA260108D4260108DC260108EE
:100B1000E7260108F02601080000000000000000A0
:100B20000000000001000000621101080000000048
:100B300000000000000000000000000004000000B1
:100B400046110108020000003811010800000000F1
:100B50000000000000000000000000000500000090
:100B60001511010800000000000000000000000056
:100B70000000000000000000000000000000000075
:100B80000000000000000000000000000500000060
:100B9000F21001080000000000000000000000004A
:100BA0000000000000000000000000000000000045
:100BB0000000000000000000000000000200000033
:100BC000E410010808000000AC100108000000005B
:100BD0000000000000000000000000000000000015
:100BE0000000000000000000000000000000803F46
:100BF000000000000000803F0000803F0000803FB8
:100C0000000080BF000080BF000000000000803FA7
:100C1000000000000000803F000080BF0000803F17
:100C20000000803F000080BF000000800000803F87
:100C30000000000000000000000080BF0000803FB6
:100C400000000000000000000000803F0000803F26
:100C5000000080BF0000803F000080BF0000803F98
:100C6000000080BF000080BF0000803F0000803F88
:100C70000000803F0000803F0000803F0000803F78
:100C80000000803F000080BF000080BF0000803F68
:100C90000000000000000000000000000000803F95
:100CA0000000000000000000000000000000803F85
:100CB000E17A14BFE17A143F0000803F0000803FDA
:100CC0001F85EBBE14AEC7BE000000BF0000803F12
:100CD000E17A143FE17A143F000080BF0000803FBA
:100CE0001F85EB3E14AEC7BE0000003F0000803FF2
:100CF0000000803F240FD4BE0000803F0000803FF2
:100D0000240FD4BE000080BF0000803F0000803F61
:100D1000000080BF240FD43E0000803F0000803FD1
:100D2000240FD43E0000803F0000803F0000803F41
:100D3000240FD43E000080BF000080BF0000803F31
:100D4000000080BF240FD4BE000080BF0000803FA1
:100D5000240FD4BE0000803F000080BF0000803F11
:100D60000000803F240FD43E000080BF0000803F81
:100D7000F704353FF70435BF0000803F0000803F97
:100D8000F70435BFF70435BF0000803F0000803F07
:100D9000F70435BFF704353F0000803F0000803F77
:100DA000F704353FF704353F0000803F0000803FE7
:100DB00000000000000080BF000080BF0000803FF6
:100DC000000080BF00000000000080BF0000803FE6
:100DD000000000000000803F000080BF0000803F56
:100DE0000000803F00000000000080BF0000803F46
:100DF000000080BF0000803F000080BF0000803FF7
:100E0000000080BF000080BF0000803F0000803FE6
:100E10000000803F0000803F0000803F0000803FD6
:100E20000000803F000080BF000080BF0000803FC6
:100E3000000080BF0000803F0000803F0000803F36
:100E4000000080BF000080BF000080BF0000803F26
:100E50000000803F0000803F000080BF0000803F16
:100E60000000803F000080BF0000803F0000803F06
:100E7000000000BFD0B35D3F0000803F0000803F16
:100E8000000000BFD0B35DBF0000803F0000803F86
:100E90000000003FD0B35D3F000080BF0000803FF6
:100EA0000000003FD0B35DBF000080BF0000803F66
:100EB000000080BF00000000000080BF0000803FF5
:100EC0000000803F000000000000803F0000803FE5
:100ED000000000000000803F000080BF0000803F55
:100EE000000080BF000080BF000000000000803FC5
:100EF000000000000000803F0000803F0000803FB5
:100F00000000803F000080BF000000000000803F24
:100F10000000000000000000000000000000803F12
:100F2000D0B35DBF0000003F0000803F0000803F65
:100F3000D0B35DBF000000BF000080BF0000803F55
:100F4000D0B35D3F0000003F0000803F0000803FC5
:100F5000D0B35D3F000000BF000080BF0000803FB5
:100F600000000000000080BF0000803F0000803FC4
:100F7000000000000000803F000080BF0000803FB4
:100F800000000000A8AAAA3F0000803F0000803FA8
:100F9000000080BFB0AA2ABF000080BF0000803FD1
:100FA0000000803FB0AA2ABF000080BF0000803F41
:100FB00000000000A8AAAA3F000080BF0000803FF8
:100FC000000080BFB0AA2ABF0000803F0000803F21
:100FD0000000803FB0AA2ABF0000803F0000803F91
:100FE0000000803F00000000000000000000803F83
:100FF000000080BF00000000000000000000803FF3
:10100000000080BF0000803F000080BF0000803FE4
:10101000000080BF000080BF0000803F0000803FD4
:101020000000803F0000803F0000803F0000803FC4
:101030000000803F000080BF000080BF0000803FB4
:10104000000000000000803F000080BF0000803FE3
:10105000000080BF000000000000803F0000803FD3
:101060000000803F000000000000803F0000803F43
:1010700000000000000080BF000080BF0000803F33
:1010800000000000A8AAAA3F000000000000803F66
:10109000000080BFB0AA2ABF000000000000803F0F
:1010A0000000803FB0AA2ABF0000000003026400D5
:1010B0000064000301640000640004026400006432
:1010C000000401640000640005026400006400057F
:1010D000006400006400060264000064000600640E
:1010E0000000640004016400006400050064000066
:1010F00064000300640000640004006400006400F5
:101100000502640000640006016400006400070337
:1011100064000064000300640000640003016400D4
:1011200000640004009C000064000401640000648A
:101130000007036400006400000C7D0000640001EF
:101140000D7D00006400040264000064000401647A
:1011500000006400050264000064000501640000F2
:10116000640005026400006400000000319700087C
:10117000DF9600089996000863970008C996000852
:101180005D970008E5A20008E5A2000871C4000808
:10119000E5A20008E5A20008E5A20008E5A2000813
:1011A000BDC40008E5A20008E5A20008E5A2000809
:1011B000E5A20008E5A20008E5A20008040100007D
:1011C0000001000001000000D01E0108682C010889
:1011D00002010000BD1E0108782C01080302000076
:1011E000BA1E0108882C010804030000B51E01087E
:1011F000902C010805040000B01E0108932C010882
:1012000006050000A71E01089A2C01080706000029
:10121000A41E0108A92C010808070000A11E01084E
:10122000B62C01080908000056220020000000002A
:101230000A0900009E1E0108BE2C01080C0A0000CD
:10124000991E0108C52C01080D0B0000941E010811
:10125000D52C01080E0C0000851E0108EA2C01089F
:101260000F0D000056220020000000000B0E0000B1
:10127000811E0108F52C0108100F00007C1E0108DA
:10128000032D0108BE340108C1340108C934010826
:10129000D2340108573501085C3501086035010872
:1012A00069350108892601087C2601086535010891
:1012B000000000006C200108DE340108E33401085E
:1012C000EB340108F4340108FC340108033501084B
:1012D0000B35010813350108000000000000000074
:1012E0006C200108DE34010818350108E3340108D8
:1012F00020350108283501082F350108033501087C
:101300000B35010813350108000000006C200108AE
:10131000DE3401083A3501084135010800000000BB
:1013200000000000000000000000000000000000BD
:1013300000000000000000006C200108DE340108FD
:101340004835010850350108000000000000000089
:10135000000000000000000000000000000000008D
:1013600000000000092D010844000000601A002060
:1013700000000000A00F0000122D01084100000035
:10138000631A00200000000001000000242D010865
:1013900041000000621A002000000000010000006F
:1013A000322D010841000000641A002000000000F6
:1013B000010000003F2D010844000000EC1B00204C
:1013C000B0040000A4060000462D010844000000FF
:1013D000EE1B002000000000D0070000502D010887
:1013E00044000000F01B002000000000D0070000B7
:1013F0005A2D010842000000E81B002000000000F8
:1014000012000000672D010841000000E91B0020C8
:1014100001000000FF000000722D010842000000E2
:10142000EA1B00200000000001000000822D0108DE
:10143000420000002A1C0020000000000100000003
:101440003831010844000000981B00200000000013
:10145000D0070000972D0108440000009A1B0020CF
:1014600000000000D0070000A42D01084400000087
:101470009C1B002000000000D0070000B02D0108D8
:10148000440000009E1B002000000000D007000068
:10149000C32D010844000000A01B00200000000034
:1014A000D0070000D32D010844000000A21B00203B
:1014B00000000000D0070000E42D010844000000F7
:1014C000A41B002000000000D0070000EF2D010841
:1014D00044000000A61B002000000000D007000010
:1014E000042E010844000000A81B00203200000068
:1014F000007D0000132E010844000000AA1B0020FC
:1015000032000000F2010000222E0108410000001C
:10151000341C002000000000010000002F2E0108F4
:1015200041000000351C0020000000000100000008
:10153000422E010841000000361C0020000000007F
:101540003C000000542E010841000000371C002020
:1015500000000000B4000000602E010842000000FE
:10156000421C0020FFFFFFFF01000000762E010853
:1015700041000000441C0020300000007E000000FC
:10158000872E010841000000E61B0020000000003B
:1015900006000000992E010841000000E71B002012
:1015A000000000000A000000AB2E0108410000000E
:1015B000681C00200000000001000000BC2E010893
:1015C00041000000691C0020000000000100000034
:1015D000D02E0108600000006C1C0020A6FFFFFF59
:1015E0005A000000E82E010860000000701C002076
:1015F0004CFFFFFFB4000000002F01084100000075
:10160000741C00200000000001000000192F0108D8
:1016100041000000751C00200000000001000000D7
:10162000242F010841000000761C0020000000006B
:1016300001000000392F010841000000771C002044
:101640000000000078000000532F01084400000053
:10165000DC1B002000000000204E0000642F010869
:1016600041000000D01B002000000000FF0000002F
:101670006F2F010841000000D31B00200A0000006A
:1016800032000000852F010841000000D41B00201B
:101690000A000000320000009B2F010841000000FA
:1016A000D51B00200A00000032000000B52F010801
:1016B00048000000D61B0020F0D8FFFF10270000D4
:1016C000C92F010844000000D81B002000000000C2
:1016D000E40C0000DE2F010841000000DB1B0020AD
:1016E0000000000001000000FC2F01084100000084
:1016F000DA1B002000000000020000000F3001088B
:1017000041000000AC1B00200000000008000000A9
:101710001A30010841000000AD1B0020000000004D
:10172000080000002430010841000000AE1B00202A
:1017300000000000080000002E30010848000000F2
:10174000B01B00204CFFFFFF680100003F30010884
:1017500048000000B21B00204CFFFFFF68010000A2
:101760005130010848000000B41B00204CFFFFFF6F
:10177000680100006130010844000000C21B002025
:10178000640000008403000077300108440000007A
:10179000B81B00200000000000010000803001089C
:1017A00041000000BE1B002000000000800000007F
:1017B0009030010844000000BA1B002064000000C3
:1017C000E8030000A130010844000000BC1B002019
:1017D00064000000E8030000B3300108810000004D
:1017E0008B1D002001000000FA000000C530010838
:1017F000810000008C1D002000000000010000009E
:10180000BC30010881000000891D0020000000009C
:1018100020000000DA300108810000008A1D00204D
:101820000000000064000000E730010881000000B3
:10183000901D00200000000096000000013101080A
:10184000840000008E1D00200100000084030000C1
:101850001B31010842000000B61B0020FFFFFFFF04
:10186000010000003131010841000000381C002057
:1018700000000000010000004531010842000000A6
:10188000391C0020FFFFFFFF010000005931010853
:10189000440000003A1C002050000000F401000049
:1018A00073310108420000003C1C002000000000D1
:1018B0000100000085310108480000003E1C0020A6
:1018C0000A00000090010000983101084200000069
:1018D000401C00200000000001000000AD310108A4
:1018E00081000000CC1C002000000000020000006D
:1018F000C2310108010100001E210020000000008B
:10190000FA000000CA310108010100001F21002077
:101910000000000064000000D23101080101000055
:10192000262100200000000064000000DE310108D4
:1019300001010000202100200000000064000000E0
:10194000E631010801010000212100200000000013
:1019500064000000EF310108010100002221002095
:101960000000000064000000F931010801010000DE
:101970002321002000000000640000000432010860
:10198000010100002421002000000000FF000000F1
:101990000D32010801010000252100200000000097
:1019A0006400000016320108040100002821002014
:1019B000E8030000D00700002532010841000000C4
:1019C0002C1C002000000000C80000003432010878
:1019D000410000002D1C002000000000C800000095
:1019E00047320108440000002E1C0020E8030000DC
:1019F000D00700005932010841000000301C0020CF
:101A000000000000010000006E32010844000000E8
:101A1000321C0020000000002C0100008A32010866
:101A200044000000F21B0020EE020000CA08000083
:101A30009632010844000000F41B0020EE02000072
:101A4000CA080000A232010881000000011E002027
:101A50000000000001000000AE320108410000005B
:101A6000B71B00200000000009000000BB32010885
:101A700081000000D41C002000000000FA000000DB
:101A8000CA32010881000000DC1C002000000000B8
:101A900064000000D932010881000000DD1C002034
:101AA0000000000064000000E7320108A000000010
:101AB000D81C00200100000014000000F7320108CB
:101AC00081000000F01C0020000000000100000068
:101AD0000633010888000000D21C0020D4FEFFFF5E
:101AE0002C0100001533010888000000D01C0020E4
:101AF000D4FEFFFF2C010000233301088100000009
:101B0000E01C00200000000030000000313301081C
:101B1000A0000000E41C0020000000000100000004
:101B200040330108A0000000E81C00200000000075
:101B3000010000004C330108A0000000EC1C002054
:101B400000000000010000005833010841000000BF
:101B5000C01B0020000000000400000066330108E4
:101B600041000000BF1B0020000000000300000037
:101B70007333010888000000CE1C0020B0B9FFFFBD
:101B8000504600008333010881000000781C0020CB
:101B900000000000050000009233010881000000F1
:101BA0007A1C002000000000C80000009A330108E1
:101BB00081000000841C002000000000C80000001C
:101BC00049300108810000008E1C00200000000048
:101BD000C8000000A233010881000000791C002029
:101BE00000000000C8000000A933010881000000C7
:101BF000831C002000000000C800000038300108ED
